:1000000000400020A9630000E9630000EB630000EA
:1000100000000000000000000000000000000000E0
:10002000000000000000000000000000ED63000080
:100030000000000000000000EF630000F16300001A
:10004000F3630000ED4A000025680000F363000040
:10005000F363000000000000F3630000F36300009E
:10006000F3630000F56A0000CD2C0000F36300008C
:10007000F3630000F3630000F3630000F363000028
:10008000F36300008D6C0000F3630000F363000075
:10009000F3630000F3630000F3630000F363000008
:1000A000F3630000F36300000000000000000000A4
:1000B0000000000000000000000000000000000040
:1000C00010B5064C2378002B07D1054B002B02D02E
:1000D000044800E000BF0123237010BD600200202F
:1000E00000000000FCDD0000044B10B5002B03D025
:1000F0000349044800E000BF10BDC04600000000F6
:1001000064020020FCDD0000164B002B00D1144BD4
:100110009D46402292029A1A924600218B460F4633
:100120001348144A121A0AF059FB0F4B002B00D047
:1001300098470E4B002B00D0984700200021040068
:100140000D000D48002802D00C4800E000BF0AF066
:1001500005FB2000290006F083FB0AF0D9FAC0460F
:100160000000080000400020000000000000000027
:1001700060020020982F0020000000000000000016
:100180000123034010D104280CD90268120909D0B8
:10019000531E9B001A1DC1180979002902D0013392
:1001A0009342F8D1180070470023FBE70378002B37
:1001B00003D05AB2002A01DB013070473F2293433B
:1001C000C03B59424B41C01803789343802BF4D174
:1001D0000130F9E710B500240378002B01D120008D
:1001E00010BDFFF7E3FF0134F6E770B5002204000D
:1001F0000D00411C092003F079F8002806D00123E6
:100200006200134343600023A34200DB70BD9A00E9
:10021000A958821891600133F6E770B5012803DC14
:100220001C2000F0A5FE70BD01230D6811201D42A9
:10023000F7D04868184206D1042804D90F23026871
:100240001340042B01D00E20EBE702F0B9FE6D1035
:100250000400002D03DDFFF7BDFFA84206DA1220DF
:10026000DFE72000FFF7A2FF0400013D012DF8D1D8
:1002700020787F2809DDDF280BDCF8233F22DB0014
:10028000800118406378134018430123400018434D
:10029000C9E7EF280BDCFC22637812019B011340B5
:1002A0003F220007000C0343A0781040ECE7F7283A
:1002B00012DCFC22637892021B031340E0228004CC
:1002C000520310403F221843E3781340FC220343BB
:1002D000A07812018001E8E701204042D5E7F0B59F
:1002E000070085B00D001C20012F06DD4C6801239E
:1002F00022001A40019203D10D2000F039FE54E093
:10030000022F02D08A681A42F6D001232E681E42BC
:1003100000D07EE0042E00D87BE01C41002C00DCE5
:100320001C000F2332681340092B29D173685B101E
:100330000193022F05D0AB68019A5B109A4200DD51
:100340000193019B01221F1B0137FB43DB171F4059
:10035000791C092002F0CAFF061E09D001237F0084
:100360001F4303002A68083347600199A14202DA5B
:10037000300005B0F0BD0134A100515802C3F4E7CC
:10038000042B46D1300002F01BFEFFF723FF029042
:10039000022F04D0AB685B10984200DD0293029BF1
:1003A0009C4204DD002003F00DF80600E0E7300079
:1003B00002F006FE0700019B9C4222DC3000019700
:1003C00002F0FEFD03903800FFF7F0FE029B0134BF
:1003D0000700A342F7DA019BC71A380002F0F2FFC8
:1003E000061EC5D002F0ECFD0400286802F0E8FD0E
:1003F000039A019B991A41183A0020000AF0D2F999
:10040000B6E73800FFF7D2FE019B070001330193E6
:10041000D1E7212071E7F8B54D680F00EB0706D44E
:10042000042D04D90F232E683340092B03D00B2051
:1004300000F09EFDF8BD6B6836095C10731EA34288
:100440000FD80321200008F085F86421642803DC1C
:100450000100032800DA03212800891902F076FF41
:1004600005002B6800201B09013B9C42E2D23A6840
:10047000A31C9B005A510123013464001C436C608F
:10048000D8E7F0B585B0012803DC1C2000F070FD32
:100490002AE001244D682200022806D08B682342FE
:1004A00003D05C10002C00DC140001231D4200D09E
:1004B00073E0042D00D870E00F272B680E683B40D6
:1004C000042B27D1033B1E4205D1042E03D93368E8
:1004D0001F40042F01D00E20D8E72800FFF750FE60
:1004E000A04203DA0120404205B0F0BD280002F02E
:1004F00067FD0700300002F063FD013C0100381980
:100500000AF079FD0028EDD00123C01B0130400026
:100510001843E9E7092B40D16B685B1000939C42BC
:10052000E0DC01231E4230D1042E2ED933683B403B
:10053000042B2AD1300002F043FD012302900193E5
:100540000397671CBB00E858864203D101986400FA
:100550002043C9E7019B18420ED104280CD9036837
:10056000039A1340042B07D102F02AFD01000298E0
:100570000AF01CFD0028E9D0009B3C009F42E0DD12
:10058000B0E71C00009B9C42ACDC631C9A00AA589C
:10059000B242F6D164000120DAE7212076E710B5F7
:1005A00002F0F2FC43000120184310BD10B57F2972
:1005B00002DC0170013010BD1A4B99420CDC402363
:1005C0008A115B42134303703F230B408021494251
:1005D000194341700230EEE7134B994210DC20239F
:1005E0000A135B4213433F24802203708B11524253
:1005F0002340214013430A43437082700330DAE7FB
:100600000A4B9942D7DCF0230370603B4370113BE7
:100610008A11FF3B1A4382703F2211401943C17077
:100620000430C8E7FF070000FFFF0000FF0F0100D4
:10063000F0B50D0085B0002803DC1C2000F098FC0C
:100640000DE009680122080010400AD002AC1141F7
:100650002000FFF7ABFF011B200002F0BFFE0400EB
:100660001AE004293FD90F230C682340092B3AD103
:100670004B685B10019303239C46019B9A420EDD5D
:1006800002F0A0FE041E07D02E68012502F098FC9F
:100690002F00019B9D421DDD200005B0F0BD013201
:1006A0009300CC580123234001D10D20C6E76410EC
:1006B0007F2C0DDD0D4E0223B44209DD0C4E634646
:1006C000B44205DD00270B4EE30FA6427B419B00A1
:1006D000C018D2E70135AB00F1583942E5D04910D6
:1006E000FFF764FFD5E72120A8E7C046FF07000019
:1006F000FFFF0000FF0F010010B5040001200840BB
:1007000010D104290DD90F230A681340042B08D1F6
:10071000080002F055FC010020000AF047FC4342AB
:10072000584110BD0020FCE7F7B50F00012803DC9D
:100730001C2000F01DFCFEBD01264D682E4006D198
:10074000042D04D90F222B681A40092A01D00B204E
:10075000EFE76A681B095410A34200D85C1E396891
:100760001E48FFF7C9FF01230190002813D1396803
:100770001B48FFF7C1FF002811D0002C0DD001232A
:10078000621C013C9C409200535123436B6004E087
:100790000136B200AB50B442FADA0020CBE73B6836
:1007A0000D20DA07C5D55B10002B11DD9C420FDB55
:1007B0009B00A200291DEB1889180433994209D126
:1007C0000123013C9C40AA181C4353606C60E4E781
:1007D0001220AEE758681860EFE7C0463FC7000038
:1007E00043C70000002310B50C000B70C30705D5EC
:1007F0000D49421020000AF035FB08E00B490028A3
:1008000002D0042804D10A4920000AF0C1FB10BD1F
:100810000428FCD90F2302681340042BF7D102F0FF
:10082000CFFB04490200E5E7F4CF000048C7000011
:100830004EC7000053C70000F0B593B0039003000B
:1008400002911C20012B1DDD029B01251B681C0051
:100850002C4000D0A8E0042B00D8A5E01A680F2394
:100860001A40092A48D10194019A029992008A58A3
:1008700016002E4005D1042A03D910681840092813
:1008800004D0222000F074FB07002CE052685210C4
:10089000A418019A013201920199039A8A42E3D184
:1008A000611C012202F022FD071E01D100271AE07F
:1008B00064002543456005000835029AB300D1580D
:1008C0004B680A685B1012099A4200D8531E002236
:1008D00093420BDCDA43D21713409B00ED18019BC7
:1008E00001369E42E9DB380013B0F0BD90000C18D1
:1008F000A46801322C50EBE7042A55D12F002600C2
:100900001D00029AB300D058384237D1042835D997
:1009100003682B40042BB4D1FFF732FC039B013654
:100920002418B342EDD1200002F04CFD071EBDD0CB
:10093000039B029D9B00EB18041D029301232E686C
:100940001E4222D1042E20D90F2233681340042BDB
:100950000DD13000FFF714FC0190300002F030FBA5
:10096000019A0100200009F01DFF019BE418029B81
:100970000435AB42E2D100232370B4E705A9FFF7A9
:1009800031FF05A80AF01CFBC8E705A93000FFF7F6
:1009900029FF05A80AF014FB0600020005A92000A3
:1009A00009F000FFA419E2E7212000F0E1FA7DE759
:1009B000F0B50D0095B0002806DC1C2000F0D8FA38
:1009C0000400200015B0F0BD0C68012123000B408D
:1009D000009306D1042C04D922680F331A40092A47
:1009E00001D00B20EAE7626852100392002A03DC70
:1009F000009802F0E7FCE3E73F4A019201280BD0A0
:100A00006868084208D1042806D902681340042BFC
:100A100002D102F0D5FA019001980AF0D1FA06004D
:100A20000F27039B0834013B04935E43039B029012
:100A30009B001B19059301232068184251D10428FB
:100A40004FD903683B40042B52D1FFF799FB059B1C
:100A500004343618A342EED1300002F0B3FC041E79
:100A6000AFD02B680593029B002B03D0686802F07F
:100A7000A7FA0190200002F0A3FA0500009B059A56
:100A80009B00D3189F68380002F09AFA01230600F1
:100A90001F4201D1042F04D807A93800FFF7A2FE96
:100AA00007AE30000AF08CFA07000200310028007F
:100AB00009F078FE029BED19002B0AD0049B009AE6
:100AC000934206DD2800029A019909F06BFE029B11
:100AD000ED18009B01330093009A039B9342CDD104
:100AE0006FE707A9FFF77EFE07A80AF069FAAEE7ED
:100AF00002F066FAF9E7C046A2CA000010B5002469
:100B0000A04207DD0B6801341C4003D05C10E343B6
:100B1000DB171C40611C0122092002F0E7FB0028C2
:100B200003D0012364001C43446010BD0B6870B502
:100B300018000125284032D1042B30D90F241A681F
:100B400049681440092C16D15C6812092C41A24254
:100B500000D8541E844205DC02200132904206DB9C
:100B600000200FE085005D19A9600130F2E78400E4
:100B700019510130F2E7032C11D1294203D113207E
:100B800000F0F6F970BD4910FF29F8D812090433B6
:100B900092009A189A42E3D919700133FAE70B20B0
:100BA00000F0E6F9DCE700000123F7B500264D6808
:100BB0000F002B400093B3420DD11E00042D0AD923
:100BC0000F222B681A40092A0FD16A681B09561098
:100BD000B34200D85E1E3968CB0713D54C10002CE9
:100BE00001DDA64219DA12202EE0042A04D12800E1
:100BF000FFF7C6FA0600EEE7009E032AEBD11E09B6
:100C0000B600E8E72E48FFF777FD002814D00AF079
:100C1000C5F8310007F084FD4C1C009B002B4CD123
:100C2000042D4AD92A680F331340092B10D10134FF
:100C3000A40064592000FEBD39682248FFF75CFD1E
:100C400034000028E9D1113000F092F90400F1E7F6
:100C5000042B2AD1280002F0B3F90600FFF7BAFAF4
:100C6000A042C0DB012C1ADC280002F0A9F9009098
:100C70003000FFF79BFA851B280002F0A3FB041E3F
:100C8000D8D002F09DF90190786802F099F9009BA4
:100C90002A00F11A4118019809F084FDCAE73000D2
:100CA000FFF784FA013C0600DCE7032B05D12C1981
:100CB000E478023B64001C43BCE70B20C4E7C04659
:100CC00038C7000043C70000F7B54C680F0001208B
:100CD000210001402AD1042C28D90F222368BE68A4
:100CE0001A40092A13D162681B0955100191AB42C1
:100CF00000D85D1E39682848FFF7FEFC002829D07F
:100D00000F2322681340092B19D1012313E0032A72
:100D10000CD1064203D1132000F02AF9FEBD721057
:100D20000192FF2AF7D81D09AD00E3E70B20F3E796
:100D300001339A00A6509D42FADA0020EEE7032B19
:100D4000FBD1230001331A1BAA42F6DC6A46127952
:100D5000DA70F7E73968CB0706D54910002901DDBD
:100D60008D4209DA1220D7E70C48FFF7C5FC2900AD
:100D7000002801D11130CFE70F2322681340092B3F
:100D800003D1013189000E51D7E7032BD5D16B4632
:100D90001B796418E370D0E73FC7000043C7000029
:100DA00010B501240868204216D1042814D90F2256
:100DB00003681A40092A01D1406810BD032A03D1F3
:100DC0001809C0002043F8E7042A05D102F0F8F81A
:100DD000FFF700FA4000F5E70B2000F0C9F8ECE758
:100DE00010B5034A0A21034803F08AFF10BDC0462C
:100DF000E8C60000E0C60000F0B585B0039301909E
:100E000002912C4E2C4B002A02D002223270013A61
:100E100000251A601B68F554019B9D4201DB05B05B
:100E2000F0BD029AAB00D058234B1C68C8239B002E
:100E300037191C1B0123184206D0204A43102100F9
:100E4000380009F0DDFF09E01D4A002802D004281F
:100E50001BD11C4A2100380009F0D2FF30000AF0F3
:100E6000AFF8154A039B1060002B0CD0019B013B8F
:100E7000AB4208DD144B984205D8431C1360202276
:100E800032540022F2540135C6E704280FD90F234B
:100E900002681340042B04D102F092F80B4A0300BD
:100EA000CDE7092B04D14368094A5B10C7E701234A
:100EB000084AC4E7A1020020C4050020F4CF0000C6
:100EC00048C700004EC700001F03000013D60000F3
:100ED000B8C90000C7C90000012307B5034002D00C
:100EE000431018000EBD04280DD90F2201680A40D6
:100EF000042A08D1019302F063F801AA044909F019
:100F0000D1FF019BEDE70D21024A1170E9E7C046D0
:100F1000F4CF0000A00200200123020010B51A4007
:100F200015D1042801D9026812090B4011D10429F6
:100F300001D90B681B090024934206D104309B00A1
:100F40000431C318984206D30124200010BD0022AA
:100F5000EBE70023EFE704780A78002C01D1002AA0
:100F6000F2D0013001319442ECD00024EDE70000D2
:100F7000014B187000207047A002002070B501F0EE
:100F800093FD094C0100251D1F2228000AF01FF8BF
:100F900028000AF015F804230430800800011843E3
:100FA0002060200070BDC0467C020020C368F0B500
:100FB0009D00836889B05D190300183306930369A7
:100FC000069A9F00069B0290DF19436901939B00DC
:100FD000D3180393CD4B1B78002B26D17F222B688F
:100FE000CB491C1213409B005B58043501929F466D
:100FF000029B587804F060FA0023029A137027E0ED
:10100000C24B1B78002B10D12B68019A1C12134085
:10101000BF4A9B009B580435E9E7069B3A1DD11A4D
:10102000BA4BD82928DD1A221A70029BB74C9B684C
:1010300021780193EA1A029B92109B7812021A43BC
:10104000029B587804F040FA0023029A2370137030
:10105000029B069A9B680193ED1A029BAD10DD601E
:10106000069BFE1A029BB6101E61039B9B1A029AF6
:101070009B10536109B0F0BD1B783C60002B01D080
:101080001700D2E72B6801991C120B40A0499B0066
:101090005B5817000435AAE7069B3A1DD11A9B4BF3
:1010A000D82902DD1A221A70BFE728681B78291D8B
:1010B0003860002B02D017000D00B6E76B6801996D
:1010C0001C120B4092499B005B58170008358EE7B5
:1010D000069B3A1DD11A8D4BD82902DD1A221A70AF
:1010E000A3E7A4001B782C193C60002B01D017004B
:1010F0009BE72B6801991C120B4085499B005B58AC
:101100001700043573E7069B3A1DD11A7F4BD82987
:1011100002DD1A221A7088E77E49A40061581B7804
:101120003960002B01D017007FE72B6801991C1252
:101130000B4077499B005B581700043557E7043F85
:10114000744B3A68A400E250704B1B78002B00D01F
:101150006BE72B68019A1C1213406D4A9B009B5849
:10116000043544E76B4BA400E058FFF7B5FE043F9D
:1011700006003868FFF7B0FE36180120654B760090
:101180000643E650614B1B78002B00D04DE72B68DF
:10119000019A1C1213405E4A9B009B58043526E7B7
:1011A000069B3A1DD11A594BD82902DD1A221A7012
:1011B0003BE70698039C0121A04202D221000C3992
:1011C00009681B783960002B01D017002DE72B68C8
:1011D00001991C120B404E499B005B5817000435C7
:1011E00005E7069B3A1DD11A484BD82902DD1A2281
:1011F0001A701AE70699039881420FD203000C3B3C
:101200001B6845495B106418E41AA40023583B602E
:101210003E4B1B78002B05D0170006E718211970EC
:101220000023F4E72B6801991C120B4038499B00FE
:101230005B5817000435DAE6069B039A934219D2ED
:1012400013000C3B1B68344A043FA4185B10E31ADC
:10125000039A39689B0099502C4B1B78002B00D0C7
:10126000E3E62B68019A1C121340294A9B009B5805
:101270000435BCE61822254B1A70EDE7069B039A4D
:1012800093422DD2244B3E1FE31814000C3C0493D0
:101290002368049A5B10D31A039A9B009858FFF7AF
:1012A0001BFE07903068FFF717FE2468049B64104C
:1012B0001C1B079BA4001F1801207F00039B0743F2
:1012C000E7503700114B1B78002B00D0ADE62B68A0
:1012D000019A1C1213400E4A9B009B58043586E667
:1012E00018220A4B1A70EDE7069B3A1DD11A074BDC
:1012F000D82902DD1A221A7097E60399A4006158D2
:101300001B783960002B09D017008EE6A002002060
:10131000B8C700007C2D0020FDFFFF3F2B6801991E
:101320001C120B40D7499B005B58170004355EE642
:10133000043F039B3A68A400E250D34B1B78002B78
:1013400000D072E62B68019A1C121340CD4A9B0014
:101350009B5804354BE6039BA4001C192368043FEB
:1013600038685E10FFF7B8FD36180120C64B7600CE
:101370001B7806432660002B00D056E62B68019AA6
:101380001C121340BF4A9B009B5804352FE6069B56
:10139000A4003F1BBC4CBB420CD82378002B00D0D0
:1013A00043E62B68019A1C121340B64A9B009B58D7
:1013B00004351CE6B54801F0F3FD2378002B00D07E
:1013C00033E62B68019A1C121340AE4A9B009B58CF
:1013D00004350CE6A300ED18002C00DA38E6AA4B21
:1013E0001B78002B00D020E62B68019A1C121340BA
:1013F000A44A9B009B580435F9E5043F3B68042B45
:1014000004D1A300ED18002C00DA21E69E4B1B78D6
:10141000002B00D009E62B68019A1C121340994A50
:101420009B009B580435E2E5043F3B68042B06D043
:10143000A200AD18002C02DA002B00D108E6924B76
:101440001B78002B00D0F0E52B68019A1C1213408A
:101450008C4A9B009B580435C9E53A1F13685B1002
:10146000013B002B06DD01215B00A4000B432D197D
:101470001360EDE5844B17001B78002B00D0D4E5FA
:101480002B68019A1C1213407E4A9B009B5804351E
:10149000ADE53A00069B0C32D31AD82B03DD1A2295
:1014A000794B1A70C1E5FF2361005B001940FE3BD8
:1014B000FF3B194339600299069889682412049108
:1014C0006D1A0299AD1089782D020D4303999D4044
:1014D000091A891099401D430B43BB60029B7D6034
:1014E0009C70E4B26A4BE4000392E358029A936062
:1014F000654A1278002A03D008331D00039F94E543
:101500001D00019A9B680C351C1213405D4A9B001C
:101510009B58039F6BE53B1F1C68039A069B9342F5
:101520002DD10A20E3070CD4042C13D90F232268F1
:101530001340042B11D1200001F042FD09F040FDC1
:101540000630643003F06CFC00280FD1043D069B8C
:1015500003937DE50720042CF3D02000431E98411F
:10156000FA234042FF3318400730EAE7029B21008C
:10157000587803F0BBFF0023029A1370E7E7039B40
:10158000039A0C3B1B6802995B109B00D31A0C3B1F
:101590001C601F1D1300083B1B685A108A70D2B2D2
:1015A0003B49D2005B0055589B0A029A9B0095600C
:1015B000ED18039B069A043B1B685B109B00D31835
:1015C0000393314B1B78002B00D02EE52B68019A3A
:1015D0001C1213402B4A9B009B58043507E53B1F08
:1015E0001868FFF779FCA40006003F1B1E2827DCC3
:1015F00000280DDC244B1B78002B00D015E52B6850
:10160000019A1C1213401F4A9B009B580435EEE4BC
:1016100001F038FA033E361801F034FA1D4B801BF6
:101620009842F9D8184B1B78002B00D0FDE42B68AA
:10163000019A1C121340134A9B009B580435D6E4B0
:101640000123029A137001F01DFA029B0A388619D1
:101650005E60FDE43B1F1868FFF73EFCA400060037
:101660003F1B002818DC084B1B78002B00D0DCE463
:101670002B68019A1C121340024A9B009B580435A8
:10168000B5E4C046B8C70000A0020020D9C90000D8
:10169000842500203F420F00CA4B984203DD1D22E3
:1016A000C94B1A70C1E40123029A137001F0EAF9E0
:1016B000FA239B005E43029B0A3E30185860C7E441
:1016C000A300FF1A002320001A003900FFF794FB43
:1016D000BE4EBF4C3168200001F080FEBD4B31682A
:1016E0001860200003F0B6FD3168200003F005FF0C
:1016F0003168200001F039FFB34B1B78002B00D07C
:1017000093E42B68019A1C121340B34A9B009B5828
:1017100004356CE4AC4BA4001B783F1B002B00D0BD
:1017200083E42B68019A1C121340AB4A9B009B5820
:1017300004355CE4029803F0D7FBA34B1B78002B25
:1017400000D072E42B68019A1C121340A24A9B003D
:101750009B5804354BE43B1F1B68002B3ED13B00DC
:101760000C3B1B68DA072CD5390001225B105800AE
:10177000083902430A60002B44DD0122590011435D
:10178000381F01603900083909681141CB1A390046
:101790000C390968114224D09B189340A4001343CC
:1017A000039AA350884B1B78002B00D03DE42B6894
:1017B000019A1C121340884A9B009B580435FFF77E
:1017C00016FC042B06D90F2219680A40092A01D1F8
:1017D0005B68C9E719227C4B1A7026E45B10013B59
:1017E000C9E7042909D90F2208680240092A04D14F
:1017F00002339B005B58A400D2E71922724B1A7087
:10180000FFF713FC0435CDE7A300069AFB189B1ADB
:10181000D82B13DC0122631E002C14DC6A4B1B78CE
:10182000002B01D0FFF701FC2B68019A1C1213401A
:10183000694A9B009B580435FFF7D9FB1A22624B7B
:101840001A70FFF7F2FB3A601C000437E3E7069AD0
:101850003B1D9B1A5C4ED82B03DD1A233370FFF718
:10186000E4FB069B039AA40093422AD23B1F18680C
:10187000FFF732FB011E21DD039B0C3B1A6852105F
:1018800082421BDB9007801A544B4018C018039B00
:101890008000C2583B1B1A604B4B3F1B1B78043720
:1018A000002B01D0FFF7C1FB2B68019A1C121340DB
:1018B000494A9B009B580435FFF799FB202333705E
:1018C000EAE71823FBE7434BA4001A683B1B1F0001
:1018D0001A603D4B04371B78002B01D0FFF7A5FBA6
:1018E0002B68019A1C1213403B4A9B009B580435FD
:1018F000FFF77DFBA3009C46FE1A002C17DC1C2280
:10190000314B1A70002333606346FF1A2E4B0437A5
:101910001B78002B01D0FFF788FB2B68019A1C1263
:1019200013402D4A9B009B580435FFF760FB0020B5
:1019300033685A108300F15801230B4003D10D2165
:10194000214A1170DFE749108A4200DD0A000130A8
:101950008442EFDC012352001343D4E7A3009C46EA
:10196000FE1A002C17DC1C22174B1A700023336060
:101970006346FF1A144B04371B78002B01D0FFF786
:1019800054FB2B68019A1C121340134A9B009B586E
:101990000435FFF72CFB002033685A108300F15800
:1019A00001230B4003D10D21074A1170DFE74910D5
:1019B0008A4200DA0A0001308442EFDC012352003F
:1019C0001343D4E780EE3600A0020020C4050020B7
:1019D000A102002008000020B8C70000FCFFFF3F64
:1019E0003B00083B1868FFF777FA3B1F06001868B2
:1019F000FFF772FA0023864200DA0433A4003A1B90
:101A000017001360E34B04371B78002B01D0FFF75E
:101A10000CFB2B68019A1C121340DF4A9B009B5859
:101A20000435FFF7E4FA3B00083B1868FFF754FA67
:101A30003B1F06001868FFF74FFAF30FC217B042BA
:101A40005341A4003A1B17009B001360D14B04378D
:101A50001B78002B01D0FFF7E8FA2B68019A1C12C3
:101A60001340CD4A9B009B580435FFF7C0FA3B005A
:101A7000083B18683B1F1968A600BE1B042381425F
:101A800002D0042802D80023336016E00123184254
:101A9000F9D10F2302681A40042AF4D1033A114203
:101AA000F1D10429EFD90A681340042BEBD1FFF7D9
:101AB00033FA431E984180003060B64BA4001B7877
:101AC0003F1B0437002B01D0FFF7AFFA2B68019AB8
:101AD0001C121340B04A9B009B580435FFF787FA4D
:101AE0003B00083B18683B1F1968A600BE1B00237B
:101AF000814202D0042802D80423336016E0012377
:101B00001842F9D10F2302681A40042AF4D1033A8B
:101B10001142F1D10429EFD90A681340042BEBD10B
:101B2000FFF7FAF94342584180003060994BA40016
:101B30001B783F1B0437002B01D0FFF776FA2B6888
:101B4000019A1C121340944A9B009B580435FFF7DE
:101B50004EFA3B00083B1868FFF7BEF93B1F060032
:101B60001868FFF7B9F9F317C20F86425341A40072
:101B70003A1B17009B001360864B04371B78002B21
:101B800001D0FFF752FA2B68019A1C121340824AC7
:101B90009B009B580435FFF72AFA3B00083B186866
:101BA000FFF79AF93B1F06001868FFF795F9002325
:101BB000864200DD0433A4003A1B17001360754B06
:101BC00004371B78002B01D0FFF72FFA2B68019AFE
:101BD0001C121340704A9B009B580435FFF707FA0C
:101BE0003B1F1B68A400043B5A1E93413A1B17007D
:101BF0009B001360674B04371B78002B01D0FFF765
:101C000014FA2B68019A1C121340634A9B009B58DC
:101C10000435FFF7ECF93B00083B1868FFF75CF967
:101C20003B1F06001868FFF757F932180120A4007F
:101C30003B1B1F00520002431A60564B04371B78AF
:101C4000002B01D0FFF7F1F92B68019A1C12134009
:101C5000514A9B009B580435FFF7C9F93B00083BEC
:101C60001868FFF739F93B1F06001868FFF734F9C9
:101C7000321A0120A4003B1B1F00520002431A60CD
:101C8000444B04371B78002B01D0FFF7CEF92B68AB
:101C9000019A1C121340404A9B009B580435FFF7E1
:101CA000A6F93B00083B1868FFF716F93B1F060032
:101CB0001868FFF711F902000120A4003B1B1F0068
:101CC0007243520002431A60324B04371B78002BD8
:101CD00001D0FFF7AAF92B68019A1C1213402E4A73
:101CE0009B009B580435FFF782F93B1F1868FFF7EC
:101CF000F3F8061E17D11F22264B1A70A4003B1BB7
:101D00001F001E60234B04371B78002B01D0FFF708
:101D10008CF92B68019A1C1213401F4A9B009B5898
:101D20000435FFF764F93B00083B1868FFF7D4F867
:101D3000310006F00FFC012640000643DEE73B1FA2
:101D40001868FFF7C9F8061E17D11F22114B1A7029
:101D5000A4003B1B1F001E600E4B04371B78002B9A
:101D600001D0FFF762F92B68019A1C1213400A4A4E
:101D70009B009B580435FFF73AF93B00083B186875
:101D8000FFF7AAF8310006F0CBFC012649000E430C
:101D9000DEE7C046A0020020B8C700003B1F18685D
:101DA000FFF79AF8C217801850400122A4003B1B8D
:101DB0001F00400010431860F64B04371B78002BBF
:101DC00001D0FFF732F92B68019A1C121340F24A36
:101DD0009B009B580435FFF70AF9A300FE1A3068F0
:101DE000012C24D1FFF778F80494079008F0D6FF6F
:101DF0000799002900DC012106F092FC049BA40055
:101E0000C918012349001943E24B3F1B1B7831607D
:101E10000437002B01D0FFF708F92B68019A1C1238
:101E20001340DD4A9B009B580435FFF7E0F8FFF7AD
:101E300053F804907068FFF74FF8049B0130C31A01
:101E40000793D3E7A300FE1A31002000049301F0AA
:101E500013FB049B3060FF1ACE4B04371B78002B1A
:101E600001D0FFF7E2F82B68019A1C121340CA4A0E
:101E70009B009B580435FFF7BAF83B00083B1868F5
:101E8000FFF72AF83B1F06001868FFF725F8020045
:101E90000120A4003B1B1F003240520002431A6085
:101EA000BC4B04371B78002B01D0FFF7BEF82B6822
:101EB000019A1C121340B84A9B009B580435FFF747
:101EC00096F83B00083B1868FFF706F806003B1F32
:101ED0001868FFF701F8320002430120A4003B1B01
:101EE0001F00520002431A60AA4B04371B78002BD4
:101EF00001D0FFF79AF82B68019A1C121340A64AEA
:101F00009B009B580435FFF772F83B00083B1868AC
:101F1000FEF7E2FF06003B1F1868FEF7DDFF320008
:101F200042400120A4003B1B1F00520002431A60E4
:101F3000984B04371B78002B01D0FFF776F82B68FD
:101F4000019A1C121340944A9B009B580435FFF7DA
:101F50004EF83B1F1868FEF7BFFFC0430122A400E4
:101F60003B1B1F004000104318608A4B04371B784E
:101F7000002B01D0FFF759F82B68019A1C1213406F
:101F8000854A9B009B580435FFF731F83B00083B1E
:101F90001868FEF7A1FF06003B1F1868FEF79CFFBC
:101FA0003200824051000122A4003B1B1F000A4363
:101FB0001A60784B04371B78002B01D0FFF735F8F7
:101FC0002B68019A1C121340734A9B009B580435DE
:101FD000FFF70DF83B00083B1868FEF77DFF060091
:101FE0003B1F1868FEF778FF3200024151000122C2
:101FF000A4003B1B1F000A431A60664B04371B7882
:10200000002B01D0FFF711F82B68019A1C12134026
:10201000614A9B009B580435FEF7E9FF3B000C3BEF
:102020001868FEF759FF3B00083B06001868FEF7EA
:1020300053FFF1170200C317300006F0C3FB3B1F2C
:10204000049005911868FEF747FF0200049805996F
:1020500006F06CFB43000120A4003E1B3700184330
:102060004C4B30601B780437002B01D0FEF7DDFFAE
:102070002B68019A1C121340474A9B009B58043559
:10208000FEF7B5FFA300FE1A310020000493FEF70F
:1020900035FD049B3060FF1A3E4B04371B78002B44
:1020A00001D0FEF7C2FF2B68019A1C1213403A4A76
:1020B0009B009B580435FEF79AFFA300FF1A3900D6
:1020C0002000FEF733FD334B1B78002B01D0FEF7C9
:1020D000ACFF2B68019A1C1213402F4A9B009B589F
:1020E0000435FEF784FFA300FE1A3100200004939C
:1020F000FEF75AFD049B3060FF1A264B04371B780D
:10210000002B01D0FEF791FF2B68019A1C1213409F
:10211000214A9B009B580435FEF769FFA300FF1A74
:1021200039002000FEF7D0FD1A4B1B78002B01D0A0
:10213000FEF77BFF2B68019A1C121340164A9B0086
:102140009B580435FEF753FFA300FE1A3100200010
:102150000493FEF725FE049B3060FF1A0D4B0437F5
:102160001B78002B01D0FEF760FF2B68019A1C1230
:102170001340094A9B009B580435FEF738FF069B25
:102180003E1DF31A034CD82B08DD1A232370FEF7EB
:102190004CFFC046A0020020B8C7000000F07CFC45
:1021A00043000120184323783860002B02D0370009
:1021B000FEF73BFF2B68019A1C121340F44A9B0068
:1021C0009B5837000435FEF712FF069B3E1DF31A9D
:1021D000F04CD82B03DD1A232370FEF726FF00F006
:1021E00051FCED4B40001840012318432378386020
:1021F000002B02D03700FEF718FF2B68019A1C1243
:102200001340E34A9B009B5837000435FEF7EFFE6E
:102210000123A600BE1B20001A003100FEF7ECFDD2
:10222000DE4C2068643002F0FBFD002802D1043D42
:10223000FEF70EFF029B21685A78D94803F06BF92C
:102240000123029A3700137000F01CFCD54B226862
:102250001B68063253431818029B5860FEF7F8FEBD
:10226000A600BE1B2000012300223100FEF7C4FDA2
:10227000CA4C2068643002F0D3FD0028D7D0C8488B
:1022800002F040FFDCE7A4003E1BFEF777FE3700BC
:10229000C04B30601B780437002B01D0FEF7C5FE21
:1022A0002B68019A1C121340B94A9B009B580435B5
:1022B000FEF79DFEA4003E1B300000F01CFC370022
:1022C000B44B30601B780437002B01D0FEF7ADFE15
:1022D0002B68019A1C121340AD4A9B009B58043591
:1022E000FEF785FEA4003E1B300000F006FC370020
:1022F000A84B30601B780437002B01D0FEF795FE09
:102300002B68019A1C121340A14A9B009B5804356C
:10231000FEF76DFEA300FE1A31002000049300F0CA
:10232000EFFB049B3060FF1A9A4B04371B78002B9D
:1023300001D0FEF77AFE2B68019A1C121340944AD2
:102340009B009B580435FEF752FEA4003F1B38004B
:1023500000F008FC8F4B1B78002B01D0FEF765FEC8
:102360002B68019A1C121340894A9B009B58043524
:10237000FEF73DFEA300FE1A31002000049300F09A
:1023800019FC049B3060FF1A824B04371B78002B2A
:1023900001D0FEF74AFE2B68019A1C1213407C4ABA
:1023A0009B009B580435FEF722FEA4003F1B38001B
:1023B00000F042FC774B1B78002B01D0FEF735FE76
:1023C0002B68019A1C121340714A9B009B580435DC
:1023D000FEF70DFE0121200000F016FC6D4B1B786E
:1023E000002B01D0FEF721FE2B68019A1C1213402E
:1023F000674A9B009B580435FEF7F9FD0021200039
:1024000000F002FC634B1B78002B01D0FEF70DFEA1
:102410002B68019A1C1213405D4A9B009B5804359F
:10242000FEF7E5FDA4003E1B300000F027FC37005E
:10243000584B30601B780437002B01D0FEF7F5FDB8
:102440002B68019A1C121340514A9B009B5804357B
:10245000FEF7CDFDA4003E1B300000F023FC37004A
:102460004C4B30601B780437002B01D0FEF7DDFDAC
:102470002B68019A1C121340454A9B009B58043557
:10248000FEF7B5FDA4003F1B380000F0E5FB414B13
:102490001B78002B01D0FEF7C8FD2B68019A1C1297
:1024A00013403B4A9B009B580435FEF7A0FDA40057
:1024B0003F1B380003F010FB364B1B78002B01D07C
:1024C000FEF7B3FD2B68019A1C121340304A9B00A3
:1024D0009B580435FEF78BFDA4003E1B300003F033
:1024E000A9FB37002B4B30601B780437002B01D041
:1024F000FEF79BFD2B68019A1C121340244A9B0097
:102500009B580435FEF773FDA4003F1B380003F011
:10251000B3FA204B1B78002B01D0FEF786FD2B6809
:10252000019A1C1213401A4A9B009B580435FEF76F
:102530005EFDA4003E1B300003F0B4FA3700154BDB
:1025400030601B780437002B01D0FEF76EFD2B683E
:10255000019A1C1213400E4A9B009B580435FEF74B
:1025600046FDA300FF1A3900200001F0B1FA094B23
:102570001B78002B01D0FEF758FD2B68019A1C1226
:102580001340034A9B009B580435FEF730FDC046BC
:10259000B8C70000A0020020FEFFFF7FC405002096
:1025A000A102002004000020A300FF1A390020002F
:1025B00001F0C6F89F4B1B78002B01D0FEF735FDCC
:1025C0002B68019A1C1213409B4A9B009B580435B0
:1025D000FEF70DFDA300FF1A3900200001F0B0F94D
:1025E000944B1B78002B01D0FEF71FFD2B68019A3E
:1025F0001C121340904A9B009B580435FEF7F7FCD1
:10260000A300FF1A3900200001F0C2F9894B1B78A2
:10261000002B01D0FEF709FD2B68019A1C12134014
:10262000854A9B009B580435FEF7E1FCA300FE1A87
:1026300031002000049303F078FB049B3060FF1A04
:102640007C4B04371B78002B01D0FEF7EEFC2B6887
:10265000019A1C121340784A9B009B580435FEF7E0
:10266000C6FCA300FE1A31002000049303F065FBB2
:10267000049B3060FF1A6F4B04371B78002B01D08E
:10268000FEF7D3FC2B68019A1C1213406A4A9B0088
:102690009B580435FEF7ABFCA300FE1A3100200066
:1026A000049303F052FB049B3060FF1A614B043724
:1026B0001B78002B01D0FEF7B8FC2B68019A1C1286
:1026C00013405D4A9B009B580435FEF790FCA30025
:1026D000FE1A31002000049303F03FFB049B30609E
:1026E000FF1A544B04371B78002B01D0FEF79DFCDA
:1026F0002B68019A1C1213404F4A9B009B580435CB
:10270000FEF775FCA300FF1A3900200001F050F815
:10271000484B1B78002B01D0FEF787FC2B68019AF1
:102720001C121340444A9B009B580435FEF75FFC83
:10273000A300FF1A3900200001F052F93D4B1B782D
:10274000002B01D0FEF771FC2B68019A1C1213407C
:10275000394A9B009B580435FEF749FCA300FE1A3A
:1027600031002000049301F0B9F8049B3060FF1A97
:10277000304B04371B78002B01D0FEF756FC2B683A
:10278000019A1C1213402C4A9B009B580435FEF7FB
:102790002EFCA300FF1A3900200001F067F8254B3A
:1027A0001B78002B01D0FEF740FC2B68019A1C120D
:1027B0001340214A9B009B580435FEF718FC069BEA
:1027C000029AFB1A9B101361A300FF1A3900200024
:1027D00002F0AAFA174B1B78002B01D0FEF725FC5C
:1027E0002B68019A1C121340134A9B009B58043516
:1027F000FEF7FDFB069B029AFB1A9B101361A300D8
:10280000FE1A31002000049302F08EFA049B30601F
:10281000FF1A084B04371B78002B01D0FEF705FC8C
:102820002B68019A1C121340034A9B009B580435E5
:10283000FEF7DDFBA0020020B8C700000023F7B5BB
:102840005A1E0192002B07DA01F058F902F060FDE0
:1028500002F0C0FE1923019300263000194B1968BD
:10286000B14212DD184B1A6801328A420FDAF024A5
:102870001A601D68154F6C43E35D002B1FD0E419EF
:10288000022B06D12000FEF791FB019BD8E7002226
:10289000EDE7012B0DD1002801D100F0F3F8F02273
:1028A0006A43BB185B680A49C31A8B4201D80223EA
:1028B000BB54F0235D43054BEB5C022BE2D00136A9
:1028C000CCE7C046C805002000000020241C0020E2
:1028D0003F420F00012200210A4B0B481A61195098
:1028E00004301950A2210420C9005850C121C02031
:1028F0008900800258501A60044BFC311960044B67
:102900001A70704700A000400405000000E100E0DC
:10291000EC05002004207047F8B550C901232200BF
:102920001A40101E2DD03340181E2AD064100020EB
:10293000192C26D81D4B761035009E4200DD1D0057
:102940001B4F3B5D012B05D00121200004F01EF937
:1029500001233B55174B1B78002B01D1FFF7BAFF22
:102960000023154A9E420DDCFF2514491448D65C0D
:10297000B44202D15E007052D5540133042BF6D11B
:102980000420F8BDD15C8C4203D10C4A5B009D52FF
:10299000F6E70133042BF5D10023D15CFF2901D1E7
:1029A000D454F2E70133042BF7D1E9E78813000090
:1029B000D0050020EC0500201C0000200E000020A7
:1029C000DC050000F8B530C9012623003340181E8D
:1029D0001BD02B003340181E17D034410020192C77
:1029E00013D8174F3B5DB34204D03100200004F0F0
:1029F000CDF83E5569100800124A1038124B90422B
:102A000004D9012252421A600420F8BD1C600F480C
:102A100005F0A0FD0E4B18800E4B1B78002B02D149
:102A2000FFF758FFF0E701220B4B9A64A922D2006E
:102A30009A588018A82280B2D2009850E4E7C04685
:102A4000D0050020908601001800002020A107007A
:102A50000C000020EC05002000A00040042070477E
:102A600001220020054B06491A61585004310330F9
:102A700058500831801858501A6070470080004044
:102A8000040500000122034B1A64A822D2009858C2
:102A90007047C0460080004010B5FFF7F3FFFA21F1
:102AA000890005F0CDFC10BD004870472CCA00001D
:102AB0001A20704770B5054E0400335C0D008B4240
:102AC00002D004F063F8355570BDC046D005002033
:102AD00070B50024064D635D012B05D10021200057
:102AE00004F054F80023635501341A2CF2D170BD60
:102AF000D005002070470D2070473520704700003A
:102B0000F8B501240B6806000D00234204D10D2006
:102B1000FEF72EFA2000F8BD5B102000052BFAD836
:102B20000E4A9B009C580E4F3B5D002B05D00021A8
:102B3000200004F02BF800233B55012E06DD6B68C6
:102B4000042B03D10221200004F020F8200003F020
:102B5000CBFE012440002043DDE7C04614CA00003C
:102B6000D0050020F8B501260568354202D044683A
:102B7000344203D10D20FEF7FBF9F8BD6D10192D7D
:102B8000FBD80A4F7B5D012B04D03100280003F0F5
:102B9000FDFF7E55064964108C4202DCE143C917F3
:102BA0002140280003F026FFE7E7C046D0050020BB
:102BB000FF03000070B501240D68254204D10D20EB
:102BC000FEF7D6F9200070BD6D10192D17D800241E
:102BD000012804DD4C68043C63425C416400094EFA
:102BE000735DA34204D02100280003F0CFFF745589
:102BF000280003F0FFFF03000420012BE3D0002096
:102C0000E1E7C046D005002070B504000D0019288A
:102C10000ED8084E335C012B04D0012103F0B6FF1F
:102C200001233355290020004D1EA94103F0CCFF9C
:102C300070BDC046D0050020036810B5DA0703D484
:102C40000D20FEF795F910BD4168581004394A422D
:102C50005141FFF7D9FFF6E737B569460A00064B41
:102C600030CB30C203680220042B02D100F068FE92
:102C700037BD00F08DFEFBE7ECC9000010B5084C35
:102C8000237D002B05D00021142003F07FFF0023BB
:102C90002375142003F0AEFF43425841800010BD5D
:102CA000D005002010B5084CA37D002B05D00021D5
:102CB000162003F06BFF0023A375162003F09AFF84
:102CC00043425841800010BDD0050020F7B5304D7B
:102CD000304E6B6C002B15D0A8240023E40037592C
:102CE0006B642D4B186800280CDB2C4B19784A427A
:102CF0005141C9B2197003F067FF294B1B88DF19D6
:102D0000BFB23751AB6C002B39D00021254B264F79
:102D1000F458A9643A780C340193244D8A4206D0C1
:102D20002B68032B03D8224AD05C03F04DFF2B689D
:102D3000204A0133134004D50422013B524213437D
:102D400001331B4900228C462B60042B18D06046AF
:102D5000C05C591CFF2802D10B000122F5E7002AB4
:102D600000D02B60012103F02FFF01233B702B6863
:102D7000114A5B009B5AE418019BA4B2F450F7BDC2
:102D800001235B422B6000233B700C4BF3E7C046F2
:102D9000FCA0004000A0004018000020EB0500202F
:102DA0000C00002044050000EA050020CC050020AE
:102DB0001C000020030000800E0000205046000090
:102DC000084B094AFF201A805A809A80DA80002333
:102DD000064A07491370074A087048708870C8701F
:102DE000136070470E000020DC050000EA0500209B
:102DF0001C000020CC0500200122024B52421A6028
:102E00007047C0461800002010B5034A042103484B
:102E100001F076FF10BDC046F4C9000034D10000B7
:102E2000E12170B54902144803F056FBFFF718FE84
:102E30000A2003F053FD0023FF21104A9954013367
:102E40001A2BFBD1012200200D4B01001A60042334
:102E50000C4A0D4D1468002CFCD02C680002013B7C
:102E600020431160002BF5D10122084B1A6003F0BA
:102E7000EFFC00F08FFF70BDAC1B0020D0050020E0
:102E800000D0004000D1004008D5004004D00040F0
:102E9000F8B50B4E070030000D0003F065FB040091
:102EA000A84200DD2C003D00EB1B9C4205DD3000FC
:102EB00003F064FB28700135F6E72000F8BDC0463A
:102EC000AC1B002010B50100014803F00DFB10BD44
:102ED000AC1B002010B5054C200003F013FBE121D2
:102EE0002000490203F0F8FA10BDC046AC1B0020D8
:102EF000C3070CD4064B1B68834208D8054B1B68DC
:102F0000984204D8031F1B68002B00D0180070479C
:102F1000F8050020F40500200023012210B50A481E
:102F2000990001334250642BFAD1084C084B002120
:102F30001A602000074A07F051FC074B074A6360FC
:102F4000074B1A6010BDC0467C2D0020FC050020F8
:102F500008000020D40900003027000000060020EF
:102F6000F005002010B5044B044A1A60044B054AD2
:102F70001A60FFF7D1FF10BDF8050020FC05002006
:102F8000F4050020D00F0020044B1B6818680009CE
:102F90000238C343DB1718407047C046F0050020D5
:102FA00000B59BB00200054901A807F05BFF01A82E
:102FB00002F0C4F802F00EFBFCE7C04692CA000023
:102FC0000A4BC20704D4042804D8094B00D0094B8B
:102FD000180070470F2203681A40031D042AF7D017
:102FE000054B092AF4D0054BF2E7C04678CA000029
:102FF0004EC7000048C700008BCA000082CA00000C
:103000000020064A0649131F186013681B09023383
:103010009B00D2188A42F6D37047C04600060020B3
:10302000D00F0020F7B50F240126304B304A196825
:10303000304B314D186813681F002740072F25D8E3
:1030400013681B0902339B00D218AA42F3D3002451
:103050002A4EA500AD192868FFF74AFF0134286001
:10306000642CF6D1264C2068FFF742FF2060254CE7
:103070002068002802D0FFF73BFF20600025224B8C
:103080001B680093009B9D4213DBF7BD1B099B004F
:10309000D3189A42D4D01F68374208D1B94206D219
:1030A000B84204D3043F3F68002F00D01F60043BA8
:1030B000EFE7F0236B43154A9B181A78002A01D1D9
:1030C0000135DFE71F693C2300266B43DB199B00BA
:1030D00001930136BB1BF3D4019BB4001C1B0B4BAB
:1030E0001C19A069FFF704FFA061F2E7F8050020B2
:1030F00000060020F4050020D00F00207C2D0020C9
:1031000008000020D00F0020C8050020241C00204B
:10311000F7B50124204244D1224B1B689C469842BB
:103120003FD3214B1B68019398423AD8031F1B6879
:10313000002B36D10200036800941B09002B0FD12D
:103140000099131F196090422BD015682B1F1B6824
:10315000990069180C68013B14600A602A00EDE7C9
:103160009D0055192968009C214218D18C4516D81C
:10317000019C8C4213D30E1F3468002C0FD10F68B2
:103180000F343C40072C07D92F60151F2B600B68AC
:103190000A601B090A00D1E700993160CEE7013BC4
:1031A000CCE7F7BDF8050020F40500200D49F0B587
:1031B0000B000F260C4D18681C1F276802090232ED
:1031C000002F0BD000208B4200D008002060900020
:1031D000091892009B18AB42EDD3F0BDB0431860C4
:1031E000F7E7C04600060020D00F0020F8B5114CCC
:1031F00026000F2233681F0913420DD07D1CAD003D
:10320000A64204D02A003100200007F0D4FA0022A0
:103210006319043564191A600237BF00064BF619AA
:103220009E42E6D31B1B9B10013B1B012360034BFB
:103230001C60F8BD00060020D00F0020F005002023
:10324000F0B59BB0FFF71EFC00240700204AA30046
:10325000D0580134FFF75CFF642CF7D11D4B186880
:10326000FFF756FF1C4B1868002801D0FFF750FFEE
:1032700000261A4B1B689E4216DBFFF797FFFFF7ED
:10328000D1FEFFF7B3FFFFF7FDFB154BC21B1B6819
:1032900014491B6801A81B09023B07F0E3FD01A8C4
:1032A00001F04CFF1BB0F0BDF02575430E4BED183F
:1032B0002B78002B01D10136DBE72B695C1E002C3B
:1032C000F9DBA300EB189869FFF722FF013CF6E752
:1032D0007C2D002008000020D00F0020C805002011
:1032E000F005002058CA0000241C0020F7B5164D38
:1032F0004F1C2B6806001B680C0001921B099F42A3
:103300000ADBFFF79DFF2B681B681B099F4203DB4D
:103310000A20FDF72DFEFEBD2868A71CBA00DB1BA6
:1033200081181B010B6029600021031F19600F2306
:103330001E4003002401264340C3083A9A189A42CB
:10334000E9D9019902C3FAE7F0050020F7B50300B7
:103350000122134004000D000193002B2AD1164BCB
:103360001B68834226D8154B1B68834222D90F2342
:10337000134F386000681840FFF7B8FF019B3C68A6
:10338000061E3B6016D0236804301B099D4200DDF9
:103390001D00AA00211D251F07F004FAFFF730FECB
:1033A0002E60FFF73FFE00232B6022680F339A4305
:1033B000226034002000FEBDF8050020F405002046
:1033C000D00F00200323043010B5C117194009188D
:1033D000891000220420FFF789FF10BD70B5050099
:1033E00008000C00FFF7EEFF0023002804D170BD99
:1033F000E95CC21811710133A342F9DBE343DB1727
:103400001C40002304192371F1E7000013B50124C7
:103410000868044016D04410200005F02FFB134923
:1034200005F0FAF907F0E0F803F028FD0022104B50
:1034300006F094FA03F0CAFC07F066F84300012096
:10344000184316BD04280DD90F2302681340042B1E
:1034500008D10194FFF7B4FD01AA064907F022FD47
:10346000019CD9E70D20FDF783FDD5E7D30237395D
:103470000000D040F4CF0000086870B501240500BA
:10348000254006D1042804D90F2302681340042BD9
:1034900003D00E20FDF76CFD70BDFFF791FD0378A2
:1034A0002900233B5A4253411022C01807F04EFE18
:1034B00080239B05C218044B9A4201D91420E9E7E6
:1034C00040002043E8E7C046FFFFFF3F10B5034A36
:1034D0000221034801F014FC10BDC046A8CA000038
:1034E000A3CA00000020704710B51E20FDF740FD64
:1034F00010BD10B51E20FDF73BFD10BD10B51E2000
:10350000FDF736FD10BD10B51E20FDF731FD10BDD5
:1035100010B51E20FDF72CFD10BD10B51E20FDF7C7
:1035200027FD10BD10B51E20FDF722FD10BD10B502
:103530001E20FDF71DFD10BD10B51E20FDF718FD66
:1035400010BD10B51E20FDF713FD10BD10B51E20D7
:10355000FDF70EFD10BD10B51E20FDF709FD10BDD5
:1035600010B51E20FDF704FD10BD704710B5034ACD
:103570000E21034801F0C4FB10BDC046C8CA0000BC
:1035800038CB00000120034B1860034B1B688340BD
:1035900018437047F40F0020D40F0020F0B5EFF36C
:1035A00010810123194083F31088134C134AA44659
:1035B0001268134E013A9340124F134A002B17D052
:1035C000146803420FD03D682C60C046C046C04618
:1035D000C046C046C046C046C0460C4C156824686C
:1035E00025605B08EAE765462C6014683460F8E7FC
:1035F00081F31088F0BDC04608050050200000206F
:103600000C050050E00F0020E80F0020DC0F002028
:1036100030B585B001AD0C220649280007F0C2F88C
:103620000024285D01210134FFF744FA0C2CF8D165
:1036300005B030BDF7CB0000F7B56A46394B01AD98
:1036400013800F239370384B2B800A23AB70FFF746
:1036500019FA364B364CC0182368984201D2002321
:1036600023602668002E3DD16B469F5D0121380006
:10367000FFF720FA01360021380003F0A5FA032EE7
:10368000F2D10026AF5D01213800FFF713FA0136B1
:103690000121380003F098FA032EF3D1C820013835
:1036A000C046C046C046C046C046C046C046C046EA
:1036B000C046C046C046C046F1D100212878FFF779
:1036C000F9F968780021FFF7F5F9A8780021FFF7EC
:1036D000F1F9FFF7D7F9FA2300251B01C018206084
:1036E0002800FEBDFFF7CEF9236800259842F7D3E6
:1036F000032003F0F9F80600042003F0F5F836186B
:103700000A2003F0F1F80B4B9B1B181A0A4BA84236
:1037100006DB18600023094A236013600125DFE7F8
:103720001D60F7E70D0E00000304000010270000E5
:10373000EC0F0020E3030000D40F0020F40F002062
:103740000022054B10B51A60044B1B68934201D050
:1037500002F072FB002010BDF00F0020D01A0020F4
:1037600010B5041E10DA1A240A4BA400E2580123F3
:103770009340094A09491360094A1160094A0A49F4
:1037800011600A4A136010BDFFF792F9A042EADD0A
:10379000EAE7C0469CD80000E80F0020080500506A
:1037A000E00F0020DC0F00200C0500501805005031
:1037B0002B4BF7B51B680C00002B03D101204042B6
:1037C000FFF7CEFF24680126250035401AD0FF22DE
:1037D0006310120260121040DAB21043FF221B0283
:1037E0001204134018431F4B1B68202B06D1B44012
:1037F0001D4BA40EA400E35800021843FFF7CEFEB1
:103800000020FEBD042CFBD90F2322681340092B96
:10381000F6D1FF2763683F025B100193019B9D4235
:10382000EEDAAB00E3189B68334216D05A105812F8
:10383000D1B238400843FF21120209040A40104364
:10384000084A1268202A06D15B009B0E06499B009D
:10385000020258581043FFF7A1FE0135DEE7C046CB
:10386000E80F002020000020E0CD000002000868E2
:1038700010B5C3070FD540101823012A03DD4A688D
:10388000042A00D10833054A1360FFF733F9FFF724
:1038900067FF002010BD01204042EDE7200000201E
:1038A00013B50124044002D04410200016BD0428A2
:1038B0000DD90F2302681340042B08D10194FFF7A0
:1038C0007FFB01AA044907F0EDFA019CEDE70D200A
:1038D000FDF74EFBE9E7C046F4CF00000868F8B5F5
:1038E000C3071AD5FFF7DCFF0300203B5E2B23D86C
:1038F0000520012258430023104E451DA84217D031
:1039000005211024375C3C4200D09B18013952003D
:1039100064100029F7D10130F0E704280CD90F22F8
:1039200003681A40042A07D11B0905D00079DBE798
:1039300001205B001843F8BD0120FCE703CC000028
:1039400070B508680D00FFF7ABFF04006868FFF76B
:10395000A7FF621E0100042A14D8451E042D11D8A9
:1039600005236B439B18012215009D402B00064840
:1039700005682B430360054B1B68002B02D0200019
:1039800002F05BFA002070BDF00F0020D01A00207A
:1039900070B508680D00FFF783FF04006868FFF743
:1039A0007FFF621E0100042A13D8451E042D10D883
:1039B00005236B439B1801229A40074803689343F1
:1039C0000360064B1B68002B03D00022200002F08E
:1039D00034FA002070BDC046F00F0020D01A00203D
:1039E000F0B5050089B008680C00FFF759FF069094
:1039F000022D36DD6068FFF753FF0190A068FFF7E6
:103A00004FFF04000127231D661E0793731C0293BA
:103A1000079B9E4235D0052373430593019B019D6F
:103A200005330493049BAB421ED0042E16D86B1EA4
:103A3000042B13D80122059B2349013B5B199A40B3
:103A40009446224A0B681068069A3A4003920DD0B9
:103A500062461A430A60012200280DD17F00013519
:103A6000E0E701240194CDE7029ECFE7624693434D
:103A70000B600028F2D0039A0299280002F0DDF9C9
:103A8000ECE7019B1E1D042E1AD8012C18D100252D
:103A900005273B0021006B439B1999400B000A4A04
:103AA000013511689943094B11601B68002B05D043
:103AB000019B0022581D290002F0BFF9052DE8D115
:103AC000002009B0F0BDC046F00F0020D01A002041
:103AD000086810B5C30703D5FFF7E2FE054B186071
:103AE000054B1B68002B03D0024B186802F0A6F9A7
:103AF000002010BDF00F0020D01A00207FB5A04C90
:103B00002368002B0AD19F4A1268002A06D19E4BD7
:103B10001B68002B01D0FFF78FFD7FBD9B4D2A68EE
:103B2000002A26D1984A1268002A1BD0FFF784FD8C
:103B30000028F2D0FFF76CFD924B24681A681C60D5
:103B4000002A16D0002C14D101AD0C229049280077
:103B500006F028FE285D00210134FEF7ABFF0C2C97
:103B6000F8D1DAE7874A1268002AE5D1002BE3D0C2
:103B7000E0E700210D2003F027F800210E2003F0DC
:103B800023F800210F2003F01FF82E68012E5DD0CE
:103B9000022E00D1A2E0002E51D101363100794C25
:103BA00004202368994303F00FF8042123680520BB
:103BB00019404B42594103F007F8102123680620B1
:103BC00019404B42594102F0FFFF8021236809014F
:103BD00019404B4259410C2002F0F6FF8021236826
:103BE000090219404B4259410B2002F0EDFF8021A0
:103BF0002368490219404B4259410A2002F0E4FF70
:103C000080212368890219404B425941092002F062
:103C1000DBFF80212368C90219404B42594108202B
:103C200002F0D2FF802321681B0319404B42594107
:103C3000072002F0C9FF31000D2002F0C5FF2B68FC
:103C40000321581C04F06CFD296066E702214D4CED
:103C50000720236819404B42594102F0B5FF082064
:103C6000216801404B42594102F0AEFF8021236898
:103C7000C90019404B425941052002F0A5FF80219F
:103C80002368490119404B425941062002F09CFF2C
:103C900080212368C90119404B425941042002F098
:103CA00093FF80212368890319404B4259410A2020
:103CB00002F08AFF802321681B0419404B425941BE
:103CC000092002F081FF31000C2002F07DFF31005D
:103CD0000B2002F079FF31000E20AEE72021294CA5
:103CE0000720236819404B42594102F06DFF4021E3
:103CF0002368082019404B42594102F065FF80219A
:103D00002368092019404B42594102F05DFF802190
:103D10002368490019404B4259410A2002F054FFE0
:103D200080212368890019404B4259410B2002F041
:103D30004BFF80212368890119404B4259410C20D7
:103D400002F042FF80212368490319404B42594148
:103D5000062002F039FF80212368C90319404B4235
:103D60005941042002F030FF802321685B04194090
:103D70004B425941052002F027FF01210F205CE74B
:103D8000F00F0020E40F0020F40F0020D80F0020D7
:103D9000F7CB0000012010B54042FFF7E1FC002006
:103DA000FFF7FCFB10BD000010B5034A09210348D2
:103DB00000F0A6FF10BDC046E0CE000028CF0000F6
:103DC00030B502248025094B094AED009C505C590E
:103DD000002CFCD0A124E400884202D30021995099
:103DE00030BD8025ED0018514019F5E700E0014095
:103DF0000405000010B5002806D1C020B021400203
:103E00008902FFF7DDFF10BDB02080218002C902CA
:103E1000F7E7000043425841064B40421840B023A8
:103E20009B02C018036800201A0E532A01D11B02FE
:103E3000180A704700C0FEFF30B501248025054BED
:103E4000054AED009C505C59002CFCD0016000211B
:103E5000995030BD00E00140040500004342584144
:103E6000074B40421840B0239B02C018A62310B550
:103E70000902DB05090A1943FFF7DEFF10BDC04642
:103E800000C0FEFF70B5012480250D4B0D4EED00E6
:103E90009C515C59002CFCD0002902DC00229A5174
:103EA00070BD557814782D02254394780139240487
:103EB0002543D478043224062C4310C0ECE7C046D6
:103EC00000E001400405000070B505004B680A00E1
:103ED0009C1C2100A400FFF7D5FF281970BD00002D
:103EE000134B1B68002B0CD08022B023D2029B0204
:103EF00000280BD11A1D5B681B0E522B00D110003D
:103F00007047B022C02392025B02F1E782420DD9D2
:103F100003681B0E522B09D1436802339B00C01863
:103F2000824203D903681B0E522BE9D00020E7E739
:103F3000F810002070B50020FFF7D2FFFF26050023
:103F4000002801D1280070BD03681C143440FFF71D
:103F5000C7FFDA2CF4D10500F2E700008022F0B5AB
:103F60005200A1B00021674806F038FC80220021F1
:103F70005200654806F032FC644BFF271B681A00AC
:103F8000049353425A4110000592FFF733FF049CFB
:103F90000020631E9C415E4B64421C405D4BE41854
:103FA000FFF7C8FF0600002E2DD10498FFF732FF5F
:103FB000411C0598FFF752FF059A574D534B2C6053
:103FC0001A60FEF787FF514B64201B68A0215A42FC
:103FD00053414F4A5B421340B0222C6892029B1817
:103FE000E41A6043490204F0B5FAA0225202030029
:103FF00000924A49220007A806F034FF07A801F002
:104000009DF821B0F0BD3268131412123A403B40C3
:1040100003921A000A3A092A49D83A4B039A995C42
:10402000002931D110223E4806F0D8FB35002B681C
:1040300003991A123A40914209D11A143A400B2AB4
:1040400027D0132A2DD00A2A01D1354B1D60280014
:10405000FFF746FF051EEAD1314B196800290FD042
:104060002000FFF731FF04002D4B5B195968002930
:1040700003D02000FFF728FF040004350C2DF3D1F6
:10408000204B0121039A99543000FFF729FF0600C5
:1040900089E73B40022BDADC214A9B00D3185D60A4
:1040A000D5E7102200211E4806F098FBCFE71A0042
:1040B000153A082AE8D8144A0399525C002AE3D139
:1040C0003500152B00D01500300003681A143A4053
:1040D000152A0FD01D2A00D10025FFF701FF002867
:1040E000F3D1002D04D020002900FFF7EDFE0400DD
:1040F000054BC6E7039A1B123B409A42EDD10500DF
:10410000EBE7C046F80F002000110020F810002057
:1041100000C0FEFF04C00200FC100020C1CF000060
:104120000C2F0020F0B50020B7B00024FFF7D8FE18
:10413000270005002600002D2ED1284D2868FFF706
:1041400069FE32003B0001900094254904A806F066
:1041500089FE04A800F0F2FF224B64201C682B6843
:10416000A0215A425341204A5B421340B02292029E
:104170009B18E41A6043490204F0ECF9A0225202B1
:10418000030000921949220004A806F06BFE04A85F
:1041900000F0D4FF37B0F0BDFF226B6829689C4661
:1041A0000233FF180B12013613409C4200DA1C0048
:1041B000FF200A14024003926246014001920091DE
:1041C000039A0B4904A806F04DFE04A800F0B6FFC0
:1041D0002800FFF785FE0500ADE7C046F810002077
:1041E00032D00000FC10002000C0FEFFDCCF000039
:1041F0001ED0000070B50020FFF70CFE0400012067
:10420000FFF708FE844200DA04000A4B1D686A4288
:10421000554128001D60FFF7EDFDA0226B425202C0
:104220001340054A28009B18044A611C1360FFF7DD
:1042300015FE70BDF810002004800100FC10002065
:10424000F8B50020FFF7E6FD07000120FFF7E2FDCB
:104250003E00204D0643204C0DD18021C020C902D4
:104260004002FFF7ADFD01213000FFF7F7FD1B4BCA
:104270002E6023601DE0874209DD0023B0212B6002
:10428000164B8902236023680020012517E00123D3
:1042900080212B60124BC9022360F4E7120E522AD0
:1042A00008D0002800D023600E4800F047FFFFF739
:1042B000A1FFF8BD28005A68023292009B188B4279
:1042C00005D21A68561CE9D10028F2D0D1E7216046
:1042D000EFE7C046F8100020FC1000200480010029
:1042E00004C00200F7CF0000F0B585B003920322AE
:1042F0000333DC17294D1440E4182B68284F5A4229
:10430000534180225B42D202A4103B409B18A21C66
:104310000291244E910000910190316800980A1892
:10432000934215D2FFF71AFE2B685A42534180225E
:104330005B421F40D202BF183368009A9B189F420D
:1043400006D2194800F0FAFE0025280005B0F0BD9D
:10435000029B356819066B461A7BA423DB051343C1
:10436000FF222F00090C1943019B12041B04134068
:1043700019432800FFF760FD0837281D210037602A
:10438000FFF75AFD002C04D00A9A21003800FFF7ED
:1043900079FD009B083BFF183760D6E7F810002036
:1043A00000C0FEFFFC1000209BCF000010B5FFF7FF
:1043B000D5FD10BD70B59AB0FFF742FFFF221E4C2D
:1043C000D2000021200006F009FAFF25FFF7B2FD18
:1043D0000026002814D10200C300E3580130591E02
:1043E0008B41D218FF28F7D1144901A806F03AFDF5
:1043F00001A800F0A3FE124800F0A0FE1AB070BDA4
:1044000003681A142A400A2A0AD11A122A40FF2ADB
:1044100003D0D200A1180B71A050FFF761FDD8E7BF
:10442000132AFAD11B122B40FF2BF6D0DB00E21827
:104430001671E650F1E7C0468425002067D00000E1
:104440007BD000000021094B094A596001315160BD
:1044500059680029FCD000211961012393600222D0
:10446000044B8131FF315A501A607047FC100040F4
:104470000010004000E100E00222064B0121DA6753
:104480000022054B5A61054A11615A69002AFCD085
:104490007047C04604E100E0FC10004000100040FE
:1044A00010B5044C2378002B01D0FFF7E5FF002066
:1044B000207010BD01120020802301205B055B6E7F
:1044C0005B001843704700000120024B1B685B0033
:1044D00018437047841200200120024B1B685B00C8
:1044E00018437047240000200120024B1B685B002A
:1044F000184370478812002070B504000D001600A4
:10450000FEF7CAFA802301215B055A6E2670002649
:1045100053006170E1706272010A5A0A6071A17100
:10452000A272010C5A0C000E5B0EA6702571E1718F
:104530002072E272237370BD10B5044C200006F0A7
:104540003FFD01002000FEF749FF10BD8D12002045
:104550000E4B10B51B680E4C5A1C0FD00D4C002B87
:104560000CD00D4C012B09D00C4C022B06D0094C61
:10457000042B03D00A4C052B00D1074C200006F079
:104580001FFD01002000FEF729FF10BD28000020BC
:1045900013D100000CD100001ED1000023D1000077
:1045A00018D1000070B5214C2278002A3DD1204B53
:1045B00001215A608022D20511605A68002AFCD07D
:1045C000002207201B4B1C4901255A500439585022
:1045D00008315A5019481A4958501A491A485A501D
:1045E0001A495A50A622D2009D50082218495A5002
:1045F000043158500220174958501749174858504D
:10460000174804395850182016495850C1218900BC
:104610005A500539FF395858921802435A501249D6
:10462000124A9950FFF70EFF257070BD011200204D
:10463000FC000040001000400C0500007469627529
:104640001C05000024050000200004022C050000C9
:1046500014050000340500003C050000FFFF0000C9
:104660002110010054050000021200200405000082
:1046700070B50E4B06001B78002B01D1FFF792FF9F
:1046800000200B4D2C7884420ED00A4B2022197842
:104690000323091B1940084B4901C918300006F0D3
:1046A00081F80120013C2C7070BDC0460112002031
:1046B0008C1200200012002002120020002370B58E
:1046C00088B0984235DD0D6801262C0034409C42AC
:1046D0002FD12300042D2CD90F222B681A40230040
:1046E000092A26D16A683F2A23DD6846FFF7C0FF02
:1046F000230000281DD06B4619783300A14203DB4C
:104700006B461B5D5B003343A200AA180134936023
:10471000202CF2D1092169444A780B7812021A43FD
:104720008B781B041A43CB781B061343024A136091
:104730000423180008B070BD8812002070B5454BE6
:104740008AB01B78002B01D1FFF72CFF02AC2000B0
:10475000FFF78EFF002802D100200AB070BD237839
:104760000B2BF9D96378012BF6D1E378012BF3D128
:1047700000231120384E394D33602B706844237963
:10478000374A417813600278090211438278120493
:104790001143C27812060A4332490A60002B0ED137
:1047A000152169444A780B7812021A438B781B044E
:1047B0001A43CB781B0613433360002318E0012B08
:1047C0001AD1152169444A780B7812021A438B7862
:1047D0001B041A43CB781A211B06134333600E23A4
:1047E000627C6944934200DD130000229A422CD17E
:1047F00000220420EA54B0E7022B03D1627B10337D
:104800001621EEE7042B0DD11521082269446846D4
:1048100005F0C8FF0098019902F048FA05F074FE0F
:104820003060CAE7052BC8D11521082269446846C3
:1048300005F0B8FF0098019902F038FA05F064FE1F
:104840003060627D0A231E21CBE7885CA8540132C8
:10485000CCE7C04601120020841200208D120020F7
:10486000280000208812002010B5134B04001B788C
:10487000002B01D1FFF796FEFFF7FEFD00200F4A47
:104880000F49104B54505860013010605868002890
:10489000FCD0002018610130906018690028FCD01D
:1048A000094B0A481B785B011B185350FFF7E4FDC6
:1048B000FFF7C8FD10BDC0460112002000100040E7
:1048C00004050000FC10004000120020021200202D
:1048D00010B588B000281DDD0A68012113000B40C7
:1048E00018D1042A16D90F2014682040092811D1A4
:1048F00050683F280EDD9800101880680024084298
:1049000001D04010C4B26846C4540133202BF2D108
:10491000FFF7AAFF002008B010BD000010B5002866
:1049200013DD0C68E30710D56410532C0DD8084B29
:104930001B78002B01D1FFF735FEFFF79DFDA1236A
:10494000044ADB00D450FFF77DFD002010BDC046B7
:10495000011200200010004010B500280EDD0C6888
:10496000E3070BD56410FF2C08D8054B1B78002BF0
:1049700001D1FFF717FE034A034BD450002010BDAE
:1049800001120020001000402405000013B500288B
:1049900014DD0C68E30711D5094B64100093094B33
:1049A0000193072C0AD8084B1B78002B01D1FFF785
:1049B000F9FD6B46054A1957054BD150002016BD2D
:1049C000E2ECF0F4F8FC00040112002000100040BA
:1049D0000C05000070B588B0002820DD01240868AF
:1049E00004401CD104281AD90F2302681340042B59
:1049F00015D1FEF7E5FA060006F0E2FA05001228E6
:104A000000D912252A0002210D326846FFF774FDF5
:104A10006B465D73A54205DC6846FFF725FF002065
:104A200008B070BD2300325D6B449A730134F1E726
:104A3000F0B50D008BB0012832DD086801220400BA
:104A400014402DD104282BD90F2301680B40042BCF
:104A500026D16B68134223D0FEF7B2FA6E680700C6
:104A60007310019306F0ACFA05000E2800D90E254C
:104A70002A000121113202A8FFF73EFD6A46127991
:104A800002AB5A7302AA73129373019B76141B0E26
:104A9000D67313745574A54205DC02A8FFF7E4FE33
:104AA00000200BB0F0BD3A5D02A963189A7401347E
:104AB000F1E730B589B0002814DD0C68E30711D5A3
:104AC000102268460021FFF717FD6B466A46651005
:104AD0005D73684663122D0E64149373D47315745A
:104AE000FFF7C2FE002009B030BD0000174B184A86
:104AF0005968002903D0002159600131916019697A
:104B000000291FD0002018618023DB00D3581149F1
:104B1000012B18D1A923DB00D3585B420B600E494F
:104B20000B78032B01D801330B7003200B490B7852
:104B3000013303400B700A495B015B18094953506C
:104B40000123936070470860FAE7C046FC100040FC
:104B500000100040240000208C12002000120020D1
:104B6000021200200405000010B5034A102103487A
:104B700000F0C6F810BDC0468CD0000083D0000005
:104B8000044A05491368C85401339B059B0D136003
:104B90007047C046BC160020BC12002070B5114CF6
:104BA000114A2368834202DC0023236016E0155C6F
:104BB000411C2E00FA3E012E05D899420FDA555CB1
:104BC000013D1F2D01D90800ECE70100151A565CC4
:104BD0006E5401318B42FADC181A206070BD1570DA
:104BE000FAE7C046C81A0020C816002010B5FDF725
:104BF00049FF064B1A68824201D900221A601B68DD
:104C0000C31A034898428041404210BDB8120020A8
:104C1000204E000010B5094C094A236812689342DF
:104C200000D110BD074AD05CFEF74CF90028F8D03F
:104C3000236801339B059B0D2360ECE7C016002021
:104C4000BC160020BC12002010B50400064B074A19
:104C50001B6812689B1ADB439B059B0DA34200DB7C
:104C600010BDFFF7D7FFF1E7BC160020C0160020EB
:104C700070B50020FFF734F9FF260500002801D1A8
:104C8000280070BD03681C143440FFF729F9DA2CA2
:104C9000F4D10500F2E7F7B5050056680191B000C0
:104CA000441C06301700FFF7CFFFFB20FFF768FF1B
:104CB0001C20FFF765FFE8B2FFF762FFE0B22412A5
:104CC000FFF75EFFE0B2FFF75BFF6B461879FFF777
:104CD00057FF0025AE4200DCF7BDAB00FB189C6817
:104CE0000135E0B2FFF74CFF2012C0B2FFF748FFDA
:104CF0002014C0B2FFF744FF200EFFF741FFE9E7A1
:104D000070B5074E3368092B08DC0C255D43054C54
:104D10000133285164196160A260336070BDC046E0
:104D2000C41600201C2F0020F0B587B002900C00A4
:104D3000012803DC1B20FCF71BF945E0244B086825
:104D40000093C30709D4042807D90F23026813402E
:104D5000042B02D1FEF734F900901D4B60680193DB
:104D6000C30709D4042807D90F2302681340042B72
:104D700002D1FEF725F901900027164B1B6804931A
:104D8000049BBB42D6DD0C267E43134B0099F618DC
:104D9000306806F00BF9051E05D17368B6680593F7
:104DA000059B9D4201DB0137EAE7306801990396D4
:104DB00006F0FCF80836002808D121000298039B71
:104DC000083102385B68984707B0F0BD0135E7E766
:104DD000A2CA0000C41600201C2F002010B5FBF74B
:104DE000FFFFFEF7E1FFFEF70FF8FEF76FFBFEF7A0
:104DF000BDFBFFF7B9FE00F063FE01F021F810BD26
:104E0000962210B512010021034805F0E7FC0022AC
:104E1000024B1A6010BDC046241C0020C8050020AB
:104E2000064B074A1B6812689B1ADB439B059B0DC8
:104E30000122834200DC002210007047BC160020D3
:104E4000C0160020F8B505000C0016001F1E0ED17C
:104E50000320FFF7E5FF002808D0FA20FFF790FEB7
:104E6000E8B2FFF78DFEE0B2FFF78AFEF8BD501DF5
:104E7000FFF7D6FF0028F9D0FB20FFF781FEE8B24C
:104E8000FFF77EFEE0B2FFF77BFEF0B2FFF778FEA1
:104E90003012C0B2FFF774FE3C00E31B9E42E5DD1A
:104EA0002078FFF76DFE0134F7E7000070B50024AD
:104EB000F0250B4B1B68A34202DCFFF7A1FF70BD7E
:104EC0002B006343074A9B181A78002A05D05978AB
:104ED000002311201A00FFF7B5FF0134E9E7C046AF
:104EE000C8050020241C0020F8B507000024F02588
:104EF0002B0063430C4A01349E18B74211D031781D
:104F000000290BD00133D15C002311201A00FFF7D8
:104F100099FF2A000021300005F060FC0A2CE7D13F
:104F2000F8BD024B1C60F9E7241C0020C8050020D6
:104F3000F0B5150001222F005E4C1740A5440190EA
:104F40000291002F11D005AB1A706A105A70120E20
:104F50001A710522691299706D140299DD70FFF7BC
:104F600071FFCF239B009D44F0BD042D1ED90F235C
:104F70002A681340042B25D1023B04AA2800137190
:104F8000FEF71EF8040006F01BF84B4B984200D9C0
:104F90001800B84204DC421C05AB02990198DEE718
:104FA00001377B1EE35C05AAD355F2E7042D7CD1C3
:104FB000032304AA043D13716B425D4105AB557197
:104FC0000222EAE7092BCCD1042205AB1A706A68E9
:104FD000511000916946521209789A70009A5970DE
:104FE0001F2A01DD202200926A46127806ACDA7090
:104FF000009BBB4202DC05ABE21ACEE70126BB00F8
:10500000EB189868064006D1042837D90F230268A8
:105010001340022B0CD10123237043106370421202
:105020001B0E4014A270E070237105340137DFE7D6
:10503000042B21D1023B2370FDF7C2FF039005F042
:10504000BFFFA31C0C2809D86070864201D19C19AF
:10505000ECE7039A925D9A550136F6E70C226270EE
:10506000039A925D9A550136092EF9D12E23E372E7
:10507000237363730E34D9E7012B07D1032304385C
:1050800023704342584160700234CFE7092B09D1A5
:10509000053B23704368E6705A105B126270A37080
:1050A0000434C3E726700134C0E7002D00D058E770
:1050B0007EE7C046C4FCFFFF2303000070B502007A
:1050C0000024F0210D4E0800604380194578954278
:1050D00003D001340A2CF6D170BDF022002105F076
:1050E0007DFB074A1368013BA34200D114600023F3
:1050F00029001A001120FFF7A5FEEDE7241C00206F
:10510000C805002010B5B2B002236A46040013702F
:1051100005F056FFC72800D9C7200023984207DCB6
:10512000421C6B46FE211420FFF78CFE32B010BDEE
:10513000694601335A1EA25CCA54EFE730B5B3B0DA
:1051400002236A460500137005F03AFF0400C728E1
:1051500000D9C72400239C420BDC20003230FFF72B
:1051600073FD621C6B46FF211420FFF76BFE33B00A
:1051700030BD694601335A1EAA5CCA54EBE70000F1
:10518000F7B5234B06001B68F02100930023009A1B
:105190009A4211DC0024F0231A0062430192019923
:1051A0001C4A55182F78002F12D001340A2CF3D145
:1051B0001948FFF7C3FF29E00A005A43154882182F
:1051C0005078B04202D11278002A1FD10133DEE7B5
:1051D000F0223900280005F001FB02230D4A019955
:1051E000EB6053540D4AF1008A58009B6E70AE700C
:1051F000AA602F616F61A34202DC054B01341C6081
:10520000002331001A001020FFF71CFEF7BDC04636
:10521000C8050020241C002025D60000842500207D
:1052200010B5FFF743FEFF24084AE3005B429B18DA
:10523000074AD35C043B012B03D8E043C0B2FFF71D
:105240009FFF013C002CEFD110BDC046FC070000C1
:1052500084250020F7B50F00FF247F2501901E4A0A
:10526000E300D31A1D4A9A181278062A01D0032A9D
:1052700020D1FF22D2009B18186883682B401C2B7A
:1052800018D1C3681A002A40042A13D102692A409F
:10529000192A0FD11B0A01339B000C30C018FDF7EF
:1052A0008FFE03780600002B10D005F089FE002346
:1052B000B84209D0013C002CD1D1F7BD019AF15C74
:1052C000D25C9142F6D101339F42F7DCE043C0B299
:1052D000FFF756FFEEE7C04684250020FC070000DC
:1052E00070B50500FF24084AE3005B429B18074A9B
:1052F000D35CAB4203D1E043C0B2FFF741FF013CB6
:10530000002CF0D170BDC046FC07000084250020B1
:10531000F7B5FDF7B7FB514B1A68824201D900225D
:105320001A601A684E49821A8A4200D883E01860CF
:10533000FDF7B2FB071E00D101370020FDF79EFCF0
:1053400001900020FDF7AEFC019B0090454C464DBE
:10535000002B14D02368002B00D07AE02B68276044
:10536000002B00D171E0414B01261B78002B63D14B
:105370000920FFF7B5FF3E4B1E703C4B1E70009B93
:10538000002B12D02B68002B0FD123682F60002B2D
:105390001ED0374B01261B78002B52D10920FFF776
:1053A0009FFF334B1E70314B1E702368002B0FD0B4
:1053B0002F4E3278002A0BD19F4200D227602368FB
:1053C000FB1A312B04D90720FFF78AFF0123337022
:1053D0002B68002B0FD0254E3278002A0BD1BB4210
:1053E00000D92F602B68FF1A312F04D90820FFF74E
:1053F00077FF012333702368002B0CD0019B002B17
:1054000009D11B4E3378002B02D10720FFF768FF2C
:105410000023236033702B68002B0CD0009B002BE3
:1054200009D1124C2378002B02D10820FFF758FF36
:1054300000232B602370F7BD0720FFF751FF0C4BB3
:105440009CE70820FFF74CFFADE7009B002B9CD1A9
:10545000ABE7009A002A95D1AAE7C046B412002013
:105460000F270000A4120020AC120020B012002070
:10547000A812002037B500240500FFF717FD01A88A
:105480000194FDF7E9FB21002000FEF759F9FEF732
:1054900035FBFDF795FCFDF7AFFCFEF77BFCFDF758
:1054A00017FBA54204D0FDF737FD0248FFF746FE83
:1054B00037BDC04616D60000002310B501001A0003
:1054C0001120FFF7BFFC10BD07B56B461970694688
:1054D0005A7013128B701314120ECB700A716B4634
:1054E000010005221320FFF7ADFC07BD10B50A002F
:1054F00001001220FFF71CFD10BD70B5050008006B
:105500000C003230FFF7A0FB2B00220000211B20F3
:10551000FFF798FC70BD10B50C00030011001420BB
:105520002200FFF78FFC10BD012370B5FF24084A4D
:1055300041185B42884201D3D84370BD06781D0AEA
:10554000234073409B009B5801306B40F2E7C046FC
:10555000F8D10000002313B501930B4BC2000400E7
:10556000D058002805D0436808309900FFF7DCFFC9
:1055700001900920FFF768FB01AB042221001720EE
:10558000FFF760FC13BDC04684250020F7B50190ED
:10559000FFF76EFB01250400FF276D42002C01D1AF
:1055A0002800FEBD266833143B40152B0DD1210089
:1055B0000198083105F0FAFC002801D135123D4070
:1055C0002000FEF78DFC0400E8E71D2BF8D1012533
:1055D0006D42F5E7F0B580279DB0FFF71BFBA54CAA
:1055E000A54D2068FF00391A4019FDF751FC2368CA
:1055F0000600C3182360002B0ED11DB0F0BD20683B
:10560000391A2818FDF744FC236806001B1823608C
:10561000FDF738FA994B1860002EF0DC2B78FA2B46
:1056200000D037E12368022B07DCFFF7DFFA002800
:10563000E3D00120FFF7B2FADFE76878AC780238F0
:1056400018282BD802F0F2FE19002C00300034008C
:10565000370040002A004A007C0086008A00A00033
:10566000F10002012A002A002A002A002A002A004A
:105670002A002A002A002A001001FF2C0ED0200048
:10568000FFF71CFD00227E4BE100CA505B181A7127
:105690002100009213001320FEF726FE0320C9E725
:1056A0002000FFF76DFDF9E72000FFF707FDF5E7A4
:1056B000FFF7B6FDF2E7FFF7F9FB0020FFF7DAFE90
:1056C0007048FFF73BFDE9E7632CE7D86E4BA2007B
:1056D000D25821001520FFF72BFCDFE7FFF7C8FAAF
:1056E000FF270400002CD9D025682B143B40152B34
:1056F00004D02000FEF7F4FB0400F3E7200008309C
:1057000005F05EFC06000530FFF79EFAFB20FFF770
:1057100037FA2D121D20FFF733FAE8B2FFF730FAFF
:10572000F0B2FFF72DFA3012C0B2FFF729FA2500C8
:105730002B1B9E42DDDD287AFFF722FA0135F7E7C1
:1057400000211D2000910B000A00FEF7CDFDFDF7A2
:10575000E3FBA3E72000FFF7FDFE9FE7FDF7A4F9B9
:1057600003AC4A4A64210090494B200005F048FBF5
:1057700002232000237005F023FC230002000021F7
:105780001620FFF75FFB89E700243D4AE300D55868
:10579000002D27D06B689E00701DFFF755FA2B0077
:1057A00000253200083321000120FFF74BFB2F00BA
:1057B000FFF75EFA2E00002818D1002F04D03A001F
:1057C00001212000FFF767FA002D04D02A000221F2
:1057D0002000FFF760FA002E04D0320000212000E4
:1057E000FFF759FA0134FF2CCFD157E7FF210368A7
:1057F0001A120A40A24209D11A140A400B2A08D1EF
:105800000B400CD0012B0CD0022B0CD0FEF768FB08
:10581000D1E7132AFAD100252F002E00F6E7060063
:10582000F4E70700F2E70500F0E70024FFF73EFB8E
:105830002200210000942300DA20FEF755FDFF220C
:105840002100D2000E4804F0C9FF80E7012C02D1EC
:10585000FEF768FC22E7022C02D1FEF7A7FD1DE748
:105860000120FFF707FE19E7002321001A001A2084
:1058700087E7C046C81A0020C8160020B8120020CA
:1058800084250020F8D500007C2D00200FD60000D4
:105890000AD60000FB2B00D0CBE62268042A00DCED
:1058A000C3E62E79E878574B360206439E4200DD68
:1058B000BFE6331D9A4200DCB7E6EB5CFE2B00D05E
:1058C000B7E66B78AC78771E1B2B61D019D8072B05
:1058D00047D0082B1CD0012B18D1FF2C16D020004C
:1058E000FFF7ECFB6D79484AB31E009221002A00B5
:1058F0000A20FEF7F9FC454BE400E0501B191D712E
:1059000004E01D2B56D048D31E2B6AD0701D91E6A3
:10591000632CFBD86A79022A13D0032A1BD0012AF0
:10592000F4D1E979AB79090219432B7AA4001B045D
:1059300019436B7A1B060B435B001343344AA35095
:10594000E4E7002FE2DDB11E2F48FDF747FD304BA5
:10595000A400E050DAE7AB79A4005A1E93419B0003
:10596000ECE7632FD2DC03AD3A002A49280004F0AB
:1059700019FF00232800EB55FFF708FE0028C5DBC0
:10598000234B8000C25821001520FFF7D1FABDE754
:1059900039002048FFF75EFCB8E7FF2CB6D06A79E3
:1059A000022AB3D818490B2000912100B31EFEF73C
:1059B0009BFCABE7632F00DD6327002303A99F4215
:1059C0000ADCFB430022DB173B40CB181A70152082
:1059D00000917B1C2100EAE7EA185279CA5401338E
:1059E000EDE7012C92D1002F90DD6B79002B03D0D5
:1059F0001C00322B00DD322464235C43064B1C6008
:105A000084E7C046F6030000CE160020842500205F
:105A10007C2D0020CD1600200400002001207047BE
:105A200010B5064C200000F041FB0549200000F0B5
:105A300065FB0122034B1A6010BDC046F41A00201A
:105A4000801A0600CC1A002010B501210D20FDF7A8
:105A500031F801210E20FDF72DF800210F20FDF770
:105A600029F8044C200000F05DFA1021200000F01D
:105A700075FA10BDD41A002010B504680D20E30794
:105A800003D56410FF2C03D91720FBF771FA10BD62
:105A9000FFF7DAFFE1B2024800F082FA0020F6E7F1
:105AA000D41A002010B5FFF7CFFF0021034800F003
:105AB00077FA43000120184310BDC046D41A0020D5
:105AC00010B5034A08210348FFF71AF910BDC04674
:105AD0003CD600007CD60000F8B5012306681E42C3
:105AE00005D045681D4202D084681C4203D10D20B8
:105AF000FBF73EFAF8BD76101520802EF8D86D1011
:105B00001620FF2DF4D86410FF2C01D91720EFE7E1
:105B10000B4B1B68002B01D1FFF782FF094FF1B23D
:105B2000380000F082FBE9B2380000F085FAE1B2FB
:105B3000380000F081FA380000F0E2FB0020D9E7DD
:105B4000CC1A0020F41A0020F7B50122140090426C
:105B500022DD0D682A421FD01D4B15411B684C6881
:105B6000002B01D1FFF75CFFE9B201272500194E98
:105B70003D40300000F059FB002D0FD03C4130007B
:105B8000E1B200F059FA300000F0BAFB0024A04264
:105B900002D02320FBF7ECF92000FEBD042CF2D943
:105BA0000F2322681340092BEDD163685B1001932A
:105BB000019BAB42E7DDAB00E3189968394204D0A2
:105BC0004910C9B2300000F037FA0135F0E7C0469D
:105BD000CC1A0020F41A0020144B70B51B68050085
:105BE0000E00002B01D1FFF71BFF114CEDB2290075
:105BF000200000F01AFBF1B2200000F01DFA002195
:105C0000200000F01DFB002801D0404270BD0122A1
:105C10002900200000F004FB200000F0FEF900281D
:105C2000FAD0200000F0FEF9F0E7C046CC1A0020C0
:105C3000F41A002010B501240368234202D0416801
:105C4000214203D10D20FBF793F910BD5810802895
:105C500001D91520F7E74910FF2901D91620F2E7ED
:105C6000FFF7BAFF40002043EFE710B5040001281A
:105C700014D105211820FFF7AFFF7F282BDC03008C
:105C80007F3301DA7F20404264235B4258437F2107
:105C900002F060FC052C00D1404210BD032811D158
:105CA00001001820FFF798FF7F2814DC03007F33E2
:105CB00001DA7F20404264235B4258437F2102F097
:105CC00049FCEAE70020052CF5D107211830FFF741
:105CD00083FF7F2802DD0138FF38D0E703007F33E0
:105CE00001DA7F20404264235B4258437F2102F067
:105CF00031FCD1E770B50120FFF7B7FF04000320A6
:105D0000FFF7B3FF05000520FFF7AFFF6D436443C6
:105D100040436419201804F02DFC01F0F7F804F05A
:105D2000F3FB43000120184370BD10B50120FFF7BD
:105D30009CFF43000120184310BD10B50320FFF75E
:105D400094FF43000120184310BD10B50520FFF754
:105D50008CFF43000120184310BD10B50821182006
:105D6000FFF73AFF0300C00FC018012340101530A1
:105D70004000184310BD0000F8B501231C009842F4
:105D800029DD0F683B4226D04E6835001D4022D1E8
:105D9000042E20D90F2231680A40092A1BD17368CA
:105DA0005C10202C00DD2024134B1B68002B01D13C
:105DB000FFF736FE7F10F9B2104F2200380000F0D6
:105DC0002FFAA54214DA380000F027F9002804D190
:105DD00001246D002C432000F8BD380000F022F9AA
:105DE0000122AB004000F31810439860AD18E8E7BB
:105DF00064000125EEE7C046CC1A0020F41A00200A
:105E00000020704701207047002070470020704735
:105E10000120704700207047002070470020704725
:105E20000020704700207047002070470020704716
:105E3000002070470020704770477047704700008F
:105E400010B5034A0E210348FEF75AFF10BDC046A5
:105E5000CCD600003CD7000010B5FCF7E1FFFDF701
:105E600081F8FEF7BBFF0448FFF768F9FEF7A2FAD6
:105E7000FFF7D6F910BDC046C5D7000010B5FCF736
:105E8000DDFC10BD70B5002504AC24780573A94273
:105E900005D10A4B0A4A23210A4804F015FC016087
:105EA0000949920052589B0002715B58A40083710B
:105EB0006358856043710223C37170BDDDD7000054
:105EC0003FD80000EBD700009CD80000037B002BDC
:105ED00004D143738373036101330373704700007C
:105EE0001FB50191A02100240068C900D2B244501E
:105EF000012A10D0A24209D0032A0AD0074A8350AF
:105F0000074B019AC250012343501FBD0222134385
:105F1000F4E70422FBE70622F9E7C0465405000037
:105F20002405000010B50400FFF7D0FFA12223686C
:105F3000A179D20099506179064A200099502179BF
:105F400004329950044B19685A689B68FFF7C8FFE0
:105F500010BDC0460C050000E81A00204BB2002B13
:105F60000FDB80233F290FD81F290FD80F290FD807
:105F700007290FD803290FD81B060168074A8B5041
:105F8000704780239B04F8E7DB04F6E71B05F4E782
:105F90005B05F2E79B05F0E7DB05EEE72405000073
:105FA0000368074A99501A00FC32D1680029FCD0D6
:105FB000A321C90058580023C0B2D3607047C0461F
:105FC0001C05000007B58022074BD2051A6000228D
:105FD0009A6002321A7111230E320093034905337D
:105FE0000348FFF74FFF07BDE81A002000300040CC
:105FF000D41A0020F8B505000E0017000024BC429A
:1060000008D02B68315D1B6828009847002801D014
:106010000134F4E72000F8BD704710B51C3000F0E3
:10602000A9F910BD10B51C3000F096F910BD10B5DF
:106030001C3000F0A5F910BD70B5437E0D00002B9B
:1060400001D1002070BD6430040000F0A2F90028E6
:10605000F7D12000290000F070F90120F2E70000DC
:10606000F7B50193FA23002504009B0083600D4BD4
:106070004560083303601C300F00160000F052F931
:106080002000643000F04EF9074A2761B600B3588B
:1060900020006375019B9B009B586576A576A375D0
:1060A000FEBDC0467CD800009CD800000123A02281
:1060B000C375837D0E49C133FF33D2059B009950D0
:1060C000437DC133FF339B009950CC220169094BBA
:1060D0005204CA5005220169243BCA50827D0169DD
:1060E0000833CA500269417D034BD1507047C04606
:1060F0000C060000240500000C050000A02200236F
:1061000010B50469D200A3500A4CA1420FD90A4C21
:106110008C425B4109495B420B40CD21C9045B18AD
:1061200004690749635005210369995010BDCC23C8
:106130005B04F5E7A086010090D00300000098FD05
:1061400024050000F7B5040000200D0001938242F1
:1061500065D01600402A00D9402627001C37380099
:1061600000F0F6F8B1232269DB00D550802201232C
:10617000216992008B50A27E002A03D1226913620A
:10618000226913600025731EAB4207D1019B002BCF
:1061900004D08022022123699200995001222369B0
:1061A0001A622369FC33DA68002A02D19A6A002A4B
:1061B000F9D09A6A002A0BD1DA60A3232269DB00A6
:1061C000D1583800C9B2013500F0B7F8B542DAD37A
:1061D000019B2269002B0FD11300FC339B6A002B1B
:1061E0000AD10133A376D3612369FC33DA6C002A28
:1061F000FCD00022DA640AE000230121A376516179
:106200001A002369FC3399680029FCD09A6023693D
:10621000FC339A6A002A01D000229A62E8B2FEBDDD
:1062200010B50123FFF78EFF10BD0300AC3310B58E
:1062300004001970643000F08BF80123637610BD00
:106240000023020070B5AC3243760D001178B12204
:1062500004000069D20081508022216992008B5095
:10626000226901331362226993602600643630008C
:1062700000F080F8002812D0300000F06DF81E4BBE
:106280002269D0502369FC331A6A002A02D19A6A23
:10629000002AF9D09A6A002A01D11A62E5E7236937
:1062A0000122002D0DD11900FC31896A002908D185
:1062B000DA612369FC33DA6C002AFCD00022DA644C
:1062C00007E05A612369FC339A68002AFCD0002257
:1062D0009A6000202369FC339A6A82420BD098624C
:1062E0002169064A8B588B501800022B03D0181FC7
:1062F000431E9841033070BD1C050000C40400001B
:1063000010B50121FFF79CFF10BD000010B513234D
:10631000122202490248FFF7A3FE10BD00400040D0
:10632000F41A002010B540220021040004F056FAAF
:10633000002320002364636410BD10B53F24026C69
:10634000531C2340446C9C4201D08154036410BD13
:106350000023036443647047436C026C934206D08D
:106360003F21C25C01330B404364100070470120A1
:106370004042FBE7036C406C181A00D54030704770
:10638000436C026C934201D0C05C704701204042D4
:10639000FBE73F22036C406C01331340181A434261
:1063A0005841C0B27047000003210A4802680A43FE
:1063B0000260094802680A4302600849084A094B1A
:1063C0009B1A03DD043BC858D050FBDC00F012F8E8
:1063D000F9F79AFE240500405405004008DE00004D
:1063E0000000002060020020FEE7FEE7FEE7FEE777
:1063F000FEE7FEE72D4B10B51A68D2B2012A0FD185
:106400002B4A126812070BD12A4AE0241168F022A5
:106410000800104021422DD12749096811422CD093
:106420001A68D2B2012A12D12149096809070ED18E
:10643000F020204909680140402908D11E49096817
:10644000014204D18020C121C005C90042501B680F
:10645000DBB2012B0DD1164B1B681B0709D1154B65
:106460001A68F0231A40A02A0FD1134A12681A4260
:106470000ED010BD3028CFD0D2E7104A104911609D
:106480008021104A09021160CAE7D02AF1D1ECE755
:106490000D4B1A68012A04D00C4A1A601A68012AA6
:1064A000FCD1C0220A4B1A60E3E7C046E00F00F0BF
:1064B000E40F00F0E80F00F0EC0F00F004050040DE
:1064C000DFFF07C0186C004000EC06407593000029
:1064D00014EC06400120704710B503681322DB69F5
:1064E000984710BD70470000054B0269D150036901
:1064F000FC331A6A002AFCD0002201201A6270477D
:106500001C050000030010B55C331A781F231A40E5
:106510001E3B19009140114AD167C222042104692F
:106520009200A150026953600269D360A023002247
:106530000169DB00CA5001230169094A5B428B50A3
:106540000169084A8B5001690C3A8B500169083285
:106550008B501430FFF7FCFE10BDC04604E100E094
:106560000C0500001405000010B51430FFF702FF01
:1065700010BD10B51430FFF703FF10BD10B5143077
:10658000FFF7EAFE10BD0000030070B55E331A7815
:106590000469724BE25003005D331A780469704B52
:1065A000E250030061331C7802696E4B012C00D06D
:1065B0009EE005005F352E78A225ED0056510200C1
:1065C00060321578A1220669D200B5500269D45014
:1065D0009623DB00994200D88CE096231B01994258
:1065E00000D88AE096235B01994200D888E0962380
:1065F0009B01994200D885E0E1239B01994200D894
:1066000082E09623DB01994200D880E0E123DB01A0
:10661000994200D87DE096231B02994200D87AE087
:10662000E1231B02994200D877E096235B0299424E
:1066300000D874E0E1235B02994200D871E0E123C5
:106640009B02994200D86EE0474B994200D86CE01B
:10665000E123DB02994200D86AE0E1220023120321
:106660008A425B41414A5B421340802252059B189B
:1066700001693F4A8B50A02304220169DB00CA5004
:1066800000210369FC33D9600369FC3319620123DB
:1066900001690B6001698B60C12104698900625046
:1066A0001F215C3002780A4093406231314AFF3149
:1066B00053500021415600293CDA0F230B40083B80
:1066C0002D4C9B089B001B1903242140A140FC3446
:1066D0008C40DD69A5432C00C0258D402900214355
:1066E000D9611F23017819401E3B8B40136070BD98
:1066F00000246CE79E23DB02BAE79D231B03B7E768
:106700001E4BB5E71E4BB3E7EC239B03B0E71D4BD5
:10671000AEE71D4BACE71D4BAAE71D4BA8E71D4B91
:10672000A6E71D4BA4E71D4BA2E78023DB049FE7F0
:106730001B4B9DE78C080F4BA400E41803230B4070
:10674000FF21C025DB009940AD0066598E43310022
:10675000C0269E4033000B436351C2E70C05000086
:10676000140500006C05000090D0030000D0BEFEB0
:106770002405000000E100E000ED00E000B013009F
:106780000050270000A04E0000F0750000509D0052
:1067900000F0EB0000903A0100E0D70100B0AF0339
:1067A00000705F07F7B5009308AB1B7800250193D5
:1067B000FA2304009B0083600E4B4560083303609E
:1067C00014300F001600FFF7ADFD23005C33276186
:1067D0001E70009B084A9B00995823005D33197076
:1067E000019B20009B009A5823005E33DD701A70D5
:1067F000FEBDC04618D900009CD80000036910B542
:106800001A00FC32D2680400002A0AD0A322D20067
:1068100099581430C9B2FFF790FD00222369FC3368
:10682000DA6010BD10B50248FFF7E8FF10BDC046A2
:10683000AC1B00201D2307B502220093024901333F
:106840000248FFF7AFFF07BD00200040AC1B00204F
:1068500010B5002801D004F07DFA10BD704700008B
:1068600010B500F011F8FFF7F9FF012000F000FA71
:10687000FFF7F2FAFFF702FB024B002BFAD000E021
:1068800000BFF7E700000000C420114B80001A5839
:1068900010491140C02212020A431A50C02180221E
:1068A000490092025A501A608023A3220021DB057E
:1068B000D20099500122F9309A60074BFF301950ED
:1068C000C120023180001950403019501A607047C1
:1068D00000E100E0FF00FFFF00100140014B1860E5
:1068E0007047C04674000020F7B500231E285AD810
:1068F000384B8000C258042A5BD007D8022A54D0F3
:1069000055D80423012A09D000234CE0062A54D08C
:1069100051D31A2A53D002231B2AF5D12E4A1168CB
:1069200008294ED909294FD00A240226A020012582
:106930002A4AC00015502A482A4D07681C20BF006B
:1069400007402948019700685759009027481B02C3
:1069500007401F43C02300989B020340FF2057516C
:106960005759000207401F43019B1F43009B5801DA
:106970006023184007433E43565101251C4B1560C8
:1069800058680028FCD000205860A1230125DB00B6
:10699000D3585560A025ED0050511BB2A14202D042
:1069A00015D2611ACB401800FEBD0823B6E71023AC
:1069B000B4E72023B2E74023B0E78023AEE701230A
:1069C000ACE708240026B1E70C000126AEE7091B5E
:1069D0008B40E8E79CD80000700000200070004069
:1069E0002C0000200405000030000020FF00FFFF05
:1069F000FC700040F0B51E285BD8364B8000C258B2
:106A0000354B1E68002E30D1C227344BBF00D859F9
:106A1000334C03250440C02000022043D851C02439
:106A200080206400800018512E4F18602E4B803C4F
:106A3000D859FF3CA043D8510437D859A843204324
:106A4000D8510837D8590C35A843844607206546E5
:106A50002843D851A820C0001E50C12080268000A5
:106A600076021E501C601C4B1C60142500202B005D
:106A70001E4C2E0046433659771C1BD14343E2502F
:106A8000A0230325C132FF329200DB05D550184BFD
:106A90001A68082A14D114234343E3189A68124849
:106AA0005132FF32920059601150DA68C1239B00C5
:106AB000C250F0BD9642E1D001300328D9D1F8E7A9
:106AC000082A02D9083AD140E5E708239A1A9140EA
:106AD000E1E7C0469CD80000101C002000E100E067
:106AE000FF00FFFF0405000000900040340000207C
:106AF000740000202149F0B54A6C2148002A14D0C6
:106B0000A025A12600230124ED05F600C258571C3C
:106B100006D0C7187F68002F02D027009740AF51DA
:106B200014333C2BF2D100234B64A0230121DB055D
:106B300000260F009C4614234B43C3181A1F1268EB
:106B4000104C0E4D920014195219526C002A10D09C
:106B50001A00143A1268551C09D0103B1B68FF2B11
:106B600005D03B00934065461A00074BEA50FC34C1
:106B7000666401310429DED1F0BDC046FC900040BE
:106B800034000020009000400C05000000B51E28D5
:106B900010D80C4A8000835803290BD8A022080083
:106BA000C133FF33D2059B0001F036FC0209050713
:106BB0000021D15000BD0C21FBE70421F9E703219E
:106BC000F7E7C0469CD800001E280AD8074B800073
:106BD000C25801239340A022D205002902D10449C2
:106BE00053507047A121C900FAE7C0469CD8000065
:106BF0000C050000030000201E2B0AD8A021A222B1
:106C0000C905D2008858034A9B009B58D8400123ED
:106C1000184070479CD80000F7B506000D000C0026
:106C20008B180193019B671B9C4207D03368217826
:106C30001B683000984701340028F3D13800FEBDAE
:106C40000849094A094B10B51B688858FA22190AE5
:106C50001B0618439200002301F0B4FD4904C00B49
:106C6000084310BD0010014004050000141C002062
:106C700070B5041E09D0FFF7E3FF050000F014F81B
:106C8000FFF7DEFF401BA042F8D370BD0022044B8B
:106C90009A60044A13680133DBB213607047C04640
:106CA000FC100140141C002070470000F0B5C646DF
:106CB00000B5CB0F9846404A4B005B0D9A1882B046
:106CC0000D000400132A2FDC002A49DB3B4F17413B
:106CD0003E000E40064323D07F08390029400C4374
:106CE0000AD03749BD438C4663445C425C418023F3
:106CF000DB021341E4071D434146CE0031492B001E
:106D00008E192200346875682000290001F000FF08
:106D1000009001910098019922002B0003F090F857
:106D200002B004BC9046F0BD332A08DD8023DB00AE
:106D30009A42F5D102000B0001F0EAFEF0E7224A88
:106D40009446012263445242DA400242E8D052089B
:106D50000242D1D094438022D2051A411443CBE79A
:106D60004B005B080343DBD00B031B0B1C4363424C
:106D7000234380244D0C24031B0B23406D042B4321
:106D800019004346DA000F4B9B181C685D6802002F
:106D90000B002000290001F0BBFE0090019100983B
:106DA000019922002B0003F04BF842464B005B0890
:106DB000D60733431900B3E701FCFFFFFFFF0F00C5
:106DC000EEFBFFFF48D90000EDFBFFFFF8B5274AB7
:106DD0004B005B0D9A180C000700132A10DC002AE8
:106DE00036DB234B13410B423AD080242403144159
:106DF000002064189C430600250030002900F8BDDF
:106E0000332A0EDD80230600DB000D009A42F4D108
:106E100002000B003800210001F07AFE06000D0090
:106E2000EBE7144D0600AC46012563446D42DD409E
:106E3000AC4663460D000342DFD033239A1A323B3F
:106E400093401818874200D94C1C63469843D2E7F8
:106E5000C90FCC070020531CCDD1074B1C43CAE7F8
:106E600006000D000028C0D1C7E7C04601FCFFFFA7
:106E7000FFFF0F00EDFBFFFF0000F03F30B5214AA0
:106E80004B0087B05B0893421EDD1F4A934205DD2D
:106E900002000B0002F0D4FF07B030BD02AA00F0E0
:106EA00095F803231840049A059B012813D0022863
:106EB0001DD0002814D00298039900F06FFB8023A6
:106EC0001B069C466144E7E7002300220093002351
:106ED00001F0DEF8E0E70298039900F05FFBDBE7E2
:106EE000012402980399009401F0D2F8D4E7012418
:106EF00002980399009401F0CBF880231B069C466E
:106F00006144C9E7FB21E93FFFFFEF7FF0B547464A
:106F1000CE4680B58DB004000D0000F067FA294B15
:106F200006001B780F005BB29846013310D0220098
:106F30002B002000290003F0CBFA8146002807D15E
:106F4000002200232000290001F014FC002806D1B3
:106F5000300039000DB00CBC90469946F0BD0123BD
:106F60000293194B0694079503934B460A934346A5
:106F700004940595002B15D0002300221900100061
:106F800002F0E2F8434608900991022B0ED103F07B
:106F9000B9FB212303600A9B0193002B0CD1089EAF
:106FA000099FD5E7002300240893099402A801F063
:106FB000C1F90028EFD1EAE703F0A4FB0A9B019393
:106FC0000360ECE77800002058D90000F0B54E4689
:106FD0004546DE465746E0B5E14B4C008FB0904643
:106FE000894664089C4200DC87E0DE4B9C4222DC40
:106FF000DD4A002900DC92E0DC4B02F021FFDB4B94
:1070000006000F009C4200D17EE1D94AD94B02F024
:1070100017FF02000B00414630000A604B60390048
:1070200002F00EFFD34BD24A02F00AFF434601257D
:107030009860D9606BE0D04B9C4200DC8FE0CF4B76
:107040009C4200DD55E1CE4A231592469A445146B2
:107050000905631A19001D00040003F055FA03F036
:1070600089FA02000B00200029000892099302F01F
:10707000E7FE0022C34B02F071FC0F00060003F094
:1070800043FA03F077FA04000D0002000B00300011
:1070900039000A940B9502F0D3FE0022B94B02F09E
:1070A0005DFC002200230C900D9101F05DFB002897
:1070B00000D192E1002300222000290001F054FBBE
:1070C000434243410133B04A41460192022208A89B
:1070D0000092524600F07CFB4B460500002B16DA6E
:1070E000802243461206944642465B68454263440A
:1070F0005360D3686344D36009E00B00020041464B
:107100000A604B600022002300258A60CB602800C3
:107110000FB03CBC90469946A246AB46F0BD934B9F
:1071200001F0F6FC914B06000F009C4200D13DE1BE
:107130008F4A904B01F0ECFC02000B0041463000FE
:107140000A604B60390002F07BFE894A894B01F0EE
:10715000DFFC012543466D429860D960D7E701F016
:1071600049F88A4A8A4B06000F0002F0F7FB00221A
:10717000884B01F0CDFC03F0C7F9050003F0FAF9E4
:10718000794A7A4B0490059102F0E8FB02000B006B
:107190003000390002F054FE754A06000F000498D2
:1071A0000599744B02F0DAFB029003911F2D00DC6D
:1071B000C7E0029A039B3000390002F041FE83468B
:1071C0008A4653465B0024155B0DE31A102B6CDDD9
:1071D00004980599D322674B520502F0BFFB0200C9
:1071E0000B00300039000292039302F029FE0A00DE
:1071F000010013000691079202003900300002F0EE
:107200001FFE029A039B02F01BFE06000F0004986B
:107210000599614A614B02F0A1FB32003B0002F08C
:107220000FFE069E079F0B000200390030000292FD
:10723000039302F005FE4B005B0D83468A46E41A79
:10724000312C32DD04980599B822544B920502F096
:1072500085FB03000C000200029303940B000698C8
:10726000079902F0EDFD02000B0006000F000698E2
:10727000079902F0E5FD029A039B02F0E1FD484AFE
:107280000290039104980599464B02F067FB029A1D
:10729000039B02F0D5FD02000B0030003900029282
:1072A000039302F0CDFD83468A465A465346414633
:1072B00030000A604B60390002F0C2FD029A039B65
:1072C00002F0BEFD44460B000200A260E3604B46A4
:1072D000002B00DB1BE75B46236080231B06534427
:1072E000636080231B069C466144A060E1606D42A0
:1072F0000DE70B00020002F0A3FD43460025986055
:10730000D9601860596002E7D3221A4B520502F087
:1073100097FD214A214B0D00040002F091FD02006F
:107320000B00414620000A604B60290002F088FDF6
:107330001A4B194A02F084FD434601259860D96032
:10734000E5E602000B003000390002F079FD6B1E0B
:10735000154A9B009B5883468A46A342A5D130E735
:10736000FB21E93F7BD9024000004054FB21F93F5B
:107370003163621A61B4D03DFB213941FFFFEF7FD9
:10738000EAFBFFFF00007041E0D9000083C8C96D2F
:10739000305FE43F0000E03F7370032E8A19A33B87
:1073A000C14920259A837B3960D90000D3220C4B38
:1073B000520501F0ADFB0B4A0B4B04000D0001F030
:1073C000A7FB02000B00414620000A604B60290029
:1073D00002F036FD034A044BB9E6032373E6C046C8
:1073E00061B4D03D7370032E8A19A33BF8B54746AC
:1073F000CE46674B80B50A000F00190005003940E2
:10740000994200D19BE004000100002F69DD3F1587
:1074100000D1B4E05F4B12039C468023120B5B0348
:1074200013435B00CA0F67449B184A00F80703D553
:10743000D20F5B009B188A0079108C4600218020B7
:107440001624894680030D189D4202DC29185B1B17
:107450008144D50F5B00013C5B1952004008002CB1
:10746000F1D100208046802020250027000609E079
:107470008B425CD0D40F5B00013DE3185200400802
:10748000002D16D0C4198B42F2DD27180E00002CF7
:1074900049DB5B1AA242894149425B1A121BD40F95
:1074A0005B00013D80443100E31852004008002D8C
:1074B000E8D113434ED143465B0837494A468846D4
:1074C000494652104244C90702D5802109060B43A0
:1074D00061460F05BD18180029000CBC904699465E
:1074E000F8BD7B005B0803433900002BF5D0002F6B
:1074F0003CD1E30A153A6405002BFAD08020400302
:1075000003423FD1002700E00F005B00791C0342DB
:10751000FAD0250020208D40401A2900D71B2200D8
:10752000C2401A4376E7FE43F60F8E19B1E7944244
:10753000A0D82718002CF6DB1E000023AEE70200BF
:107540003B002800390002F009FA2A003B0001F054
:10755000DFFAC2E74346013303D0434601335B08F9
:10756000ABE7012398460023C144A6E73B00020095
:1075700002F066FC02000B0001F0E6FDADE713002F
:107580000022BBE70127210020207F42C6E7C0463A
:107590000000F07F01FCFFFF0000E03FF0B5474630
:1075A000CE4680B587B000920193754B4F0081465F
:1075B00088467F089F4263DC02F0A6FF002800D1C6
:1075C000D4E04A4643464846414602F0C7F9040023
:1075D0000D006C4A6C4B02F0C1F96C4A6C4B01F027
:1075E00097FA22002B0002F0B9F96A4A6A4B02F0BE
:1075F00027FC22002B0002F0B1F9684A684B01F029
:1076000087FA22002B0002F0A9F9664A664B02F0C5
:1076100017FC22002B0002F0A1F9644A644B01F030
:1076200077FA22002B0002F099F9029003910022D0
:10763000604B2000290002F091F9029A039B06009A
:107640000F002000290002F089F9009A019B040034
:107650000D004846414602F081F902000B0020006F
:10766000290002F0EDFB02000B003000390002F0AF
:10767000E7FB02000B0000204F4902F0E1FB70E045
:1076800002000B0002F06AF904000D003D4A3E4B77
:1076900002F064F93D4A3E4B01F03AFA22002B0019
:1076A00002F05CF93B4A3C4B02F0CAFB22002B0083
:1076B00002F054F9394A3A4B01F02AFA22002B0021
:1076C00002F04CF9374A384B02F0BAFB22002B008B
:1076D00002F044F9354A364B01F01AFA2B00220029
:1076E00002F03CF9354B029003919F429FDD344BF1
:1076F00000229F423DDC334900207B182E491600B2
:107700001F0002F09DFB049005910022294B2000F0
:10771000290002F023F932003B0002F091FB029AAB
:10772000039B06000F002000290002F017F9009AC1
:10773000019B04000D004846414602F00FF902008B
:107740000B002000290002F07BFB02000B00300040
:10775000390002F075FB02000B000498059902F055
:107760006FFB07B00CBC90469946F0BD0020124953
:10777000F7E7154B002604920593144FC5E7C04662
:10778000FFFF3F3ED43888BEE9FAA8BDC4B1B4BDFE
:107790009EEE213EAD529C804F7E923E9015CB19BD
:1077A000A001FA3E7751C1166CC1563F4C55555554
:1077B0005555A53F0000E03F0000F03F3233D33F76
:1077C0000000E93F0000E0FF0000E73F0000D23F7B
:1077D000F0B5DE464E4645465746E0B5DC4CA5447E
:1077E0000D9114001900A49A0993DA4B9200D6580F
:1077F0004D1E03901821E01E0696029500F0AAFE89
:10780000C3430100DB1719404B1C9A009B1ADB0095
:107810001B190B9105934C1B771918D4A59BA50038
:107820009C463F1922AE6544013707E0286802F004
:10783000A1FE013403C60435BC4208D0002CF5DAA1
:1078400000200021013403C60435BC42F6D1069B5A
:10785000002B01DA00F0FDFB069B03990133DB00EE
:107860009A46099BDA00944600920022914672AA39
:107870000492B94A6144934688469AAB63449B4458
:10788000029B002B00DABCE15D4600260027039C2A
:107890004D442A686B6803CC02F060F802000B00CC
:1078A0003000390001F034F9083D06000F0044456E
:1078B000EFD1049B4B441E605F6008239C46E1446B
:1078C000D145DDD10EA804218446494261448C464D
:1078D000069A93009C44614684460A910399083BAA
:1078E00063448C460C93009B009263449B46009A31
:1078F0000498D10003008C46634408911E685F68B9
:10790000002A33DD954980468C466244D300984472
:1079100070AB9A460EAB99460022914B300039006D
:1079200002F01CF802F0F0FD02F024FE00228D4B64
:1079300004000D0002F012F802000B0030003900C4
:1079400002F07EFA02F0E0FD4B4601C39946434641
:1079500020001A685B68290001F0DAF808235B420E
:107960009C46E04406000F00D045D5D1059B300071
:107970001A003900984600F0DFFCFF2300229B0527
:1079800004000D0001F0EAFF00F038FC0022764B05
:1079900001F0E4FF02000B002000290002F050FA81
:1079A0000D00040002F0B0FD814602F0E3FD02008C
:1079B0000B002000290002F043FA060040460F00A9
:1079C000002800DCEEE0009B18215A1E92000EAB4E
:1079D0009B58091A1D000D41A9448D405D1B0EAB3B
:1079E0009D5017231B1A1D41002D2DDD01239C46A0
:1079F000009BE144002B00DC1CE20E9C0123002CC8
:107A000000D0B5E0009A012A09D099000EAA545876
:107A10000133002C00D0ACE0009A9A42F5D1059BCE
:107A2000002B0EDD012B00D1A8E1022B09D1009B18
:107A30000EA95A1E92000EAB9B5807939B029B0AFD
:107A40008B50022D00D1C1E000230022300039000C
:107A500000F08AFE009B002800D194E2069A591E8D
:107A60008A4210DC414A0A9894460EAA634494461E
:107A700000229B0063441C68043B22438342FAD1EA
:107A8000002A00D0C0E0069B0EAA013B9B00D35801
:107A9000002B00D0B3E001220C9B043B596801325B
:107AA0000029FAD0009B9C466244110007921A00FC
:107AB00001338B4246DC0B9863468046A59C4344C9
:107AC000A046099C9B00A1464A449844D30022AAA0
:107AD0009146049A99449446089BA59A6344844627
:107AE000614494469A468B00634400934346586829
:107AF00002F040FD4B4618605960029B002B24DBCE
:107B00004D46039C0026002701E0286869680CCCDC
:107B100001F024FF02000B003000390000F0F8FFF4
:107B2000083D06000F005C45EFD153469E60DF60C4
:107B300004239C460433E0449C46009BE144E24419
:107B40009845D3D1079B0093D1E600260027ECE7A8
:107B500094FDFFFF28DB000018FEFFFFFFFFFF1F63
:107B60000000703E0000704100002040FFFFFF3F1A
:107B7000002180225204141B0EAA545000999942ED
:107B80000EDD0EA884469B000EAA8900D2586144DF
:107B90006344CF4800E01A68821A04C38B42FAD1CA
:107BA00001243CE7059B002B06D1009B0EAA013B5C
:107BB0009B00D558ED1517E70022C64B300000F0AA
:107BC000F7FD002800D024E100253DE732003B000E
:107BD0000020C14902F034F906000F00002C00D14A
:107BE00032E7059A0020BC4900F0A6FB02000B001A
:107BF0003000390002F024F906000F0024E70122CA
:107C000050E70026002754E64B46059A079388461E
:107C10008B000EA9CB58183A08950592002B0DD170
:107C20008C464146AD4B43449B006344043B58683B
:107C30000139183A0028F9D088460592059A0020A3
:107C4000A54900F079FB434604000D00002B00DA43
:107C500005E29E000EAB9C464346DB0066449C4614
:107C6000059370AB9946049F67440097306802F013
:107C700081FC22002B0001F071FE00223860796047
:107C8000974B2000290001F069FE083F04000D0019
:107C9000043EB945EAD14AAB03939B4600239A467A
:107CA000069B4246994643460132029204934B4654
:107CB000002B00DAAAE080208A4B009D9846C00580
:107CC000894900260027002408E008239C4608353F
:107CD000E044544511DC4346186859682A686B68CB
:107CE00001F03CFE02000B003000390000F010FFF4
:107CF000013406000F00A145E7DA5B46C0C39B468E
:107D000001239C46009BE244083B0093029B9A455A
:107D1000CDD1049B9846A49B022B00DD8EE0002B66
:107D200037DC1FD1059B00271D00039B00249C46C8
:107D30001E006544083E2A686B683800210000F088
:107D4000E7FE083D07000C00AE42F4D1089B002B73
:107D500003D080231B069C4664443A0023000D99FF
:107D60000A604B600720079B18409B239B009D44A3
:107D70003CBC90469946A246AB46F0BD009B0EA97E
:107D80005A1E92000EAB9B5807935B025B0A8B5006
:107D900057E64346002B00DA70E100200021DB00AB
:107DA0004AAAD61848AF32687368083E00F0B0FEA1
:107DB000B742F8D1089B002B00D025E10B00020050
:107DC0004A984B990D9C2260636002F039F8434653
:107DD00007000C00002B13DD01254CAEB146380026
:107DE0002E0021004C4601360CCC00F091FEA1463D
:107DF000B045F7DA089B07000C00002B00D015E116
:107E00003A0023000D998A60CB60ABE7002600277B
:107E100073E701239C46009BE1440225002B00DD13
:107E2000EBE532003B0000202B4902F009F8060088
:107E30000F0009E60024F2E54AAB0393A49B032B51
:107E400000D08FE74346002B00DC14E1039ADB00EF
:107E50009B46130091465B441E685F68234B434476
:107E60000293DB00994448AB9A464B465C681B681A
:107E70001800210032003B000090019100F048FE04
:107E800004000D0002000B000098019901F0D8FFDA
:107E90003B00320000F03CFE4B469860D9601C600D
:107EA0005D6008235B429C46E14426002F00CA45E2
:107EB000DBD14346012B00DCE3E0039A13005B4473
:107EC0001E685F68029BDB0099464A44904610E0BA
:107ED000FFFFFF000000E03F0000F03FFFFFFF3F1B
:107EE0000000703EE8DA0000FB21F93FFFFFFF1FB2
:107EF000984643465C681B681800210032003B002E
:107F00000090019100F004FE04000D0002000B003F
:107F10000098019901F094FF32003B0000F0F8FD59
:107F20004346039A9860D9601C605D60083B260058
:107F30002F009A42DCD14D46944600260024474645
:107F4000083565442A686B683000210000F0E0FDC8
:107F5000083D06000C00AF42F4D1039B4A9F5D68C8
:107F60009968D868089B002B65D080221206944639
:107F70000D9B6544604464441F605D609960D860F7
:107F80001E615C61EEE69A464B460793059B300006
:107F90005A423900089500F0CFF900223A4B06000A
:107FA0000F0000F005FC002824D0384B00223000E0
:107FB000390001F0D3FC02F0A7FA52460400950004
:107FC00002F0D8FA0022304B01F0C8FC02000B008E
:107FD0003000390001F034FF02F096FA0EAA505139
:107FE0000122059B524418339046059393000EAA34
:107FF000D45023E65346300039009C0002F084FA46
:108000000EAB1851D04619E680230D9A1B06CB18EB
:10801000106053600B0002004A984B9901F010FF6A
:10802000434607000C00002B00DDD5E680231B062D
:108030009C466444E4E62B003A000D9D2A606B6088
:108040000A000300AA60EB60320023002A616B6122
:1080500088E6099BDB00009372AB049332E4A49B97
:10806000022B00DDE8E6002B00DD92E600D079E689
:10807000002700246AE6002600246EE70020002185
:1080800098E60026340068E7000070410000703E6A
:10809000F0B5CE46474680B587B000920193474A77
:1080A0004B00814688465B08934207DC41464846C0
:1080B00002F02AFA4146031E484666D04A46434625
:1080C0004846414601F04AFC04000D0002000B0046
:1080D0004846414601F042FC394A3A4B06000F003F
:1080E0002000290001F03AFC374A384B01F0A8FE85
:1080F00022002B0001F032FC354A364B00F008FD1F
:1081000022002B0001F02AFC334A344B01F098FE88
:1081100022002B0001F022FC314B324A00F0F8FC27
:108120000E9B02900391002B34D0009801990022FD
:108130002D4B01F013FC029A039B04900591300033
:10814000390001F00BFC02000B000498059901F0C6
:1081500077FE22002B0001F001FC009A019B01F048
:108160006FFE224A04000D00214B3000390001F05F
:10817000F5FB02000B002000290000F0C9FC020002
:108180000B004846414601F05BFE07B00CBC904630
:108190009946F0BD02000B002000290001F0DEFB33
:1081A000124A134B01F04CFE32003B0001F0D6FBAB
:1081B0004A46434600F0ACFCE7E7C046FFFF3F3EBF
:1081C0007CD5CF5A3AD9E53DEB9C2B8AE6E55A3E61
:1081D0007DFEB157E31DC73ED561C119A0012A3FFD
:1081E0001111813FA6F810110000E03F4955555587
:1081F0005555C53F49004B0819007047474AF0B52F
:108200004F4691464B005B0D99444646D6464A463A
:10821000C0B505000C000E0088460700132A27DCB5
:10822000002A4BDB3E4B13419A460B00524613404B
:10823000034318D03B4A3C4B2800210000F068FC67
:108240000022002300F0AAFA002847D0002C04DA0C
:1082500080234A465B031341984446465346002711
:108260009E43380031001CBC90469946A246F0BDA2
:10827000332A08DD8023DB009945F4D102000B008E
:1082800000F046FCEFE7294A94460122634452423B
:10829000DA4092460242E6D0224A234B28002100CF
:1082A00000F036FC0022002300F078FA002815D0F8
:1082B000002C1EDB534646469F430FE0194A1A4BDB
:1082C0002800210000F024FC0022002300F066FAC0
:1082D000002803D0002C04DB0027002638003100E2
:1082E000C1E76400640825430027002DF6D0104E36
:1082F000F4E74B46142B0BD03422D21A01239340BF
:108300005D19BD4208D201239C462F00E044D1E70D
:10831000133B9C46E044CDE72F00CBE701FCFFFF79
:10832000FFFF0F009C7500883CE4377EEDFBFFFFEC
:108330000000F0BF002070474B0070B55B0D1400CB
:108340000A00002B1AD14B005B08034315D0234BC6
:10835000002201F003FB224B9C422DDB0A004B0064
:108360005B0D363B1F4DE318AB422ADC002B0DDDC5
:108370001D4C1B0522401A43110070BD1B4DAB4222
:10838000F0D102000B0000F0C3FBF6E71D0035350D
:1083900019DA174B02009C4209DD0B0015481649FB
:1083A00000F032F8134A144B01F0D8FAE5E70B005D
:1083B0001248134900F028F8104A114B01F0CEFA88
:1083C000DBE70200E9E7084C363322401B05134384
:1083D000190000220B4B01F0C1FACEE70000504318
:1083E000B03CFFFFFE070000FFFF0F80FF0700000B
:1083F00050C300009C7500883CE4377E59F3F8C2F6
:108400001F6EA5010000903C30B54A00DB0FDB0772
:1084100052081A43110030BD02B4714649084900A0
:10842000095C49008E4402BC7047C04603B47146E3
:10843000490840004900095A49008E4403BC70476E
:10844000002243088B4274D303098B425FD3030A93
:108450008B4244D3030B8B4228D3030C8B420DD3A6
:10846000FF22090212BA030C8B4202D31212090234
:1084700065D0030B8B4219D300E0090AC30B8B4272
:1084800001D3CB03C01A5241830B8B4201D38B0320
:10849000C01A5241430B8B4201D34B03C01A5241C5
:1084A000030B8B4201D30B03C01A5241C30A8B4208
:1084B00001D3CB02C01A5241830A8B4201D38B02F3
:1084C000C01A5241430A8B4201D34B02C01A524197
:1084D000030A8B4201D30B02C01A5241CDD2C30909
:1084E0008B4201D3CB01C01A524183098B4201D385
:1084F0008B01C01A524143098B4201D34B01C01A70
:10850000524103098B4201D30B01C01A5241C308E7
:108510008B4201D3CB00C01A524183088B4201D356
:108520008B00C01A524143088B4201D34B00C01A42
:108530005241411A00D20146524110467047FFE7AE
:1085400001B5002000F0F0F802BDC0460029F7D0C8
:1085500076E7704703460B437FD4002243088B42E3
:1085600074D303098B425FD3030A8B4244D3030BBA
:108570008B4228D3030C8B420DD3FF22090212BA7F
:10858000030C8B4202D31212090265D0030B8B42FB
:1085900019D300E0090AC30B8B4201D3CB03C01AE5
:1085A0005241830B8B4201D38B03C01A5241430BC0
:1085B0008B4201D34B03C01A5241030B8B4201D3B0
:1085C0000B03C01A5241C30A8B4201D3CB02C01A1B
:1085D0005241830A8B4201D38B02C01A5241430A93
:1085E0008B4201D34B02C01A5241030A8B4201D382
:1085F0000B02C01A5241CDD2C3098B4201D3CB0129
:10860000C01A524183098B4201D38B01C01A5241D7
:1086100043098B4201D34B01C01A524103098B42DB
:1086200001D30B01C01A5241C3088B4201D3CB00C6
:10863000C01A524183088B4201D38B00C01A5241A9
:1086400043088B4201D34B00C01A5241411A00D259
:1086500001465241104670475DE0CA0F00D04942C2
:10866000031000D34042534000229C4603098B4232
:108670002DD3030A8B4212D3FC22890112BA030ABA
:108680008B420CD3890192118B4208D3890192113C
:108690008B4204D389013AD0921100E08909C309C1
:1086A0008B4201D3CB01C01A524183098B4201D3C3
:1086B0008B01C01A524143098B4201D34B01C01AAE
:1086C000524103098B4201D30B01C01A5241C30826
:1086D0008B4201D3CB00C01A524183088B4201D395
:1086E0008B00C01A5241D9D243088B4201D34B00B0
:1086F000C01A5241411A00D20146634652415B10F2
:10870000104601D34042002B00D5494270476346D2
:108710005B1000D3404201B5002000F005F802BD17
:108720000029F8D016E770477047C046D0400B1CB0
:108730001141203A03D49C461341184363465242E8
:10874000934018437047C0468446101C62468C46CE
:10875000191C634600E0C0461FB501F097F80028D9
:1087600001D40021C8421FBD10B500F0EFFF404208
:10877000013010BD10B501F089F8002801DB0020A0
:1087800010BD012010BDC04610B501F07FF80028D3
:1087900001DD002010BD012010BDC04610B501F064
:1087A00011F8002801DC002010BD012010BDC046DA
:1087B00010B501F007F8002801DA002010BD0120F3
:1087C00010BDC046F0B5CE46474615042D0C2E0010
:1087D00080B50704140C3F0C9946030C7E435D439F
:1087E000674363437F19340CE4199C46A54203D9BF
:1087F00080235B029846C4444B4643435143250CB7
:1088000036046544360C2404A4195B195918200059
:108810000CBC90469946F0BDF0B54E4657464546CD
:10882000DE46E0B543025B0A450083B00F1C994663
:108830002D0EC60F002D57D0FF2D24D08020DB0039
:10884000C0041843002381469A469B467F3D7C0224
:108850007A00FB0F640A120E984623D0FF2A4BD0F1
:10886000E30080240020E4047F3A1C43AD186B1C15
:1088700047460193534677403A000F2B48D87D492D
:108880009B00CB589F46002B00D085E008339A46CA
:10889000063B9B467C027A00FB0FFF25640A120E02
:1088A0009846DBD1002C00D090E0524601231A43B9
:1088B00092460120DBE74C4658461700022824D098
:1088C000032800D1CFE00022002301284DD1580217
:1088D000D205400AFF071043384303B03CBC904622
:1088E0009946A246AB46F0BD002B5BD104239A46C5
:1088F000033B00259B46AAE7FF35002C60D152467A
:1089000002231A4392460220B1E7FF220023DEE74A
:108910004B461B0C9C464B462604360C18046146FD
:108920003300220C6446000C43434E4350435443EF
:1089300080191A0C1218964203D9802149028C46DC
:1089400064441B041B0C1004C01883015E1EB34159
:10895000800E1843130C1B199B0103431C002301B9
:1089600079D5012362081C401443019A7F32002A02
:108970004DDD630704D00F232340042B00D00434C3
:10898000230103D53C4B019A1C408032FE2ABCDCFB
:10899000A3015B0AD2B29AE70C239A46093BFF2552
:1089A0009B4654E7180001F071FE4A46431F7625A6
:1089B0009A4000236D4291462D1A9A469B4646E7FF
:1089C000524603231A439246032050E7200001F049
:1089D0005DFE431F2D1A9C40763D002047E7802313
:1089E0000027DB03FF2272E7424666E74C4632006F
:1089F000584662E780234A46DB031A4222D01C42D3
:108A000020D123435B025B0A4746FF225FE7012335
:108A10009A1A1B2A21DC23000199D3409E318C40F5
:108A20001A0023005C1EA34113435A0704D00F22EF
:108A30001A40042A00D004335A0111D49B015B0A66
:108A4000002244E780234A46DB0313435B025B0AB0
:108A50003700FF223BE7019587E70022002336E736
:108A60000122002333E78023DB0323435B025B0AFD
:108A7000FF222CE738DB0000FFFFFFF770B500286E
:108A80003DD0C317C5185D40C40F280001F0FEFD9E
:108A90009E22121A962A07DCD2B2082833DD083843
:108AA00085406802400A23E0992A0BDD052329004E
:108AB0001B1AD94003001B339D402B005D1EAB41A8
:108AC00019430D00052801DD431F9D402B000F4970
:108AD0000B406E0709D00F263540042D05D0043316
:108AE0005D0102D59F220B40121A9B01580AD2B297
:108AF0004002D205400AE4071043204370BD002421
:108B000000220020F4E76802400AF1E7FFFFFFFBC4
:108B1000F0B54F464646D6460C000903C0B5490A93
:108B2000470F5E0039431F03DB0F9C4665007B0A3D
:108B3000570F1F436D0DE40F760DA146C000B846D8
:108B4000D200AB1B64457BD0002B5FDD002E00D034
:108B5000A4E03E00164300D112E15E1E002E00D0BC
:108B60009EE1871A4346B84280410125C91A404216
:108B7000091A0B0200D431E149024E0A002E00D13D
:108B80006EE1300001F082FD0300083B1F2B00DD89
:108B900061E120223900D21A9E40D1409F400E430D
:108BA0009D4200DD51E15D1B6B1C1F2B00DD7CE154
:108BB0002021C91A3D0030008F408840DD40791ED9
:108BC0008F41310007222843D940002507433A400E
:108BD000002A09D00F233B40042B05D03B1DBB428C
:108BE000BF417F42C9191F000B0200D426E26A1C54
:108BF000C64B55056D0D9A4200D106E1C44AFF08E7
:108C00000A40530752023B43120B8EE0002B00D068
:108C1000B8E06B1C5B055B0D012B00DC30E1871AB3
:108C20004346B842B641CB1A76429E1B330200D56A
:108C30004CE13B003343A1D100220024002570E029
:108C4000002B00DCE5E0002E00D183E0AF4EB54202
:108C500060D0802636043743B846382B00DC3EE12E
:108C6000434613431F007A1E97413F1887428041B5
:108C7000404209180B0200D4B0E0A44B01359D42DC
:108C800000D1C3E0A24A7B080A4001210F401F43E4
:108C90005108D30707221F433A4099E79B4EB5423C
:108CA00038D0802636043743B846382B00DDDCE068
:108CB0001F2B00DC30E11E004746203EF740BC463B
:108CC000202B04D04026F31A46469E40324317001C
:108CD00063467A1E97411F43CCE0002B00D104E28B
:108CE0004346134300D159E14B07C0081843802382
:108CF000C9081B03194208D04546ED081D4204D19E
:108D00004346D008590708432900420FC9007F4D48
:108D10001143C0004B07CA087C49C00803438D4279
:108D200068D012036D05120B6D0D0021120318009F
:108D3000130B0A0D12051A43764B2D0513402B43D6
:108D40005B00E4075B08234319001CBC904699466E
:108D5000A246F0BD3E00164312D05E1E002E00D08B
:108D600000E18718874280414144404209180125AB
:108D70000B0233D5022585E76446330041461000D7
:108D80001D00C7E7002D00D0DAE00C000443F3D04B
:108D90005C1C00D19FE15D4CA64200D12FE1DB437A
:108DA000382B00DD66E11F2B00DD83E12024050068
:108DB000E41A0F00DD40D940A0404346A7405B1AAB
:108DC000441EA04198462F433843171ABA42924195
:108DD00043465242991A64463500CAE607223A4091
:108DE000002A00D0F6E64B07CA084849FF083B4373
:108DF0008D4296D11900114300D19EE180210903D3
:108E00000A431203120B414D8FE715000022002385
:108E10008BE7002B00D0C7E06B1C5F057F0D012F97
:108E200000DCF1E0394DAB4200D1B9E085180A0011
:108E3000854289414244494251180722CF076D08B3
:108E40002F4349083A401D00C2E607223049ED1A77
:108E500031403A40BCE63E002838864000279FE675
:108E6000380001F013FC20308EE6434613431F0008
:108E70007A1E9741C71BB84280414042091A78E6E2
:108E80000E003B0006431343002D61D1002E00D09D
:108E9000F4E0002B00D11BE164463900100039E7F3
:108EA0001A4FBB427AD03300FFE630001F3DE84046
:108EB000202B03D04021CB1A9E4037437B1E9F417D
:108EC000072207433A400021002589E7171A434645
:108ED000BA42B641591A76428E1B64464EE61F2BA3
:108EE00000DDADE020264746F61AB740B946170028
:108EF000B246DF404E463E4337005646B240561E0D
:108F0000B24117434246DA408918AEE6FF07000037
:108F1000FFFF7FFFFFFF0F8020264746F61AB7406E
:108F2000B9461700B246DF404E463E43370056462C
:108F3000B240561EB24117434246DA40891A99E7B9
:108F40007F4CA6425BD0802424045B42214327E768
:108F5000002E0CD1002B00D1CBE06446390010006C
:108F6000774DD7E6764FBB4218D0330075E6002B1D
:108F700014D04B07C00818438023C9081B031942AB
:108F800007D0FC081C4204D17907D0080843E14609
:108F900021004C46420FC9001143C000684DB9E69C
:108FA0001D0000220023C0E6002D5BD10D0005430B
:108FB00000D1E2E65D1C00D1B0E0614DAE421FD0B1
:108FC000DB43382B71DC1F2B00DD96E020250F00E2
:108FD000ED1AAF40B9460700AA46DF404D463D4373
:108FE0002F005546A840D940451EA8418844074354
:108FF000BF18974292415142414435003AE66446D7
:1090000035004146100085E60B000343002D00D0DB
:1090100063E6002BF5D04346134300D17AE6871868
:109020008742804107224144404209183A400B02DE
:1090300000D4D5E6434B01351940C9E5380069E64F
:109040001E004746203EF740BC46202B04D0402659
:10905000F31A46469E403243170063467A1E9741F4
:109060001F4302E6364DAE42CAD080252D045B4236
:109070002943A6E70843411E8841A6E6002B00D1FC
:1090800048E6871A4346B842B641CB1A76429E1B41
:1090900033024BD5171A4346BA429241591A5242EB
:1090A000891A072264463A4092E501430F00791E6F
:1090B0008F419DE71C000F00203CE740202B03D090
:1090C0004024E31A99400843411E884138437CE616
:1090D0000022002425E6171A4346BA429241591A43
:1090E0005242891A6446350043E541461000144D4A
:1090F00010E680220024120380E61D000F00203DB0
:10910000EF40BC46202B03D04025EB1A9940084382
:1091100007006346781E87411F4369E78718974217
:109120009B4141445B42C9183500A3E53B003343F2
:10913000CED0072231003A4052E600231A00F4E56F
:10914000FF070000FFFF7FFFF0B55746DE464E46A3
:109150004546E0B5834607000E03480085B09246B9
:109160001C00360B400DCD0F002800D19DE0954B23
:10917000984239D08023F6001B041E43924A7B0F8D
:10918000334399469446030063440093002300262A
:10919000FF00029323031B0B98466300E40F524623
:1091A0005B0D019400D1B3E086498B4200D19EE073
:1091B0004246D100802212040A435146490F11430E
:1091C0008B46814952468C4600996344CB1A002154
:1091D000D20000932B0063409A460F2E00D905E180
:1091E0007A4BB6009B599F465B463343994600D065
:1091F000B8E002230826002700900293CAE7CB4676
:109200003A0002990195019B9A46022927D0032929
:1092100000D180E2012944D06D49009B8C46634413
:109220001C00002C38DD530700D013E2D2085B4647
:10923000DB0109D55946674B19408B468021C9008F
:109240008C46009B63441C00634B9C4207DC5B46DE
:1092500064055F075B0217431B0B620D02E00023EE
:109260000027584A00211B031C0B0B0D1B05234331
:1092700014055A4A380013401C4353466400DB0768
:1092800064081C43210005B03CBC90469946A246A8
:10929000AB46F0BD0122524201231B1B382B00DCE0
:1092A000ADE1002200230027DCE75B46334399460B
:1092B0005ED0002E00D18AE1300001F0E7F9030012
:1092C0000B3B1C2B00DD7BE11D22D31A5A4601000B
:1092D000DA4008398E4013005F46334399468F4089
:1092E0003F4B00261B1A00930023029352E741468E
:1092F00053460B433B499B468C46009B634400937B
:109300005B46002B3BD1022300221E43022161E772
:10931000434613439B4637D04346002B00D162E1BE
:10932000404601F0B3F903000B3B1C2B00DD53E179
:1093300002004146083A914088461D21CB1A514609
:10934000D9400B0041460B439B46534693401A00BD
:10935000009B25499C46604403008C46634400936F
:10936000002137E70323B14600900C26029311E752
:109370000023009301330426002702930AE7032306
:10938000C3461E43032125E701331E43002201216A
:1093900020E700239A46802300271B03094A61E740
:1093A000802349461B03194200D1E2E05946194285
:1093B00000D0DEE00B431B0317001B0BA246014A43
:1093C00050E7C046FF07000001FCFFFF78DB00000C
:1093D000FF030000FFFFFFFEFE070000FFFF0F80FE
:1093E0000DFCFFFF01F8FFFFF3030000D94500D992
:1093F000CBE000D1C6E03C0048460027009B013B83
:1094000000935B46160E1B021E431302984633045C
:109410001B0C9946310C0191FFF798F84A464243DC
:109420000B04210C050019438A4207D98919013D13
:109430008E4203D88A4201D9851E8919881A01995A
:10944000FFF784F809048C464A46210464464243E7
:10945000090C030021438A4204D98919013B8E4239
:1094600000D8F1E02D041D43AB464346891A42461D
:10947000280C12041D0C5B46140C22001B041B0C50
:109480005A4303946B434443029568431B19150CDC
:10949000EB189C4203D980246402A44660441C0C4F
:1094A00015041B042D0C20185D19814277D373D04D
:1094B0000C1AA24A7D1BAF42BF419446009B7F42DB
:1094C0006344E01B1C00864200D1DBE00199FFF7FA
:1094D0003DF84A4642430B04290C070019438A42CF
:1094E00007D98919013F8E4203D88A4201D9871EC4
:1094F0008919881A0199FFF729F809044A4689460B
:1095000029044D464243090C030029438A4207D9E6
:109510008919013B8E4203D88A4201D9831E8919D9
:109520003F04891A3A00039F1A43380013041B0CA6
:10953000584381460298150C6F43434345434846C0
:10954000000C8446DB1963449F4203D9802040020B
:109550008446654448461F0C00041B04000C7D191A
:109560001818A94200D284E000D17FE001231A43F9
:1095700057E680234A461B0313431B031B0BAA46D3
:109580006F4A6FE6BA4200D935E74B46DC07580808
:109590007B081C43FF0734E70024AF4289D24744CD
:1095A0004745A4415B466442A4196418013BA642A6
:1095B0001ED2A0426DD800D1B6E0241A9B4678E7AF
:1095C00003005A46283B9A400027914688E65846B1
:1095D00001F05CF8203072E603005246283B9A40C6
:1095E00093460022B4E6504601F050F820309AE647
:1095F000A642E2D1B845DCD9341A9B4659E71F2B65
:1096000065DC504C0099A4465C46614408008C40DF
:1096100011008240D940501E82410C4314435A46E7
:10962000DA401300620709D00F222240042A05D035
:109630002200141D9442894149425B181A0262D5E6
:109640000122002300270DE68A4200D80AE7831E84
:10965000891907E70F231340042B00D1E6E5171DF6
:109660009742924153429B44FA08E0E5002800D11A
:10967000D7E57118531EB14227D3A94215D358D04C
:109680001A0073E7002B00DC04E6012300229B4450
:10969000CDE502234744474589415B429C46494208
:1096A00089190C19E344241A03E743465F00474530
:1096B0009B41B8465B429E19023A8919A94200D0E3
:1096C00054E7404500D051E7ABE51A00F6E71F210B
:1096D0005F4649420C1BE740202B07D01A49009BEC
:1096E0008C46634418005B4683401A43501E8241F7
:1096F0003A4307270023174009D00F2100231140C8
:109700001400042995D122005F075B021B0BD208CD
:1097100017430022A6E5802359461B030B431B0376
:1097200017001B0B064A9DE5BD42B2D89B4600249C
:10973000BFE68045B9D31A00C3E7C046FF03000067
:10974000FF0700001E0400003E040000F0B54F4675
:109750004646D6468446C0B58046194E18030F03C8
:109760004D00000B5C0082463F0B6D0DC90F91460A
:10977000640DDB0F0120B5420AD0B44203D0A542EC
:1097800001D157450CD01CBC90469946A246F0BD6D
:1097900066463E43F7D1AC42F5D154461443F2D16C
:1097A0000120C845EFD1994207D0002DEBD1634687
:1097B0001F433800471EB841E5E70020E3E7C046F5
:1097C000FF070000F0B54F464646D6464D00C0B5EF
:1097D0000E03C90F8A462C491F035C008046360BD6
:1097E0006D0D91463F0B640DDB0F8D421ED08C42F8
:1097F00016D0002D1ED130438446002C01D13A43AF
:1098000023D06246002A1AD09A4529D05146022018
:109810000139084001381CBC90469946A246F0BD6B
:1098200039001143E5D002204042F4E73043FAD139
:10983000AC420FD0002C0FD13A43E7D00CE001220C
:10984000013B934318000130E5E763460020002BFD
:10985000E1D0DBE73A43E6D19A45D7D1A542D5DC42
:10986000A54205DBBE42D1D808D00020BE42D2D2EC
:1098700050460123013898430130CCE7C845C5D88C
:109880000020C845F4D3C6E7FF070000F0B54F46F7
:109890004646D6464D00C0B50E03C90F8A462E492E
:1098A0001F035C008046360B6D0D91463F0B640D27
:1098B000DB0F8D4218D08C4211D0002D18D13043CF
:1098C0008446002C1ED13A431CD163460020002B55
:1098D00030D0514602200139084001382AE03900D1
:1098E0001143EAD0022025E03043FBD1AC4226D020
:1098F000002C26D13A4324D1514602200139084098
:10990000013817E06246002A0FD09A45E1D1A542FE
:1099100005DBBE42DDD819D00020BE420AD2504637
:10992000012301389843013004E00122013B9343B5
:10993000180001301CBC90469946A246F0BD3A433F
:10994000D0D19A45C5D1A542C3DCE0E7C845C0D80F
:109950000020C845E3D3EDE7FF070000F0B5574608
:10996000DE464E464546E0B5834606000F034800F6
:1099700087B092461D003F0B400DCC0F002800D150
:109980006FE0DE4B984238D08023FF001B041F435A
:10999000730F3B430193DA4B0027994600239B4604
:1099A000F60081442B0369001B0B52469846490D73
:1099B000ED0F002900D185E0D04B994200D173E032
:1099C0004346DA0080231B0413435246CC48520F0F
:1099D00084461343524600206144D200894421004A
:1099E000694000918C46012149448A460F2F00D9D5
:1099F00090E0C449BF00CF59BF465B463B4301934B
:109A000000D06AE102230827002681469B46C9E769
:109A100032005846019B61460091022800D175E052
:109A2000032800D1FEE1012800D02CE1002300270B
:109A3000002600253F032A0D3F0BB34812053A4389
:109A400002401B051343009A5B00D1075B080B43E0
:109A50003000190007B03CBC90469946A246AB4680
:109A6000F0BD5B463B43019300D12FE1002F00D1B5
:109A7000A5E1380000F00AFE03000B3B1C2B00DDC3
:109A800096E11D22D31A5A460100DA405E46083993
:109A90008F4013008E403B4301939C4B00271B1AC1
:109AA000994600239B467DE7414653460B43934925
:109AB0008C46E144002B00D01AE102220220174319
:109AC00000228CE7134300D10DE14346002B00D167
:109AD00081E1404600F0DAFD02000B3A1C2A00DD6D
:109AE00072E10100434608398B4098461D239A1ABB
:109AF0005346D3401A004346134352468A404946D0
:109B0000081A824989468144002068E77B4B002778
:109B100000268EE7140C1204120C1100370C3604C8
:109B2000350C794328008C462E0060436044834600
:109B300056432100300C80465846794340440291F8
:109B4000844506D98846802149028C46E044414636
:109B500002913604010C360C00048B4681191E0C50
:109B60001B041B0C0391190079438C462800754394
:109B70006544A8465843050C45447743A94203D998
:109B8000802149028C466744290C8C463900000428
:109B9000000C2D042D186144AB44059159460491E5
:109BA00001990F043F0C080C390051434243904681
:109BB00002008C46090C8B4662437C4344445C445F
:109BC000A04503D98021490288464244210C884699
:109BD00061460904090C8C463900594343437043DC
:109BE0007E430F0CF6182404BE19644442448C468C
:109BF000B34203D980235B0298464044029B6146EE
:109C00009846049B370443449B46AB45AD416B42A9
:109C10000D0405992D0C8C467F196744FD18A84644
:109C20005D462D19A542A44193466442A446C3440F
:109C3000DC448F42BF4198459B4193459241A445E6
:109C4000A4415B427F421F43360C52426442BF191B
:109C50002243BF18624638184302D20D03991343BA
:109C60006A020A43501E82416146ED0D2A434E02AC
:109C70003243D90100D4B3E00126500832400243F8
:109C8000DE0732435B08224C5444002C62DD51074E
:109C900009D00F201040042805D0101D9042924199
:109CA00052429B180200D90104D580241948E400CF
:109CB000034054441848844200DD27E75E075B02F6
:109CC000D2081F0B630516435B0DB2E600239946CD
:109CD0000133042700269B4664E60323019781464F
:109CE0000C279B465EE6012201201743002276E600
:109CF000032303201F43434671E6C046FF070000CD
:109D000001FCFFFFB8DB0000FFFF0F800DFCFFFF31
:109D1000FF030000FFFFFFFEFE0700000023802777
:109D200000933F030026434B83E6019B3200A44689
:109D3000584670E6AC466EE6802701993F033942EB
:109D40002DD03B422BD11F433F033F0B0095160004
:109D5000384B6EE601252D1B382D00DD66E61F2DE4
:109D600040DC35481C005044160082408440EE40E0
:109D7000501E824134431443EB40620709D00F2246
:109D80002240042A05D02200141D94428041404202
:109D90001B181A023ED501230027002649E680271A
:109DA000019B3F031F433F033F0B0094214B40E6C1
:109DB00003005A46283B9A40002601926DE6584619
:109DC00000F064FC203057E603005246283B9A40DE
:109DD0001300002293E6504600F058FC20307BE64A
:109DE000CA4650E71F201E004042041BE640202DBB
:109DF00003D0124C5444A3401A43501E82413243B4
:109E000007260027164009D00F2000231040140019
:109E10000428B9D122005E075B021F0BD20816434B
:109E2000002306E680273F031F433F033F0B160036
:109E3000004BFEE5FF0700001E0400003E0400008A
:109E4000F8B557464E464546DE460C000903E0B5D8
:109E5000490A460F5F0031431E03DB0F760A9B461B
:109E6000530F3343C84E6500C000E40FD2006D0DA0
:109E7000A24681467F0D9C469046B74200D1B9E08C
:109E80005B46012673409B46EE1BA34500D183E051
:109E9000002E63DD002F00D0B1E06346134300D1F4
:109EA00023E1731E002B00D0BAE1861A6346B0424C
:109EB00080410125C91A4042091A0B0200D447E12A
:109EC00049024B0A98464346002B00D189E140469F
:109ED00000F0DCFB0300083B1F2B00DD7CE12022AF
:109EE0003000D21A4146D040994002009E400A43B9
:109EF0009D4200DD6AE15D1B6B1C1F2B00DD94E1C0
:109F0000202110003500C91A8E40DA408840DD401B
:109F1000711E8E411100072228430025064332405E
:109F2000002A09D00F233340042B05D0331DB34240
:109F3000B641764289191E000B0200D43DE26A1C2C
:109F4000914B55056D0D9A4200D119E18F4AF608E3
:109F50000A40570752023743120B9BE0002E00D0F5
:109F6000C5E06E1C7605760D012E00DC48E16746E3
:109F7000861ACB1BB042BF417F42B8461F00434602
:109F8000FF1A3B00B8461B0200D55FE137439AD168
:109F900000220024002579E0002E00DCFAE0002FEA
:109FA00000D18DE0784B9D4267D0802367461B042B
:109FB0001F43BC46382E00DC52E1634613435A1E51
:109FC00093411E1886428041404209180B0200D47A
:109FD000BEE06D4B01359D4200D1D2E06B4A730863
:109FE0000A4001210E401E435108D30707221E4399
:109FF000324095E71E00164300D045E740E7624B2C
:10A000009D423AD0802367461B041F43BC46382E2E
:10A0100000DDEBE01F2E00DC3AE133006746203B19
:10A02000DF403B00202E05D04027BF1B6646BE40C8
:10A03000324390464646721E96413343DAE0002B87
:10A0400000D114E26346134300D168E180234E0738
:10A05000C008C9081B030643194208D06046C0085F
:10A06000184204D163460100D2085E071643F3008C
:10A070009946C900720F444D11434B46DE08424BCE
:10A080004F073743CA089D4200D16EE012036D05A9
:10A09000120B6D0D00211203130B0A0D12051A434A
:10A0A0003B4B2D0513402B435B00E4075B08234328
:10A0B000380019003CBC90469946A246AB46F8BD14
:10A0C0006346134311D0731E002B00D007E186189E
:10A0D0008642804161444042091801250B0237D570
:10A0E00002257BE73E00614691463500C5E75C46A8
:10A0F000002D00D0E1E00B000343F3D0731C00D12E
:10A10000ACE1214B9F4200D13AE1F343382B00DD13
:10A110006FE11F2B00DD8CE120250E00ED1AAE4013
:10A12000B0460600AA46DE40454635432E00554659
:10A13000D940A8406346451EA8415B1A9C4630435F
:10A14000161AB242924163465242991A3D00B4E651
:10A1500007223240002A00D0E4E60B4BF6084F07F6
:10A160003743CA089D4200D090E73B00134300D11B
:10A17000A6E180231B031A431203120B024D89E749
:10A1800015000022002785E7FF070000FFFF7FFF83
:10A19000FFFF0F80002E00D0C7E06B1C5E05760D20
:10A1A000012E00DCF0E0C84DAB4200D1B9E08518CB
:10A1B0000A00854289416244494251180722CE076C
:10A1C0006D082E43490832401D00A9E6BF49ED1A2B
:10A1D000114007223240A3E6320028388240002690
:10A1E00086E6300000F052FA203073E663461343EF
:10A1F0005A1E9341C61AB04280414042091A5CE699
:10A200000E00674606431743002D5ED1002E00D096
:10A21000F3E0002F00D11EE15C46614691462CE739
:10A22000A94FBE427BD01E00F1E610001F3DE84062
:10A23000202B03D04021CB1A9A401643731E9E4117
:10A240000722064332400021002583E7161A6346A1
:10A25000B2428041591A40420B1A98465C4632E697
:10A260001F2E00DDABE02027BB1B9A4663465746F6
:10A27000BB40994613004F46F3401F433B005746EF
:10A28000BA40571EBA4113436246F240891898E615
:10A290002027BB1B9A4663465746BB40994613008E
:10A2A0004F46F3401F433B005746BA40571EBA4142
:10A2B00013436246F240891A9CE7834B9F425FD06A
:10A2C00080252D047342294320E7002E0CD1002F56
:10A2D00000D1D0E05C46614691467B4DCDE67A4F99
:10A2E000BE421CD01E0065E6002F18D0C0084E07E5
:10A2F00006438020C9080003014208D06346DC08F9
:10A30000044204D12100DA46D2085E071643F30066
:10A31000994601245346C900720F11431C406A4DEF
:10A32000ABE61D0000220027B4E6002D59D10B003A
:10A33000034300D1D6E6731C00D1B2E0624B9F42CA
:10A340001ED0F343382B6FDC1F2B00DD97E0202558
:10A350000E00ED1AAE40B0460600AA46DE40454665
:10A3600035432E005546A840D940451EA8418C448F
:10A370000643B61896429241514261443D0025E69B
:10A380003D006146914678E60B000343002D00D066
:10A3900055E6002BF5D06346134300D16DE68618D1
:10A3A0008642804161444042091800220B0200D4D9
:10A3B000D0E6464B01351940B2E5B1465DE63300C3
:10A3C0006746203BDF403B00202E05D04027BF1BC7
:10A3D0006646BE40324390464646721E964133431F
:10A3E000EFE5394B9F42CBD080252D0473422943A2
:10A3F000A8E70843411E8841A2E6002F00D13CE6B1
:10A400006346861ACF1AB0429B415B42FB1A9846BC
:10A410001B024ED5161A6346B2429241591A524255
:10A42000891A5C4600227BE501430E00711E8E41B5
:10A430009FE71D000E00203DEE40B046202B04D0CB
:10A440004025EB1A99400843814648464346411E41
:10A450008841184374E60022002417E6161A634662
:10A46000B2429241591A5242891A3D0025E561468D
:10A470009146154D01E680220024120379E61D0065
:10A480000E00203DEE40B046202B04D04025EB1AB4
:10A490009940084381464E464346711E8E411E43F5
:10A4A00067E7861896429B4161445B42C9183D00AC
:10A4B0008CE547463743CED007224146324049E635
:10A4C00000273A00E6E5C046FF070000FFFF7FFFD8
:10A4D00070B50C4E0D031C0349005B002D0B490D9C
:10A4E000240B5B0DB14208D0064900208B4203D1FA
:10A4F00014432000441EA04170BD05430120002DDF
:10A50000FAD1F1E7FF07000030B5144D0A034B0004
:10A51000120B5B0DC90F0024AB4211DD104CA3429E
:10A5200010DC8024640322430E4CE41A1F2C0CDD43
:10A530000D48C31ADA4013005C42002900D11C0008
:10A54000200030BD094BCC18FAE7094DE040AC467D
:10A5500063449A4013000343EEE7C046FE03000045
:10A560001D0400003304000013040000FFFFFF7F00
:10A57000EDFBFFFF70B500282DD0C317C5185D4057
:10A58000C40F280000F082F8154B1B1A5B055B0D09
:10A590000A2815DD0B38854000222D032D0B0021E4
:10A5A00010002D030A0D2D0B12052A430D4D1B051E
:10A5B0002A4013435B00E4075B082343190070BD86
:10A5C00002002900153291400A000B21081AC540EB
:10A5D0002D032D0BE3E70024002300250022DEE7F6
:10A5E0001E040000FFFF0F804100090E4B1C70B5D8
:10A5F000DBB24602750AC40F012B14DDE0239B0079
:10A600006D07360BCB1800210A0D280012051C4DD2
:10A6100032435B052A405B0813435B00E4075B0899
:10A620002343190070BD002914D1002D1ED028002D
:10A6300000F02CF80A281CDC0B232A001B1ADA4035
:10A64000030015339D400F4B12031B1A5B05160BBD
:10A650005B0DD8E7002D06D0320B802636036D0740
:10A660001643094BCFE7084B0026CCE70023002612
:10A67000C9E703002A000B3B9A400025E3E7C046E8
:10A68000FFFF0F8089030000FF0700001C2101234A
:10A690001B04984201D3000C10391B0A984201D3C5
:10A6A000000A08391B09984201D30009043902A2A3
:10A6B000105C40187047C04604030202010101010A
:10A6C000000000000000000030B51C00094B050030
:10A6D0001B6885B0D868084B002A01D1074B1A00C7
:10A6E0000292019300912B002200054900F026F808
:10A6F00000F020FE7C000020F8DB0000A2CA000071
:10A7000005DC0000014B18687047C0467C00002043
:10A71000084B10B50400002B02D0002100E000BF60
:10A72000054B1868836A002B00D09847200001F081
:10A73000C9FFC0460000000034DC00000EB403B5C1
:10A74000010003AB044804CB0068019300F076F8E5
:10A7500002B008BC03B018477C00002070B500268A
:10A760000C4D0D4C641BA410A64209D1002601F02B
:10A77000ABFF0A4D0A4C641BA410A64205D170BD64
:10A78000B300EB5898470136EEE7B300EB58984713
:10A790000136F2E74C0200204C0200204C0200205F
:10A7A0005C020020002310B59A4200D110BDCC5CA1
:10A7B000C4540133F8E710B5884202D98B18984287
:10A7C00003D3002307E08B5C8354013AFBD210BD16
:10A7D000CC5CC45401339A42FAD1F8E70300121852
:10A7E000934200D1704719700133F9E7936810B5AF
:10A7F000013B9360002B04DA9469A34207DB0A292A
:10A8000005D01368581C10601970080010BD00F0C6
:10A81000B1FC0100F9E7F8B506000F001400D518E7
:10A82000AC4201D1002007E021783A003000FFF768
:10A83000DDFF0134431CF3D1F8BD0000F0B59FB03B
:10A8400002900F0016000593002805D08369049339
:10A85000002B01D100F080FE7B4B9F425BD1029B1D
:10A860005F68BB891B0762D53B69002B5FD0002363
:10A8700006AC6361203363761033A37635002B7802
:10A88000002B01D0252B5CD1AB1B04930CD03200E4
:10A8900039000298FFF7BFFF431C00D1C4E0626992
:10A8A000049B9446634463612B78002B00D1BBE08A
:10A8B000012200235242626002A9543252186E1CD7
:10A8C0002360E360A3601370A365317805225F48BD
:10A8D00000F082FF751C002835D12268D30604D50C
:10A8E000532302A95B1820211970130704D55323A1
:10A8F00002A95B182B21197033782A2B2CD0350034
:10A9000000210A20E3682A786E1C303A092A64D9AB
:10A9100000292ED026E04E4B9F4202D1029B9F6819
:10A920009FE74C4B9F429CD1029BDF6899E739001F
:10A93000029800F089FC002899D0012040421FB005
:10A94000F0BD01359BE7414B2268C01A01238340CB
:10A95000134323602E00B8E7059B191D1B68059162
:10A96000002B01DB099304E05B42E3600223134305
:10A9700023602B782E2B0AD16B782A2B35D1059B9F
:10A9800002351A1D1B680592002B2BDB0793324EF4
:10A9900029780322300000F01FFF002806D0402352
:10A9A000801B8340226801351343236029780622E7
:10A9B0002A486E1C217600F00FFF00283AD0284B61
:10A9C000002B25D10722059B0733934308330593BA
:10A9D0006369039A9B18636150E7434301219B1805
:10A9E000350090E701235B42D0E700230A201A00DC
:10A9F0000135636029786E1C3039092903D9002B91
:10AA0000C5D00792C3E74243012352183500F1E74E
:10AA100005AB00933A00134B2100029800E000BF01
:10AA20000390039B0133D3D1BB895B0600D584E738
:10AA30000B9884E705AB00933A000A4B210002987B
:10AA400000F080F8ECE7C0468CDC000038DC000049
:10AA5000ACDC00006CDC00003EDC000042DC0000EE
:10AA60000000000017A80000F7B5150001938A68E0
:10AA70000B6900900C00934200DA130022002B6057
:10AA800043321278002A01D001332B6023689B06E1
:10AA900002D52B6802332B60062723681F4027D07E
:10AAA000230043331B785A1E93412268920630D408
:10AAB0002200019943320098089EB047431C25D0DC
:10AAC000062320682A68E16803400025042B03D18F
:10AAD0008D1AEB43DB171D40A3682269934201DD09
:10AAE0009B1AED180027BD4220D1002010E001374D
:10AAF000E3682A689B1ABB42D2DD22000123193287
:10AB000001990098089EB047431CF0D101204042B3
:10AB1000FEBD3020E1184331087021005A1C453138
:10AB20000978A218433202331170C1E722000123D1
:10AB30001A3201990098089EB047431CE6D00137AD
:10AB4000D1E70000F0B589B004920A0043320593C2
:10AB5000039002920A7E0C000E9B6E2A00D186E0C2
:10AB60001FD8632A33D008D8002A00D18CE0582A95
:10AB70004DD0250042352A7030E0642A01D0692A80
:10AB8000F7D1196825680A1D280629D508681A60B2
:10AB9000002803DA2D23029A404213706B4E0A27D5
:10ABA0004FE0732A74D008D86F2A1FD0702AE0D1E2
:10ABB000202209680A43226003E0752A16D0782A09
:10ABC000D7D12200782145321170614E22E0250054
:10ABD0001A684235111D196013682B70012365E056
:10ABE00008681A606906D3D500B2D1E719682568EC
:10ABF000081D186008682E0605D5544E08276F2AD0
:10AC00001BD00A2719E06D06F7D580B2F5E745316C
:10AC10004E4E0A7018682268011D006819601506FA
:10AC200021D5D30702D520231A43226010270028FC
:10AC300003D1202322689A43226023000022433359
:10AC40001A706368A360002B58DB042221689143CB
:10AC50002160002854D1029D002B5AD02500337862
:10AC600042352B7055E05506DBD580B2D9E71A681E
:10AC70000D68101D4969186013682E0601D519600A
:10AC800002E06D06FBD519800023029D23614FE091
:10AC90001A68111D1960156800216268280000F00B
:10ACA0009BFD002801D0401B606063682361002386
:10ACB000029A13703CE023692A0004990398059DC9
:10ACC000A847431C3ED023689B0715D4079BE06828
:10ACD000984239DA180037E022000123193204992A
:10ACE0000398059EB047431C2CD00135E368079AB2
:10ACF0009B1AAB42F0DCE9E70025F7E70028ADD06E
:10AD0000029D3900FDF722FC735C013D2B70002889
:10AD1000F7D1082F09D12368DB0706D563682269BC
:10AD2000934202DC3023013D2B70029B5B1B2361AD
:10AD3000059B07AA00932100049B0398FFF794FE4C
:10AD4000431CB8D10120404209B0F0BD49DC0000ED
:10AD50005ADC00000D4B70B51C680500A36B002B7E
:10AD60000FD1182000F01CFD094BA0630360094BB4
:10AD700001224360084B83600B238381002302611F
:10AD800043610022A36B1D615A6170BD7C000020ED
:10AD90000E33CDAB34126DE6ECDE0500124B10B570
:10ADA0001C68A36B002B0FD1182000F0F9FC0F4B8F
:10ADB000A06303600E4B012243600E4B83600B23A4
:10ADC0008381002302614361A46B0B4A206961699E
:10ADD0000A4BFDF7F7FC012200238018594120613E
:10ADE00061614800400810BD7C0000200E33CDABEF
:10ADF00034126DE6ECDE05002D7F954C2DF4515894
:10AE00000CB430B5164B9DB00C1E1D6808DA8B23B0
:10AE100001202B6040421DB030BC08BC02B0184776
:10AE2000822302A99B008B810023029008619C422F
:10AE300000D0631E8B604B6101235B42CB81209A63
:10AE400021AB2800019300F003FE431C01DA8B23A1
:10AE50002B60002CDFD00023029A1370DBE7C04682
:10AE60007C0000200EB400B50B499CB01DAB0290D5
:10AE70000690079104910948094904CB059100689F
:10AE800002A9019300F0E4FD0023029A13701CB0A4
:10AE900008BC03B01847C046FFFFFF7F7C000020BE
:10AEA0000802FFFF0EB4812370B59DB002AC21AD46
:10AEB0009B0040CDA3810290069000F081F80B4BDF
:10AEC000606063620023606109486363A364013BBF
:10AED000E38132002B0021000068019500F012FF91
:10AEE0001DB070BC08BC03B01847C0461DAF0000C1
:10AEF0007C00002070B50C000E25495F01F0E8F9D8
:10AF0000002803DB636D1B18636570BDA389024ACB
:10AF10001340A381F9E7C046FFEFFFFF0020704711
:10AF2000F8B51F008B8905000C001600DB0505D560
:10AF30000E23C95E0022022300F0B2FBA389054A5A
:10AF400028001340A38132000E23E15E3B0000F095
:10AF500067F9F8BDFFEFFFFF70B50C000E25495FE4
:10AF600000F09EFBA389421C03D1054A1340A38134
:10AF700070BD802252011343A3816065F8E7C0468B
:10AF8000FFEFFFFF10B50E23C95E00F0DBF910BD27
:10AF9000020010B51378541C002B05D1CC5CD4549E
:10AFA0000133002CFAD110BD2200F3E702780B78B0
:10AFB000002A03D0013001319A42F7D0D01A7047ED
:10AFC0000023C25C0133002AFBD1581E704730B504
:10AFD0000500002A00D130BD0C78013A6B1C2C70A2
:10AFE0000131002C05D19A189A42F4D01C7001331B
:10AFF000FAE71D00EDE710B50378002B0FD10B78B1
:10B000005A4253415B42184010BD0023CA5C002ADB
:10B01000FAD0C45C944201D10133F7E701300378E0
:10B02000002BF2D11800EFE7F0B51F000E0087B03B
:10B030000590019102920C98347800F020FB0822D0
:10B0400000194378751C134036D12D2C36D1B51C10
:10B0500074780126002F62D0102F09D1302C07D12F
:10B0600020222B789343582B54D110276C7802352B
:10B070002D4B3900F31818000393FDF767FA04917C
:10B0800001210023494202008C461800210030397A
:10B0900009291AD80C00A74223DD591C09D06346A0
:10B0A000824206D302D10499A14202DB01237843F4
:10B0B00020182C780135E9E72E00BCE72B2C01D0B5
:10B0C0001E00C7E7B51C7478FAE721004139192939
:10B0D00001D8373CDFE721006139192901D8573CF5
:10B0E000D9E75A1C08D1059A23331360029B0398B1
:10B0F000002B09D107B0F0BD002E00D04042029ACB
:10B10000002AF7D0002B01D06B1E0193029B019AFD
:10B110001A60EFE73024002FAAD10827A8E7302CC7
:10B120009ED00A27A4E7C046FFFFFF7F13B5054C5A
:10B130002468246A002C00D1034C0094FFF774FFAC
:10B1400016BDC0467C000020E000002037B513008B
:10B15000064A05001068046A002C00D1044C0A005D
:10B1600000942900FFF760FF3EBDC0467C00002030
:10B17000E0000020F8B505000E001400002804D0FF
:10B180008369002B01D100F0E7F9224B9C422DD1BD
:10B190006C68A369A360A3891B0731D52369002BC1
:10B1A0002ED023682269F7B2981A6369F6B28342F7
:10B1B00005DC2100280000F061F9002826D1A368F1
:10B1C0000130013BA36023685A1C22601F70636931
:10B1D000834204D0A389DB071AD50A2E18D1210097
:10B1E000280000F04BF9002812D00FE00A4B9C42D7
:10B1F00001D1AC68CDE7094B9C42CAD1EC68C8E7E5
:10B200002100280000F020F80028CAD0012676424C
:10B210003000F8BD8CDC0000ACDC00006CDC000011
:10B2200070B50500080011000022064C22601A00CB
:10B2300001F040FA431C03D12368002B00D02B609F
:10B2400070BDC046942F0020364B70B51D680600B7
:10B250000C00002D05D0AB69002B02D1280000F0B6
:10B260007BF9314B9C420FD16C680C23E25E93B2A8
:10B2700019072DD4D90611D409230120336037339F
:10B280001343A381404270BD284B9C4201D1AC685E
:10B29000EBE7274B9C42E8D1EC68E6E75B0713D568
:10B2A000616B002908D023004433994202D030005A
:10B2B00000F09EFA002363632422A3899343A381B1
:10B2C00000236360236923600823A2891343A381B9
:10B2D0002369002B0BD1A0218022A3898900920031
:10B2E0000B40934203D02100300000F015FA0123F7
:10B2F000A289134011D00023A36063695B42A3615C
:10B30000002023698342BED10C23E25E1306BAD526
:10B3100040231343A3810138B5E7920700D4636942
:10B32000A360EDE77C0000208CDC0000ACDC0000BA
:10B330006CDC000010B5062001F04AF8012001F095
:10B34000C1F90000002370B5064C05000800236019
:10B3500001F06AF9431C03D12368002B00D02B6055
:10B3600070BDC046942F0020F7B58A8905000C00F7
:10B37000130760D44B68002B04DC0B6C002B01DC42
:10B380000020FEBDE76A002FFAD000232E682B6054
:10B3900080235B01216A1A4034D0606DA3895B076A
:10B3A00006D56368C01A636B002B01D0236CC01AEA
:10B3B0000200216A00232800E76AB847A189431CDC
:10B3C00006D12B681D2B30D82B4ADA40D3072CD559
:10B3D0000023636023692360CB0405D5431C02D19D
:10B3E0002B68002B00D16065616B2E600029C7D0EF
:10B3F00023004433994202D0280000F0F9F90020DC
:10B400006063BEE701232800B847431CC6D12B6800
:10B41000002BC3D01D2B01D0162B01D12E60AFE71E
:10B420004023A2891343A381ABE740230B430120B0
:10B43000A3814042A5E70F69002FA1D00B680F60E0
:10B44000DB1B01930023920700D14B69A360019B92
:10B45000002B00DC94E7019B3A00216A2800A66AD1
:10B46000B047002803DC4023A2891343DFE7019B98
:10B470003F181B1A0193EAE7010040200B6970B5E1
:10B4800005000C00002B01D1002070BD002804D065
:10B490008369002B01D100F05FF80B4B9C4209D16E
:10B4A0006C680C22A35E002BEED021002800FFF771
:10B4B0005BFFEAE7054B9C4201D1AC68F1E7044B26
:10B4C0009C42EED1EC68ECE78CDC0000ACDC0000C8
:10B4D0006CDC0000002310B504000360436083604F
:10B4E00081814366C281036143618361190008223F
:10B4F0005C30FFF773F9054B24626362044BA3626F
:10B50000044BE362044B236310BDC046F5AE00005C
:10B5100021AF000059AF000085AF000010B502490F
:10B5200000F08CF810BDC0467DB4000070B56825F1
:10B530004A1E55430E002900743100F0A3F9041E81
:10B5400008D000212A00016046600C30A0606832FB
:10B55000FFF744F9200070BD836913B50400002B88
:10B5600028D18364C3640365134B144A1B68826249
:10B570000193984201D101238361200000F020F85B
:10B580006060200000F01CF8A060200000F018F8B7
:10B590000022E06004216068FFF79CFF012209217E
:10B5A000A068FFF797FF02221221E068FFF792FFE1
:10B5B0000123A36113BDC04634DC00001DB50000AB
:10B5C000F8B51C4B07001E68B369002B02D1300090
:10B5D000FFF7C2FF4836B4687368013B04D533688F
:10B5E000002B07D03668F6E70C22A55E002D0DD0A3
:10B5F0006834F2E704213800FFF798FF3060002834
:10B60000F0D10C2304003B602000F8BD20000A4B61
:10B61000656625606560A560E36025616561A5617B
:10B62000082229005C30FFF7D9F86563A563A5649B
:10B63000E564E9E734DC00000100FFFFF7B5040032
:10B640000700002601914834002C01D13000FEBDD6
:10B650006368A5680093009B013B009301D52468B3
:10B66000F2E7AB89012B08D90E22AB5E013304D07F
:10B6700029003800019B984706436835EBE7EC301A
:10B6800000687047044B1B681B6A002B00D1034BFA
:10B69000EC3318687047C0467C000020E0000020B2
:10B6A00070B50500080011000022064C22601A0047
:10B6B00000F0E2FF431C03D12368002B00D02B6075
:10B6C00070BDC046942F002070B50E001D000E23E3
:10B6D000C95E96B01400002907DA00232B60B389F5
:10B6E0001B0611D48023DB000FE06A4600F06EFFDA
:10B6F0000028F2DBF022019B12021340054A9B183E
:10B700005A4253412B60EDE740230020236016B0DE
:10B7100070BDC04600E0FFFFF7B502268B8905002B
:10B720000C00334206D023004733236023610123FA
:10B730006361F7BD01AB6A46FFF7C6FF00990700DA
:10B74000280000F09FF8002808D10C22A35E9A057B
:10B75000EFD4032293431E43A681E4E70F4BAB6271
:10B760008023A28920601343A381009B2061636131
:10B77000019B002B0DD00E23E15E280000F038FF66
:10B78000002806D00322A38993431A000123134300
:10B79000A381A0893843A081CBE7C0461DB5000036
:10B7A00010B5034B0100186800F06CF810BDC046DE
:10B7B0007C00002082B0002900D101A9101E06D013
:10B7C000002B06D013780B601078431E984102B00E
:10B7D000704702204042FAE7C9B28218904201D174
:10B7E0000020704703788B42FBD00130F6E7000061
:10B7F00070B50500002910D00C1F2368002B00DA5B
:10B80000E418280000F006FF1D4A1368002B05D13C
:10B8100063601460280000F0FEFE70BDA34209D9E9
:10B82000216860188342F3D118685B684118216071
:10B83000EEE713005A68002A01D0A242F9D919682C
:10B840005818A0420BD12068091858181960824274
:10B85000E0D110685268411819605A60DAE7A042D6
:10B8600002D90C232B60D5E721686018824203D1EE
:10B87000106852684118216062605C60CAE7C04687
:10B88000181C0020032370B5CD1C9D43083506000D
:10B890000C2D1ED20C25A9421DD8300000F0BAFE96
:10B8A000254A14682100002919D1244C2368002B53
:10B8B00003D1300000F020FD20602900300000F0AE
:10B8C0001BFD431C2BD10C233000336000F0A3FE82
:10B8D00003E0002DDFDA0C233360002070BD0B681D
:10B8E0005B1B19D40B2B03D90B60CC18256003E02C
:10B8F0004B688C420DD11360300000F08CFE2000AC
:10B9000007220B30231D9043C31AE7D05A42E2505E
:10B91000E4E763600C00EFE70C004968C3E703232A
:10B92000C41C9C43A042E1D0211A300000F0E4FC8A
:10B93000431CDBD1C7E7C046181C00201C1C00209C
:10B94000F8B507000D001600002905D11100FFF71A
:10B9500099FF04002000F8BD002A03D1FFF748FF3B
:10B960003400F7E700F058FE2C00B042F2D231006C
:10B970003800FFF787FF041EECD029003200FEF7E5
:10B9800011FF29003800FFF733FFE3E7F0B58E68B9
:10B9900085B007000C00039201939E423CD890238F
:10B9A0008A89DB001A4234D00325096923685B1AAF
:10B9B0000293636902985D43EB0F5D19019B6D1063
:10B9C00001331B18AB4200D91D00530532D52900A5
:10B9D0003800FFF757FF061E09D10C233B604023B8
:10B9E0000120A28940421343A38105B0F0BD029A11
:10B9F0002169FEF7D7FEA389144A1A408023134316
:10BA0000A381029B2661F61826606561019EED1AEE
:10BA1000A560019B9E4200D9019E320003992068D7
:10BA2000FEF7C9FEA36800209B1BA36023689E1934
:10BA30002660DAE72A003800FFF782FF061EE0D111
:10BA400021693800FFF7D4FEC7E7C0467FFBFFFF40
:10BA5000F0B59FB0029005938B890F0016001B066E
:10BA600011D50B69002B0ED14021FFF70BFF386079
:10BA70003861002805D10C23029A013813601FB0E9
:10BA8000F0BD40237B61002306AC63612033637605
:10BA90001033A37635002B78002B01D0252B46D10F
:10BAA000AB1B04930CD0320039000298FFF76EFFF5
:10BAB000431C00D1AEE06269049B94466344636119
:10BAC0002B78002B00D1A5E00122002352426260B6
:10BAD00002A9543252186E1C2360E360A3601370F5
:10BAE000A365317805225448FFF776FE751C0028BF
:10BAF0001FD12268D30604D5532302A95B18202145
:10BB00001970130704D5532302A95B182B21197050
:10BB100033782A2B16D0350000210A20E3682A78D2
:10BB20006E1C303A092A4ED9002918D010E0013590
:10BB3000B1E7414B2268C01A0123834013432360BD
:10BB40002E00CEE7059B191D1B680591002B01DB1C
:10BB5000099304E05B42E3600223134323602B78E4
:10BB60002E2B0AD16B782A2B35D1059B02351A1D55
:10BB70001B680592002B2BDB0793304E297803229C
:10BB80003000FFF729FE002806D04023801B8340A9
:10BB900022680135134323602978062228486E1C49
:10BBA0002176FFF719FE00283CD0264B002B25D12B
:10BBB0000722059B07339343083305936369039A70
:10BBC0009B18636166E7434301219B183500A6E794
:10BBD00001235B42D0E700230A201A00013563608D
:10BBE00029786E1C3039092903D9002BC5D007925A
:10BBF000C3E74243012352183500F1E705AB009338
:10BC00003A00114B2100029800E000BF0390039B13
:10BC10000133D3D1BB890B985B0600D42FE70120F9
:10BC200040422CE705AB00933A00074B21000298F5
:10BC3000FEF788FFEAE7C04638DC00003EDC000083
:10BC400042DC0000000000008DB9000070B5140057
:10BC50004B1C03D101256D42280070BD9389202221
:10BC60009343626BA381CEB2CDB26368002A10D039
:10BC7000A26B9A4207DD2368013B23601E70636854
:10BC800001336360E8E7210000F056FC0028F2D0A1
:10BC9000E0E721692268002907D0914205D2511EB0
:10BCA0000878A84201D12160EAE7236423004433E5
:10BCB00063630323A36323004633E2631E702360A0
:10BCC0000123DEE710B50C00496B00290ED02300DC
:10BCD0004433994201D0FFF78BFD0020236C606351
:10BCE0006360834202D0E36B236010BD23690120AF
:10BCF00023600023A289636020331343A381404261
:10BD0000F3E70000F0B5B94CC025A5440593002326
:10BD10000C004A934B93862107AB4C93BE230190B2
:10BD2000170004A8B24A490040185B00C250B14A4B
:10BD30006D0042513B78002B00D154E1FFF7A2FC8B
:10BD400008223B787E1CC01802934378134023D00E
:10BD50006368002B14DDFFF795FC082123681A782F
:10BD6000801842780A4201D13700E3E74B9A013349
:10BD7000029201324B9262682360013A6260E7E707
:10BD8000862204AB52009B185B5921000198029354
:10BD900098470028DFD0E7E7029A252A6DD149931A
:10BDA00047937B782A2B02D11A3B4793BE1C37005E
:10BDB0000A2239787B1C03930B00303B092B24D9D2
:10BDC0008D4E03223000FFF707FD002807D0012326
:10BDD000801B8340479A039F1343049247933B7809
:10BDE0007E1C672B35D8652B00D3BBE0472B14D8BE
:10BDF000452B00D3B6E0002B00D1F1E0252B3CD041
:10BE000003234D930733489369E0499B039F0493B1
:10BE10005343303B59184991CBE75B2B00D17DE070
:10BE200010D8582BECD1479A0292802202999200A6
:10BE30000A434792102248926E229A429B415B42EB
:10BE400003334BE0632B00D175E0642BD8D10A2279
:10BE5000F1E7702B38D008D86E2B00D173E03AD8B8
:10BE6000692BCDD100234893EAE7752BEFD0782BCF
:10BE7000D9D0732BC4D1022330E06368002B0FDDCF
:10BE8000236802991A788A4200D0ACE001336268D4
:10BE900023604B9B013A0293013362604B9363E74B
:10BEA000862204AB52009B185B5921000198039332
:10BEB00098470028E4D04A98002800D08CE0013848
:10BEC000A9239B009D44F0BD479A0292202202992B
:10BED0000A434792A7E708234893043B4D936368BE
:10BEE000002B41DD479B02935B0608D4FFF7CAFB9A
:10BEF000082123681A78801842780A4240D14D9B65
:10BF0000022B55DC05AB220047A9019800F078F818
:10BF1000012868D0022800D026E7CCE7310007A826
:10BF200000F0FCF9479B060002934023029A13435A
:10BF300047930123D2E7479B02934023029A13437E
:10BF400047930023CAE74798C30600D50CE7059B33
:10BF50004B9A191D05911B68C70701D51A8003E785
:10BF60001A6001E70523B9E7862204AB52009B184B
:10BF70005B5921000198029398470028B2D09AE7B4
:10BF80004B9A029201324B926268013A6260002A37
:10BF900002DD01332360A9E7862204AB52009B181F
:10BFA0005B59210001980293984700289ED082E7B0
:10BFB000042B06DC05AB220047A9019800F086F8A7
:10BFC000A6E70E4B002B00D1CEE605AB220047A919
:10BFD000019800E000BF9BE7A3895B0600D46FE7F0
:10BFE000012040426CE74A986AE7C0465CFDFFFFCB
:10BFF0004DBC0000C5BC00003EDC0000000000009D
:10C00000F7B515008A6801900C00002A04D18A69EE
:10C01000002A17D10132A2602268D20603D41A681E
:10C02000111D196017680026A369002B1FD0012B72
:10C030000BD12B6862691B78D35C002B17D1002EC3
:10C0400033D109E001225242E5E7022B06D0002E4F
:10C050002BD1A369012B28D10120FEBDFFF712FBD4
:10C0600008222B681B78C01843781342EFD11022A6
:10C0700023680136134203D12B681B783B700137CC
:10C080002A686B6801322A60A268013B013A6B6042
:10C09000A260002A09D0002BC6DCC0235B00E35855
:10C0A0002900019898470028BED010232268134029
:10C0B00006D1E2680132E260A269002A00D03B703A
:10C0C000236900209E192661C7E70000F0B50C0027
:10C0D0008BB00293784B0490160007AA23CB23C29F
:10C0E000764B0593A369032B01D1754B0593AE22C3
:10C0F0000020A3685200591E0390914205D95E3B6F
:10C10000FF3B03935E23FF33A36023001C330193A3
:10C11000D023002722681B0113432360019B009357
:10C12000336807A81978BB0002221858FFF754FBA0
:10C1300000282BD0012F62D16368002B06D1083371
:10C1400022686360F933FF33134323605D4B226839
:10C1500013402360A3685A1EA260002B16D03368D8
:10C160005A1C32601B78009A13707368551C013B8F
:10C170007360002B09DCC0235B00E3583100049896
:10C1800000939847002800D080E000950137032FE6
:10C19000C6D16368002B01D10A33636010210027E8
:10C1A00063686069C91A484BC91800F0B7F8009D68
:10C1B000A36822680093002B41D031686369087836
:10C1C0001B5C002B3BD0302829D180231B011A4255
:10C1D00025D0039B0137002B05D01A00009B013AA4
:10C1E00001330392A3607368013B7360002B1DDD74
:10C1F000336801333360A368013BA360D8E7022FA3
:10C20000A8D1C02180232268C90011409B00994217
:10C21000BFD1F13BFF3B6360F033134399E72B4BF6
:10C22000134023600B782B700135DCE7C0235B00E3
:10C23000E35831000498009398470028DBD0236826
:10C24000DB050ED5019B9D4207D9BE23013D5B0056
:10C250002978E358320004989847019B01209D42B9
:10C2600027D0102223681A401CD12A7063680199D4
:10C270000498059EB047029B21681B688A0607D573
:10C280001A1D02990A601B68186008E00027D6E7AB
:10C290001A1DCE07F5D502990A601B681880E3685D
:10C2A0000133E3600020019BED1A2369EF19DF19C8
:10C2B00027610BB0F0BDC046D4DC000019C50000FA
:10C2C0002DB10000FFFAFFFFE0DC0000FFF6FFFFEA
:10C2D00070B50500080011000022064C22601A000B
:10C2E00000F0D2F9431C03D12368002B00D02B604F
:10C2F00070BDC046942F0020002370B5064C050089
:10C300000800236000F0C8F9431C03D12368002B08
:10C3100000D02B6070BDC046942F002070B50B7804
:10C3200005005E2B18D04A1C002128006C1CFF342D
:10C3300001700130A042FBD1501E002B0BD0012018
:10C340004140E9541478501C2D2C0CD05D2C02D0A7
:10C35000002C05D1100070BD8A1C4B780121E4E748
:10C3600023000200EDE756785D2EF9D0B342F7DCEA
:10C3700002320133E9549E42FBDCE3E770B504006E
:10C380000D001F2904D9162303600120404270BD0F
:10C39000436C002B04D08A009B181A68002A08D12D
:10C3A000200000F031F82A000100200000F01AF807
:10C3B000EDE70020012AEAD0511C03D116230130F9
:10C3C0002360E4E7002428001C6090472000DEE79B
:10C3D00010B5034B01001868FFF7D0FF10BDC04631
:10C3E0007C000020002370B5064C050008001100F9
:10C3F000236000F039F9431C03D12368002B00D0DF
:10C400002B6070BD942F002010B500F01DF910BDF9
:10C41000F0B51F000E0085B00390019102920A98BA
:10C420003478FFF72CF9082200194378751C134063
:10C4300038D12D2C38D17478B51C01330093002FDE
:10C4400065D0102F09D1302C07D120222B789343AF
:10C45000582B57D110276C78023501203900404203
:10C46000FBF7EEFF0600012039004042FCF76EF8B2
:10C47000002301228C46180052422100303909293C
:10C4800017D80C00A74222DD002B1EDB13008642CA
:10C4900005D301D1A44502DB0123784320182C7871
:10C4A0000135EAE72E00BAE72B2CC7D1B51C74780A
:10C4B000C4E721004139192901D8373CE2E72100BE
:10C4C0006139192903D8573CDCE71300E7E7002B53
:10C4D00009DA22230120039A40421360029B002BB9
:10C4E0000AD105B0F0BD009A002A00D04042029A5D
:10C4F000002AF6D0002B01D06B1E0193029B019AFB
:10C500001A60EEE73024002FA7D10827A5E7302CCA
:10C510009BD00A27A1E7000013B5054C2468246AC4
:10C52000002C00D1034C0094FFF772FF16BDC046EB
:10C530007C000020E00000200B00F7B54D6B443379
:10C540000C009D421CD18026F6003100FFF79AF9BD
:10C55000002802D101204042FEBD23006063A66393
:10C5600046331A78104BC254230045331A780F4BC8
:10C57000C2542A780E4BC254C01820600020EBE74A
:10C580008E6B290073001A000193FFF7D9F9051E7D
:10C59000E0D08719010032003800FEF703F9019B53
:10C5A00027606563A363E9E7FF030000FE03000063
:10C5B000FD0300000B1E04D0FF2A04D98A23036068
:10C5C0008B3B180070470A700123FAE7002370B50F
:10C5D000064C050008001100236000F02DF8431CF4
:10C5E00003D12368002B00D02B6070BD942F002056
:10C5F000002370B5064C05000800236000F02CF8FD
:10C60000431C03D12368002B00D02B6070BDC046B3
:10C61000942F0020704770470B1F1B68181F002BBA
:10C6200001DA0B58C018704758220120014B4042D4
:10C630001A607047942F002058220120014B40427D
:10C640001A607047942F002058220120014B40426D
:10C650001A607047942F00205822024B00201A6065
:10C660007047C046942F002058220120014B4042C1
:10C670001A607047942F002058220120014B40423D
:10C680001A607047942F002058220120014B40422D
:10C690001A607047942F0020044A1368002B00D1C1
:10C6A000034B1818106018007047C046201C00206B
:10C6B000982F002058220120014B40421A607047F9
:10C6C000942F0020FEE7C046F8B5C046F8BC08BC71
:10C6D0009E467047F8B5C046F8BC08BC9E467047F9
:10C6E00064617461000000005CC70000EB010000A1
:10C6F00065C70000170400006DC70000290700008F
:10C7000074C700003908000079C70000DF0200008C
:10C7100084C700008304000089C70000B10900003D
:10C7200095C700001B0200009FC7000031060000F3
:10C73000ADC700009F05000072616E646F6D0061FF
:10C740006C6C006C6173740066616C73650074726C
:10C75000756500252E3135732E2E2E006D616B65AB
:10C760004C697374006164644C6173740064656C3B
:10C77000657465006A6F696E00636F707946726FE9
:10C780006D546F0066696E64006A6F696E537472EF
:10C79000696E677300756E69636F646541740075D7
:10C7A0006E69636F6465537472696E670066726563
:10C7B000654D656D6F727900F00F0000001000008C
:10C7C0001A10000098100000D010000006110000A0
:10C7D0003E11000064110000A0110000E2110000F1
:10C7E000381200007C120000E81200003013000034
:10C7F000561300008E130000D4130000FA1300003B
:10C80000281400005A1400009214000016150000AD
:10C81000DE15000054160000C016000014170000BA
:10C820003417000056170000081800004E180000CA
:10C83000C6180000F00F0000F00F0000F418000010
:10C840005C190000E0190000261A00006E1A0000B2
:10C85000E01A0000521B00009A1B0000E01B0000C1
:10C86000161C00005C1C0000A21C0000EA1C00005A
:10C870003E1D00009C1D0000DA1D0000441E00004B
:10C880007A1E0000C21E00000A1F0000521F000096
:10C890008C1F0000D41F00001C200000F00F0000BF
:10C8A000F00F0000F00F000084200000F00F0000E7
:10C8B000BA200000E62000001C21000048210000F2
:10C8C000F00F0000F00F0000F00F0000F00F00006C
:10C8D0007E210000CA210000F00F0000F00F0000D0
:10C8E000102200006022000086220000F00F0000ED
:10C8F000F00F0000F00F0000B4220000E42200005E
:10C90000142300004A23000074230000AA2300001F
:10C91000D4230000FC230000242400005424000041
:10C9200084240000AE240000D82400000825000064
:10C9300032250000F00F0000F00F0000F00F0000A3
:10C94000F00F0000F00F000062250000A825000095
:10C95000D4250000002600002C26000062260000DE
:10C9600098260000CE260000042700003027000093
:10C970005C27000092270000F00F0000F00F00007D
:10C98000F00F0000F00F0000F00F0000F00F0000AB
:10C99000F00F0000F00F0000F00F0000F00F00009B
:10C9A000F00F0000F00F0000F00F0000F00F00008B
:10C9B000BE270000F4270000282564206974656DF7
:10C9C000206C6973742900286F626A65637420742F
:10C9D0007970653A2025642900537461636B207572
:10C9E0006E646572666C6F770000000007000000DF
:10C9F0000300000035CA0000152900003DCA0000F0
:10CA0000C529000046CA00005D2A00004FCA000088
:10CA100019290000150000000100000002000000BC
:10CA200004000000050000000600000043616C6C7B
:10CA3000696F706500686173546F6E6500706C613A
:10CA400079546F6E6500686173536572766F007319
:10CA50006574536572766F00474320746F6F6B2067
:10CA600025642075736563733B20667265652025B8
:10CA70006420776F726473003C496E7465676572F9
:10CA80003E003C4F626A6563743E003C4C697374BF
:10CA90003E000D0A564D2050616E69633A202573A1
:10CAA0000D0A006D69736300B8CA00007934000094
:10CAB000C1CA00000D340000686578546F496E7477
:10CAC0000073696E000000003CCB0000E5340000FC
:10CAD00044CB0000E93400004ECB000007350000D5
:10CAE00057CB00001135000062CB00001B35000061
:10CAF0006ECB0000253500007ECB00002F350000F6
:10CB00008ECB000039350000A3CB00004335000078
:10CB1000B8CB00004D350000C4CB000057350000F5
:10CB2000D4CB000061350000E0CB0000F3340000FE
:10CB3000EDCB0000FD3400006E6574006861735732
:10CB40006946690073746172745769466900737449
:10CB50006F705769466900776966695374617475C7
:10CB600073006D7949504164647265737300737426
:10CB70006172744874747053657276657200737470
:10CB80006F7074487474705365727665720068745F
:10CB90007470536572766572476574526571756518
:10CBA000737400726573706F6E64546F4874747040
:10CBB000526571756573740068747470436F6E6E3E
:10CBC00065637400687474704973436F6E6E656357
:10CBD000746564006874747052657175657374006F
:10CBE00068747470526573706F6E736500687474E6
:10CBF00070436C6F7365000D0E0F04050C0B0A0675
:10CC0000070809000000000008080800080A4A4058
:10CC100000000A5FEA5FEA0ED92ED36E193244890A
:10CC2000330C924C924D0808000000048808080458
:10CC30000804848488000A448A4000048EC480006A
:10CC40000000048800000EC000000000080001225F
:10CC50004488100C9252524C048C84848E1C824C5A
:10CC6000901E1EC244924C06CA525FE21FF01EC1C3
:10CC70003E02448ED12E1FE24488100ED12ED12EBA
:10CC80000ED12EC488000800080000048004880229
:10CC900044880482000EC00EC008048244880ED16D
:10CCA00026C0040ED135B36C0C925ED2521C925C3D
:10CCB000925C0ED010100E1C9252525C1ED01C9032
:10CCC0001E1ED01C90100ED013712E12525ED25226
:10CCD0001C8808081C1FE242524C125498149210EF
:10CCE0001010101E113B75B131113935B3710C9212
:10CCF00052524C1C925C90100C92524C861C925CCE
:10CD000092510ED00C825C1FE484848412525252E1
:10CD10004C1131312A44113135BB7112524C9252AF
:10CD2000112A4484841EC488101E0EC808080E10E0
:10CD3000080482410EC242424E048A4000000000B4
:10CD400000001F0804800000000ED2524F10101C7B
:10CD5000925C000ED0100E02424ED24E0C925C90AD
:10CD60000E06C81C88080ED24EC24C10101C9252DF
:10CD70000800080808024002424C10149814920857
:10CD800008080806001B75B131001C925252000CB5
:10CD900092524C001C925C90000ED24EC2000ED0FB
:10CDA00010100006C8049808080EC8070012525256
:10CDB0004F0011312A4400113135BB00124C8C92C6
:10CDC00000112A4498001EC4881E06C48C8486085C
:10CDD0000808080818080C881800000C8360000078
:10CDE000000000000100000002000000030000003D
:10CDF000040000000500000006000000070000001D
:10CE000008000000090000000A0000000B000000FC
:10CE10000C0000000D0000000E0000000F000000DC
:10CE200010000000120000001400000016000000B6
:10CE3000180000001A0000001C0000001E00000086
:10CE40002000000023000000260000002900000050
:10CE50002C0000002F00000032000000360000000F
:10CE60003A0000003E0000004200000046000000C2
:10CE70004B00000050000000550000005A00000068
:10CE800061000000680000006F00000076000000F4
:10CE90007D000000840000008B0000009200000074
:10CEA00099000000A0000000A7000000AE000000F4
:10CEB000B5000000BC000000C3000000CA00000074
:10CEC000D1000000D8000000DF000000E6000000F4
:10CED000ED000000F4000000FB000000FF00000077
:10CEE00030CF0000853500003BCF0000D13A000074
:10CEF00045CF00004137000052CF0000413900000B
:10CF000059CF00009139000062CF0000E1390000E4
:10CF10006ECF0000DD3800007FCF0000B137000089
:10CF20008CCF00006D380000646973706C6179000B
:10CF30006C696768744C6576656C006D62446973F2
:10CF4000706C6179006D62446973706C61794F66D1
:10CF500066006D62506C6F74006D62556E706C6F20
:10CF600074006D62447261775368617065006D6230
:10CF70005368617065466F724C6574746572006EBB
:10CF8000656F506978656C53656E64006E656F50AF
:10CF90006978656C53657450696E004E6F742065D6
:10CFA0006E6F75676820726F6F6D206576656E2095
:10CFB000616674657220636F6D70616374696F6E12
:10CFC00000436F6D70616374656420466C617368C3
:10CFD00020636F64652073746F72650A2564206234
:10CFE0007974657320757365642028256425252967
:10CFF000206F6620256400426164207265636F7251
:10D000006420666F756E6420647572696E6720694E
:10D010006E697469616C697A6174696F6E00256408
:10D020002025642025642028256420776F7264738E
:10D0300029002564207265636F7264732C20256457
:10D0400020776F7264732C206D61784944202564C9
:10D050002C20636F6D70616374696F6E20637963F8
:10D060006C657320256400526573746F726564206B
:10D0700025642073637269707473005374617274F1
:10D08000656400726164696F000000002AD10000CD
:10D09000A144000037D100003D47000047D1000007
:10D0A000BD46000055D10000D148000060D100000D
:10D0B000C944000070D100005145000084D1000037
:10D0C0003945000093D10000B34A00009FD1000011
:10D0D000314A0000A8D10000D5490000B3D10000BA
:10D0E0001D490000BED1000059490000C7D1000011
:10D0F0008D490000D0D10000D9440000DFD10000EC
:10D10000B9440000E8D10000E94400006E756D628A
:10D110006572006E6F6E65006F7468657200706195
:10D12000697200737472696E670064697361626C1E
:10D1300065526164696F006D6573736167655265FF
:10D14000636569766564007061636B6574526563DD
:10D1500065697665007061636B657453656E640024
:10D160007265636569766564496E746567657200AA
:10D1700072656365697665644D657373616765544F
:10D180007970650072656365697665645374726968
:10D190006E670073656E64496E74656765720073CF
:10D1A000656E64506169720073656E645374726970
:10D1B0006E67007365744368616E6E656C007365BD
:10D1C0007447726F757000736574506F7765720085
:10D1D0007369676E616C537472656E67746800641E
:10D1E00065766963654944006C6173744D6573735A
:10D1F0006167654944000000000000009630077731
:10D200002C610EEEBA51099919C46D078FF46A703A
:10D2100035A563E9A395649E3288DB0EA4B8DC795A
:10D220001EE9D5E088D9D2972B4CB609BD7CB17EDA
:10D23000072DB8E7911DBF906410B71DF220B06AAA
:10D240004871B9F3DE41BE847DD4DA1AEBE4DD6DBA
:10D2500051B5D4F4C785D38356986C13C0A86B64BA
:10D260007AF962FDECC9658A4F5C0114D96C0663DA
:10D27000633D0FFAF50D088DC8206E3B5E10694CBA
:10D28000E44160D5727167A2D1E4033C47D4044BFA
:10D29000FD850DD26BB50AA5FAA8B5356C98B242DA
:10D2A000D6C9BBDB40F9BCACE36CD832755CDF455A
:10D2B000CF0DD6DC593DD1ABAC30D9263A00DE518A
:10D2C0008051D7C81661D0BFB5F4B42123C4B3567A
:10D2D0009995BACF0FA5BDB89EB802280888055FFA
:10D2E000B2D90CC624E90BB1877C6F2F114C68585A
:10D2F000AB1D61C13D2D66B69041DC760671DB0148
:10D30000BC20D2982A10D5EF8985B1711FB5B60619
:10D31000A5E4BF9F33D4B8E8A2C9077834F9000F59
:10D320008EA8099618980EE1BB0D6A7F2D3D6D08F9
:10D33000976C6491015C63E6F4516B6B62616C1CE9
:10D34000D83065854E0062F2ED95066C7BA5011B19
:10D35000C1F4088257C40FF5C6D9B06550E9B712B9
:10D36000EAB8BE8B7C88B9FCDF1DDD62492DDA1579
:10D37000F37CD38C654CD4FB5861B24DCE51B53A99
:10D380007400BCA3E230BBD441A5DF4AD795D83D99
:10D390006DC4D1A4FBF4D6D36AE96943FCD96E34D9
:10D3A000468867ADD0B860DA732D0444E51D0333B9
:10D3B0005F4C0AAAC97C0DDD3C710550AA410227C9
:10D3C00010100BBE86200CC925B56857B3856F2099
:10D3D00009D466B99FE461CE0EF9DE5E98C9D929F9
:10D3E0002298D0B0B4A8D7C7173DB359810DB42E39
:10D3F0003B5CBDB7AD6CBAC02083B8EDB6B3BF9A85
:10D400000CE2B6039AD2B1743947D5EAAF77D29D10
:10D410001526DB048316DC73120B63E3843B6494F0
:10D420003E6A6D0DA85A6A7A0BCF0EE49DFF0993F0
:10D4300027AE000AB19E077D44930FF0D2A3088760
:10D4400068F2011EFEC206695D5762F7CB67658010
:10D4500071366C19E7066B6E761BD4FEE02BD38910
:10D460005A7ADA10CC4ADD676FDFB9F9F9EFBE8E70
:10D4700043BEB717D58EB060E8A3D6D67E93D1A1B0
:10D48000C4C2D83852F2DF4FF167BBD16757BCA690
:10D49000DD06B53F4B36B248DA2B0DD84C1B0AAF30
:10D4A000F64A0336607A0441C3EF60DF55DF67A8B0
:10D4B000EF8E6E3179BE69468CB361CB1A8366BC40
:10D4C000A0D26F2536E2685295770CCC03470BBB90
:10D4D000B91602222F260555BE3BBAC5280BBDB290
:10D4E000925AB42B046AB35CA7FFD7C231CFD0B530
:10D4F0008B9ED92C1DAEDE5BB0C2649B26F263EC22
:10D500009CA36A750A936D02A906099C3F360EEB2F
:10D510008567077213570005824ABF95147AB8E2EF
:10D52000AE2BB17B381BB60C9B8ED2920DBED5E5CF
:10D53000B7EFDC7C21DFDB0BD4D2D38642E2D4F11F
:10D54000F8B3DD686E83DA1FCD16BE815B26B9F6AF
:10D55000E177B06F7747B718E65A0888706A0FFF0F
:10D56000CA3B06665C0B0111FF9E658F69AE62F8CF
:10D57000D3FF6B6145CF6C1678E20AA0EED20DD7CF
:10D580005483044EC2B30339612667A7F71660D0EF
:10D590004D476949DB776E3E4A6AD1AEDC5AD6D92F
:10D5A000660BDF40F03BD83753AEBCA9C59EBBDE4F
:10D5B0007FCFB247E9FFB5301CF2BDBD8AC2BACAFF
:10D5C0003093B353A6A3B4240536D0BA9306D7CD6F
:10D5D0002957DE54BF67D9232E7A66B3B84A61C48F
:10D5E000021B685D942B6F2A37BE0BB4A18E0CC34F
:10D5F0001BDF055A8DEF022D416C6C207461736B3B
:10D60000732073746F707065640076303737002054
:10D610002573202573004D656D6F727920636C65ED
:10D6200061726564004E6F20667265652074617377
:10D630006B20656E747269657300000084D600000B
:10D64000F55C000091D600005B5D00009DD60000F7
:10D650002B5D0000A3D600003B5D0000A9D60000B2
:10D660004B5D0000AFD600001D5A0000B9D6000087
:10D67000795D0000C1D60000495B000073656E73E0
:10D680006F727300616363656C65726174696F6E5C
:10D690000074656D70657261747572650074696C93
:10D6A00074580074696C74590074696C745A00740D
:10D6B0006F756368526561640069326352656164C5
:10D6C00000693263577269746500000040D700003A
:10D6D000015E00004ED70000055E000057D7000035
:10D6E000115E000061D70000155E00006AD70000DF
:10D6F000195E00006FD700001D5E000074D70000A7
:10D70000215E000080D70000255E000087D7000062
:10D71000295E000090D700002D5E000095D7000024
:10D72000315E0000A0D70000355E0000AAD70000DF
:10D73000095E0000B4D700000D5E0000746674003E
:10D74000656E61626C65446973706C6179006765D0
:10D7500074576964746800676574486569676874BC
:10D7600000736574506978656C006C696E65007251
:10D7700065637400726F756E6465645265637400EE
:10D78000636972636C6500747269616E676C6500D1
:10D790007465787400746674546F756368656400AA
:10D7A000746674546F7563685800746674546F754A
:10D7B00063685900746674546F756368507265735A
:10D7C000737572650057656C636F6D6520746F20AB
:10D7D0004D6963726F426C6F636B732100705F738E
:10D7E000706920213D204E554C4C002F686F6D65AF
:10D7F0002F72656E6172642F2E706C6174666F7229
:10D800006D696F2F7061636B616765732F667261FD
:10D810006D65776F726B2D61726475696E6F6E6F77
:10D82000726469636E7266352F6C696272617269C7
:10D8300065732F5350492F5350492E637070005316
:10D840005049436C6173733A3A535049436C617366
:10D8500073284E52465F5350495F547970652A2CA5
:10D860002075696E74385F742C2075696E74385F2A
:10D87000742C2075696E74385F74290000000000F4
:10D880000000000039600000F55F00001B60000030
:10D89000256000002F6000001960000000000000FB
:10D8A000010000000200000016000000040000005B
:10D8B000050000000600000007000000080000004E
:10D8C000090000000A0000000B0000000C0000002E
:10D8D0000D0000000E0000000F0000001A00000004
:10D8E0001B000000140000001300000011000000E5
:10D8F00003000000100000001C0000001D000000DC
:10D900001E000000120000001500000017000000BB
:10D9100018000000190000000000000000000000D6
:10D92000E9640000196C0000696500007D65000075
:10D9300073650000E5640000D9640000896500009B
:10D9400005650000D56400000000000000003043C1
:10D9500000000000000030C373717274000000000A
:10D96000FB21F93FFB2109407CD91240FB211940E2
:10D970007A6A1F407CD92240BBFD2540FB2129400B
:10D980003A462C407A6A2F405C4731407CD932407D
:10D990009C6B3440BBFD3540DB8F3740FB21394069
:10D9A0001BB43A403A463C405AD83D407A6A3F4020
:10D9B0004C7E40405C4741406C1042407CD9424024
:10D9C0008CA243409C6B4440AC344540BBFD454079
:10D9D000CBC64640DB8F4740EB584840FB214940CF
:10D9E00083F9A200444E6E00FC291500D157270090
:10D9F000DD34F50062DBC0003C99950041904300A6
:10DA00006351FE00BBDEAB00B761C5003A6E240077
:10DA1000D24D42004906E00009EA2E001C92D100D6
:10DA2000EB1DFE0029B11C00E83EA700F535820081
:10DA300044BB2E009CE98400B4267000417E5F0048
:10DA4000D6913900538339009CF439008B5F8400F0
:10DA500028F9BD00F81F3B00DEFF97000F98050076
:10DA6000112FEF000A5A8B006D1F6D00CF7E36001C
:10DA700009CB2700464FB7009E663F002DEA5F00A6
:10DA8000BA277500E5EBC7003D7BF100F7390700C9
:10DA900092528A00FB6BEA001FB15F00085D8D00A7
:10DAA000300356007BFC4600F0AB6B0020BCCF007F
:10DAB00036F49A00E3A91D005E619100081BE600A0
:10DAC00085996500A0145F008D40680080D8FF0034
:10DAD00027734D0006063100CA561500C9A8730009
:10DAE0007BE260006B8CC00000000040FB21F93F2E
:10DAF000000000002D44743E000000809846F83C71
:10DB00000000006051CC783B00000080831BF0399E
:10DB10000000004020257A38000000802282E33691
:10DB2000000000001DF36935020000000300000042
:10DB3000040000000600000010890000BA88000000
:10DB4000BA880000E8890000B6880000B6880000A6
:10DB5000DE890000E8890000B6880000DE89000048
:10DB6000B6880000E8890000EC890000EC8900001C
:10DB7000EC890000F4890000EC9300005E92000044
:10DB8000A292000006920000A29200009293000070
:10DB9000A2920000069200005E9200005E920000D9
:10DBA0009293000006920000FE910000FE9100009A
:10DBB000FE910000A0930000149B0000169A000044
:10DBC000169A0000349D0000109A0000109A000080
:10DBD0001C9D0000349D0000109A00001C9D000058
:10DBE000109A0000349D00002A9D00002A9D00002C
:10DBF0002A9D0000389D00002C2066756E637469B4
:10DC00006F6E3A2000617373657274696F6E2022C3
:10DC1000257322206661696C65643A2066696C65CB
:10DC200020222573222C206C696E652025642573C3
:10DC300025730A0080000020232D302B2000686C03
:10DC40004C0065666745464700303132333435361F
:10DC50003738394142434445460030313233343558
:10DC60003637383961626364656600000000000081
:10DC700000000000000000000000000000000000A4
:10DC80000000000000000000000000000000000094
:10DC90000000000000000000000000000000000084
:10DCA0000000000000000000000000000000000074
:10DCB0000000000000000000000000000000000064
:10DCC0000000000000000000000000004300504F72
:10DCD00053495800F2DC0000F5DC0000F8DC0000DD
:10DCE000412D46612D66383930313233343536377F
:10DCF0005D002B2D003030007858000020202020BF
:10DD000020202020202828282828202020202020EB
:10DD100020202020202020202020202088101010CB
:10DD20001010101010101010101010100404040423
:10DD30000404040404041010101010101041414198
:10DD40004141410101010101010101010101010103
:10DD50000101010101010110101010101042424296
:10DD600042424202020202020202020202020202D3
:10DD70000202020202020210101010200000000035
:10DD80000000000000000000000000000000000093
:10DD90000000000000000000000000000000000083
:10DDA0000000000000000000000000000000000073
:10DDB0000000000000000000000000000000000063
:10DDC0000000000000000000000000000000000053
:10DDD0000000000000000000000000000000000043
:10DDE0000000000000000000000000000000000033
:10DDF0000000000000000000000000000000000023
:08DE00000823FF7F0100000070
:10DE0800FFFFFFFF4006000001000000E803DC05FB
:10DE1800DC05DC05DC050000FFFFFFFFFFFFFFFF5F
:10DE28001800000019FCFFFFFFFFFFFF02000000C1
:10DE380003000000FFFFFFFF0000000001000000DA
:10DE48000000020001000000FFFFFFFF00000000CB
:10DE5800020000000000040002000000FFFFFFFFB6
:10DE6800000000000300000000000800030000009C
:10DE78000A000000080000000100000080000020E7
:10DE8800000000008CDC0000ACDC00006CDC000052
:10DE9800000000000000000000000000000000007A
:10DEA800000000000000000000000000000000006A
:10DEB800000000000000000000000000000000005A
:10DEC800000000000000000000000000000000004A
:10DED800000000000000000000000000000000003A
:10DEE80043000000000000000000000000000000E7
:10DEF800000000000000000000000000000000001A
:10DF080043000000000000000000000000000000C6
:10DF180000000000000000000000000000000000F9
:10DF280043000000000000000000000000000000A6
:10DF380000000000000000000000000000000000D9
:10DF48004300000000000000000000000000000086
:10DF580000000000000000000000000000000000B9
:10DF68004300000000000000000000000000000066
:10DF78000000000000000000000000000000000099
:10DF88004300000000000000000000000000000046
:10DF98000000000000000000000000000000000079
:10DFA8004300000000000000000000000000000026
:10DFB8000000000000000000000000000000000059
:10DFC800B5C50000B5B7000000000000FBDC00008C
:10DFD8005AC70000A2CA0000A2CA0000A2CA0000D4
:10DFE800A2CA0000A2CA0000A2CA0000A2CA000079
:10DFF800A2CA0000A2CA0000FFFFFFFFFFFFFFFF49
:10E00800FFFFFFFFFFFF00000100415343494900A4
:10E0180000000000000000000000000000000000F8
:10E02800000000000000000000004153434949007F
:10E0380000000000000000000000000000000000D8
:10E04800000000000000000000000000E9000000DF
:10E05800C55F00000D63000035680000C1000000C6
:04000003000063A9ED
:00000001FF
